:10000000000003208DC4010071C4010029C4010057
:1000100029C4010029C4010029C4010029C4010028
:1000200029C4010029C4010029C4010071C40100D0
:1000300071C4010029C4010045B90100BDBB010024
:1000400071C4010071C4010071C4010071C40100D8
:1000500071C4010071C4010071C4010071C40100C8
:1000600071C4010071C4010071C4010071C40100B8
:1000700071C4010071C4010071C4010071C40100A8
:1000800071C4010071C4010071C4010071C4010098
:1000900071C4010071C4010071C4010071C4010088
:1000A00081830100DD84010071C4010071C401007D
:1000B00071C4010071C4010071C40100E1D60100E6
:1000C00071C40100CDFE010071C4010029000200CD
:1000D00071C401005901020071C4010071C4010022
:1000E00071C4010071C4010071C4010071C4010038
:1000F00071C4010071C4010071C4010071C4010028
:1001000071C4010071C4010071C4010071C4010017
:1001100071C4010091DF010071C4010071C40100CC
:1001200071C4010071C4010071C4010071C40100F7
:1001300071C4010071C4010071C4010071C40100E7
:1001400091B6010071C401008902020071C401006E
:1001500071C4010071C4010071C4010071C40100C7
:1001600071C4010071C401003986010071C401002D
:1001700071C4010071C4010071C4010071C40100A7
:1001800071C40100994D010071C4010071C40100E6
:1001900071C4010071C40100B903020071C40100FF
:1001A00071C4010071C4010071C4010071C4010077
:1001B00071C4010071C4010071C4010071C4010067
:1001C00071C4010071C4010071C4010071C4010057
:1001D000FFFFFFFFFFFFFFFFFFFFFFFFFFFFFFFF2F
:10040000FFFFFFFFFFFFFFFFFFFFFFFFDEF9FFFF23
:1004100010B5054C237833B9044B13B10448AFF33E
:1004200000800123237010BD00F0002000000000B8
:10043000E46F0200084B10B51BB108490848AFF340
:1004400000800848036803B910BD074B002BFBD0A0
:10045000BDE81040184700BF0000000004F0002075
:10046000E46F020034EC002000000000704700BF81
:1004700010B54FF4097104461CF0CCF9204610BDAC
:1004800070B54FF06A522DED028B064644F6587354
:1004900008EE902A40F6DB72C0F202034FF61A050E
:1004A00040F6DA70C4F24902C2F20005C3F64920F0
:1004B00008EE102A336000240FE007EE904AF8EEB1
:1004C000E77A77EE807A67EEA87A67EE887A27EE89
:1004D000800A20F099FA10EE100A23F057FA41EC46
:1004E000100B20F0F9F800230022CCF2900351EC1D
:1004F000100B23F09FFA41EC100B20F001F951ECA6
:10050000100B23F06FFD0134B4F5806FB6EE000AD6
:1005100025F8020FD1D14FF06A534FF21A0508EEB9
:10052000103AC2F20005002407EE904AF8EEE77A8E
:10053000013467EE887A17EE900A23F027FA9FEDD0
:10054000140B41EC110B20F05FFB002351EC100B5E
:100550000022C3F6F07323F0B9F800230022C4F29E
:10056000B00323F067FA23F05DFD23F00FFA41ECAE
:10057000100B20F0C5F851EC100B23F033FDB4F54F
:10058000806F25F8020FCFD1BDEC028B304670BDD5
:100590000000000000000040704700BF10B54FF49D
:1005A000097104461CF036F9204610BD2DE9F04FC4
:1005B0004DF6A466C2F200060A9D0B989DF83070B5
:1005C000B6F800C044F67074C0F20204C5EB000A2D
:1005D000002F18BF0C466FEA0C0B0AF1200A4DF6EB
:1005E000A4294DF6A448043A271FA1F1040E0FFADE
:1005F0008BFB4FEAAA1AC2F20009C2F200080026D9
:1006000027E0B4F5007F02D08CB3C943C9B239F8F2
:1006100011104CEA010101EBC00080B20BEA0004AA
:10062000E143C9B2241238F8111001F58061490084
:10063000E14010EA0C0F18BFC94357F8044F09985E
:1006400009B2013604EB8131402E03444EF8041FF9
:1006500010D052F8041F1944891301F44074554412
:10066000B4F5807FC9B2A8B2CBD1C943C9B239F8B9
:100670001110D0E7BDE8F08F2DE9F04F4DF6A465DD
:10068000C2F2000509982E880A9D9DF82C7044F648
:100690007074C0F20204C0EB050E002F14BF0F46A9
:1006A00027466FEA06090EF1200E4DF6A4284DF6F6
:1006B000A44C3C1F0D1F0FFA89F9FC374FEAAE1E00
:1006C000C2F20008C2F2000C2AE0BBF5007F04D0A1
:1006D000BBF1000F30D0C943C9B238F81110314313
:1006E00001EBCA0A1FFA8AFA09EA0A0B6FEA0B0140
:1006F000C9B24FEA2B2B3CF8111001F5806149007B
:100700001AEA060F21FA0BF154F804AF18BFC943D7
:1007100009B20AEB8131BC421A4445F8041F0ED0DD
:10072000911301F4407B7044BBF5807F1FFA80FA7F
:10073000C9B2CAD1C943C9B238F81110D0E7BDE86F
:10074000F08F00BF2DE9F04F4DF6A46083B0C2F2E8
:1007500000000D9EB0F800C00C9C9DF840A00F9FBB
:100760000E980E9D019344F6707EC0F2020EC4EB0B
:10077000060B6FEA0C06BAF1000F14BF8A46F24668
:1007800033B20BF1200B4DF6A4294DF6A448AAF183
:10079000040600686D680093A1F1040E0AF1FC0ADA
:1007A0004FEAAB1B0137C2F20009C2F2000829E090
:1007B000B0F5007F02D098B3DB43DBB239F81330D9
:1007C0004CEA030303EBC101009B89B203EA010079
:1007D000C343DBB2001238F8133003F580635B00CB
:1007E000C34011EA0C0F18BFDB4356F8041F0198F1
:1007F0001BB29B031944564502444EF8041F284679
:1008000011D01D4643193B4113449B1303F4407020
:100810005C44B0F5807FDBB2A1B2C9D1DB43DBB26F
:1008200039F81330CEE70E9A1560536003B0BDE877
:10083000F08F00BF2DE9F04F46F2302403EB430365
:10084000C0F2020404EBC3050646144689460FCDE8
:1008500091B00AAF0FC795E80300002387E80300B3
:10086000012704F160088DF8247007978DF8253072
:100870008DF826300AAD48E00AF1FF3101EB011195
:1008800006EB0111133121F00F0194E80140C0146F
:10089000C0F500706060BEF1000F3FD0BEF5FE7F76
:1008A0003EDA10AFBA441AF81CCCBCF1000F04D0E9
:1008B00012F1000C18BF4FF0010CC3F301123AB152
:1008C00010AF07EB020B1BF81CBCBBF1000F34D1BF
:1008D00003F0C003C02B02D11B9B0F2B41DDA3688B
:1008E000E2680190CDF808C0CDF800E03046FFF78F
:1008F000C3FE9DF81C300AF81C3CE368A26803EBB9
:100900008213E3601034A04514D055F8043B13F073
:10091000030A03F00402AFD14946B6E740F2FF1ED6
:10092000B0F5FE7FBDDB002AE7D110AB9A440AF890
:100930001C2CE2E711B0BDE8F08F013A02EB021285
:10094000E368CDF80CC006EB02120290CDF804E08B
:10095000A0680090133222F00F023046FFF726FE07
:10096000C7E71F46E268A36803971A9F0190CDF876
:1009700010C00297CDF800E03046FFF7E3FEB8E77D
:1009800000207047704700BF704700BF704700BF2E
:10099000704700BF704700BF10B504461AF0FAFD5B
:1009A000204610BD10B5044624F00AF80146204642
:1009B000BDE810401FF08EB810B5044624F000F8D2
:1009C000014620461FF086F804464EF24020C2F24F
:1009D00000001BF0E9F9204410BD00BF45F20810EB
:1009E00008B51621C0F202001FF074F841F2C050A1
:1009F000C2F201004FF20F6119F0FCFC45F2201029
:100A00001421C0F202001FF065F84FF20F601EF0D3
:100A1000D7F945F23810C0F202000F211FF05AF842
:100A20004EF24020C2F20000BDE808401BF0BCB905
:100A300045F2481008B51521C0F202001FF04AF82F
:100A400041F67863C2F20103FA21986C03681B68CF
:100A5000984745F260100F21C0F202001FF03AF8EB
:100A60004FF60F201EF0ACF945F23810C0F202002C
:100A70000F211FF02FF84EF24020C2F20000BDE817
:100A800008401BF091B900BF45F2701008B518215D
:100A9000C0F202001FF01EF841F67863C2F20103B3
:100AA000FB21986C03681B68984745F260100F2182
:100AB000C0F202001FF00EF84FF60F301EF080F962
:100AC00045F23810C0F202000F211FF003F84EF279
:100AD0004020C2F20000BDE808401BF065B900BF2D
:100AE00045F28C1008B51421C0F202001EF0F2FF8E
:100AF00041F67863C2F20103FC21986C03681B681D
:100B0000984745F260100F21C0F202001EF0E2FF8C
:100B10004FF60F401EF054F945F23810C0F20200B3
:100B20000F211EF0D7FF4EF24020C2F20000BDE8B8
:100B300008401BF039B900BF45F2A41008B51D21CB
:100B4000C0F202001EF0C6FF41F67863C2F2010354
:100B5000FE21986C03681B68984745F260100F21CE
:100B6000C0F202001EF0B6FF4FF60F601EF028F92B
:100B700045F23810C0F202000F211EF0ABFF4EF21A
:100B80004020C2F20000BDE808401BF00DB900BFD4
:100B900038B545F2C4104EF2402541F29054102170
:100BA000C2F20104C2F20005C0F202001EF092FF80
:100BB00028461BF0F9F820680EF0A2FE20680EF01F
:100BC000ABFD20680EF0BCFD45F2D8101B21C0F231
:100BD00002001EF07FFF41F67863C2F20103FF219D
:100BE000986C03681B68984745F260100F21C0F2AB
:100BF00002001EF06FFF4FF60F701EF0E1F845F295
:100C00003810C0F202000F211EF064FF2846BDE834
:100C100038401BF0C9B800BF10B50446240445F2A3
:100C2000F41004F4FE041521C0F2020044F47344ED
:100C30001EF050FF44F0020441F2C0502146C2F2BF
:100C4000010019F0D7FB45F220101421C0F2020078
:100C50001EF040FF20461EF0B3F845F23810C0F2F7
:100C600002000F211EF036FF4EF24020C2F20000BB
:100C7000BDE810401BF098B845F20C2008B51021D3
:100C8000C0F202001EF026FF41F2C050C2F2010085
:100C90004FF60F2119F0AEFB45F220101421C0F2DF
:100CA00002001EF017FF4FF60F201EF089F845F2E4
:100CB0003810C0F202000F211EF00CFF4EF240204F
:100CC000C2F20000BDE808401BF06EB845F22020DB
:100CD00008B50F21C0F202001EF0FCFE41F2C05028
:100CE000C2F201004FF60F4119F084FB45F22010CB
:100CF0001421C0F202001EF0EDFE4FF60F401EF070
:100D00005FF845F23810C0F202000F211EF0E2FE3B
:100D10004EF24020C2F20000BDE808401BF044B88B
:100D200045F2302008B51321C0F202001EF0D2FEB9
:100D300041F2C050C2F201004FF60F3119F05AFBD8
:100D400045F220101421C0F202001EF0C3FE4FF63F
:100D50000F301EF035F845F23810C0F202000F21B6
:100D60001EF0B8FE4EF24020C2F20000BDE808407E
:100D70001BF01AB845F2442008B51821C0F2020051
:100D80001EF0A8FE41F2C050C2F201004FF60F6102
:100D900019F030FB45F220101421C0F202001EF0C1
:100DA00099FE4FF60F601EF00BF845F23810C0F2B6
:100DB00002000F211EF08EFE4EF24020C2F2000013
:100DC000BDE808401AF0F0BF38B505464EF24024A1
:100DD00045F26020C2F200041E21C0F202001EF0A3
:100DE00079FE294600230A2220461AF0EFFF45F239
:100DF00080200E21C0F202001EF06CFE4DF6A863AA
:100E0000C2F200030A22197C204600231AF0DEFFFA
:100E100045F290200121C0F202001EF05BFE204648
:100E20001AF0C2FF002038BD38B545F2C4104EF2AA
:100E3000402541F290541021C2F20104C2F2000593
:100E4000C0F202001EF046FE28461AF0ADFF2068F0
:100E50000EF056FD20680EF05FFC20680EF070FC6E
:100E600045F294201621C0F202001EF033FE41F23A
:100E7000C050C2F201004FF60F7119F0BBFA45F2F3
:100E800020101421C0F202001EF024FE4FF60F7055
:100E90001DF096FF45F23810C0F202000F211EF03F
:100EA00019FE2846BDE838401AF07EBF45F2AC2056
:100EB00008B51B21C0F202001EF00CFE41F678635B
:100EC000C2F20103F621986C0368DB6C984745F287
:100ED00060100F21C0F202001EF0FCFD4FF20F6007
:100EE0001DF06EFF45F23810C0F202000F211EF017
:100EF000F1FD4EF24020C2F20000BDE808401AF0B9
:100F000053BF00BF10B5044645F2C8201F21C0F2F0
:100F1000020004F00F041EF0DDFD44F010044FF257
:100F2000021343EA044441F2C0502146C2F20100D8
:100F300019F060FA45F220101421C0F202001EF0F0
:100F4000C9FD20461DF03CFF45F23810C0F20200FA
:100F50000F211EF0BFFD4EF24020C2F20000BDE89E
:100F600010401AF021BF00BF45F2E82008B5182153
:100F7000C0F202001EF0AEFD41F67863C2F201033A
:100F8000FE21986C03681B68984745F260100F219A
:100F9000C0F202001EF09EFD41F2C050C2F20100FC
:100FA0004FF60F6119F026FA45F22010C0F2020048
:100FB00014211EF08FFD4EF24020C2F20000BDE869
:100FC00008401AF0F1BE00BF45F2043008B50F2109
:100FD000C0F202001EF07EFD41F67863C2F201030A
:100FE000FC21986C03681B68984745F260100F213C
:100FF000C0F202001EF06EFD41F2C050C2F20100CC
:101000004FF60F4119F0F6F945F22010C0F2020038
:1010100014211EF05FFD4EF24020C2F20000BDE838
:1010200008401AF0C1BE00BF45F2143008B51021C7
:10103000C0F202001EF04EFD41F67863C2F20103D9
:10104000FA21986C03681B68984745F260100F21DD
:10105000C0F202001EF03EFD41F2C050C2F201009B
:101060004FF60F2119F0C6F945F22010C0F2020028
:1010700014211EF02FFD4EF24020C2F20000BDE808
:1010800008401AF091BE00BF45F2283008B5132180
:10109000C0F202001EF01EFD41F67863C2F20103A9
:1010A000FB21986C03681B68984745F260100F217C
:1010B000C0F202001EF00EFD41F2C050C2F201006B
:1010C0004FF60F3119F096F945F22010C0F20200E8
:1010D00014211EF0FFFC4EF24020C2F20000BDE8D9
:1010E00008401AF061BE00BF38B545F2C4104EF298
:1010F000402541F290541021C2F20104C2F20005D1
:10110000C0F202001EF0E6FC28461AF04DFE2068F0
:101110000EF0F6FB20680EF0FFFA20680EF010FBD0
:1011200045F23C301621C0F202001EF0D3FC41F61D
:101130007863C2F20103FF21986C03681B6898472B
:1011400045F260100F21C0F202001EF0C3FC41F214
:10115000C050C2F201004FF60F7119F04BF945F281
:101160002010C0F2020014211EF0B4FC2846BDE895
:1011700038401AF019BE00BF45F2543008B51621A8
:10118000C0F202001EF0A6FC41F67863C2F2010331
:10119000F621986C0368DB6C984745F260100F21CC
:1011A000C0F202001EF096FC41F2C050C2F20100F3
:1011B0004FF20F6119F01EF945F22010C0F2020043
:1011C00014211EF087FC4EF24020C2F20000BDE860
:1011D00008401AF0E9BD00BFF8B5064645F26C308C
:1011E0000C46C0F20200122115461EF073FC711E5F
:1011F000C9B20F2915D841F67867C2F2010741F04C
:10120000A001B86C03681B689847B86C036804F0C9
:101210007F011B689847B86C036805F07F011B6865
:10122000984745F280300A21C0F202001EF052FCBD
:101230006B1E1B02240404F4FE0403F470632343B6
:10124000310143F4504343F00D03C9B241F2C050A1
:101250001943C2F2010019F0CDF845F22010C0F296
:10126000020014211EF036FC4EF24020C2F20000B3
:10127000BDE8F8401AF098BD1F2970B50C46054628
:1012800008D84DF6A863C2F2000318790FF020FBCE
:101290000BF08AF845F28C300D21013DC0F20200BE
:1012A0001EF018FCE9B20F290FD841F67866C2F299
:1012B000010641F0C001B06C03681B689847B06C30
:1012C000036804F07F011B68984745F260100F2106
:1012D000C0F202001EF0FEFB230403F4FE03290209
:1012E00043F4404343F00C0301F4706141F2C050F9
:1012F0001943C2F2010019F07DF845F22010C0F246
:10130000020014211EF0E6FB4EF24020C2F2000063
:10131000BDE870401AF048BDF8B54DF6A863C2F2BA
:1013200000030E461B7C1446054623B1984202D0AA
:10133000FFF74AFD38B141F29053C2F20103314642
:1013400018680EF0B3F845F29C301221013DC0F24E
:1013500002001EF0BFFBE9B20F2915D841F67867ED
:10136000C2F2010741F08001B86C03681B6898471E
:10137000B86C036806F07F011B689847B86C036877
:1013800004F07F011B68984745F260100F21C0F2FE
:1013900002001EF09FFB230603F0FE43310443F4DA
:1013A000004301F4FE012D0243F008030B4341F218
:1013B000C05005F470611943C2F2010019F01AF827
:1013C00045F22010C0F2020014211EF083FB4EF201
:1013D0004020C2F20000BDE8F8401AF0E5BC00BFB2
:1013E000F8B54DF6A863C2F200030E461B7C144606
:1013F000054623B1984202D0FFF7E6FC40B141F226
:101400009053C2F201032246186831460DF00EFED9
:1014100045F2B0301121013DC0F202001EF05AFB2E
:10142000E9B20F2915D841F67867C2F2010741F0F9
:101430009001B86C03681B689847B86C036806F0A5
:101440007F011B689847B86C036804F07F011B6834
:10145000984745F260100F21C0F202001EF03AFBDF
:10146000230603F0FE43310443F4104301F4FE016C
:101470002D0243F009030B4341F2C05005F47061A3
:101480001943C2F2010018F0B5FF45F22010C0F276
:10149000020014211EF01EFB4EF24020C2F200009A
:1014A000BDE8F8401AF080BCF8B541F29053C2F2A2
:1014B000010305461B6801F5005645F2C4300C4691
:1014C000013D0D21C3F8C060C0F202001EF002FB16
:1014D000E9B20F2915D841F67867C2F2010741F049
:1014E000E001B86C03681B689847B86C036806F0A5
:1014F0007F011B689847B86C0368C6F3C6111B6868
:10150000984745F2601004F30D040F2104F50054D0
:10151000C0F202001EF0DEFA2902230403F4FE03E7
:1015200001F47061194341F46041640404F0FE4425
:1015300041F00E0141F2C0502143C2F2010018F007
:1015400059FF45F22010C0F2020014211EF0C2FA29
:101550004EF24020C2F20000BDE8F8401AF024BC70
:10156000F0B54AF23472C2F2010283B040F2706305
:1015700011680091C2F2010300991E68126801927D
:1015800041F28855C2F2010541F25452C2F2010201
:10159000891B45F2D4304EF24024C2F20004019F70
:1015A000298000260C21C0F2020016701F601EF078
:1015B00091FA2B8820464EF6602191FBF3F11AF048
:1015C00095FB45F2E4300521C0F202001EF082FADC
:1015D000298820461AF08AFB45F2EC300F21C0F230
:1015E00002001EF077FA20461AF0DEFB03B0F0BDD1
:1015F00008B541F25451C2F201014AF6AB230A7810
:101600000132D2B2CAF6AA23A3FB02031B0903EBE1
:101610004303A2EBC30313F0FF0F0A7001D1FFF7DE
:101620009FFF45F2FC301021C0F202001EF052FA7A
:1016300041F2C050C2F201004FF60F0118F0DAFE7D
:1016400045F220101421C0F202001EF043FA4FF6BA
:101650000F001DF0B5FB45F23810C0F202000F215B
:101660001EF038FA4EF24020C2F20000BDE80840F9
:101670001AF09ABB08B541F25451C2F201014AF680
:10168000AB230A780132D2B2CAF6AA23A3FB020323
:101690001B0903EB4303A2EBC30313F0FF0F0A7014
:1016A00001D1FFF75DFF45F210401521C0F20200A5
:1016B0001EF010FA41F67863C2F20103F821986C2B
:1016C00003681B68984745F260100F21C0F20200C2
:1016D0001EF000FA4FF60F001DF072FB45F23810B5
:1016E000C0F202000F211EF0F5F94EF24020C2F2C6
:1016F0000000BDE808401AF057BB00BF08B541F232
:101700005451C2F201014AF6AB230A780132D2B237
:10171000CAF6AA23A3FB02031B0903EB4303A2EBB4
:10172000C30313F0FF0F0A7001D1FFF719FF45F251
:1017300028401021C0F202001EF0CCF941F6786377
:10174000C2F20103F821986C03681B68984745F2C0
:1017500060100F21C0F202001EF0BCF941F2C0502F
:10176000C2F201004FF60F0118F044FE45F22010BE
:10177000C0F2020014211EF0ADF94EF24020C2F278
:101780000000BDE808401AF00FBB00BF1F2970B56C
:101790000C46054608D84DF6A863C2F20003187936
:1017A0000FF096F80AF000FE45F23C401221013D90
:1017B000C0F202001EF08EF9E9B20F290FD841F6EF
:1017C0007866C2F2010641F0C001B06C03681B6884
:1017D0009847B06C036804F07F011B68984745F296
:1017E00060100F21C0F202001EF074F9230403F40C
:1017F000FE03280243F4404343F00C0300F47060FE
:1018000018431DF0DDFA45F23810C0F202000F2136
:101810001EF060F94EF24020C2F20000BDE87040B8
:101820001AF0C2BA1F2938B50C46054608D84DF63D
:10183000A863C2F2000318790FF04AF80AF0B4FD69
:10184000240404F4FE04013D45F2504044F44044B5
:101850002D020D2105F47065C0F2020044F00C0465
:101860001EF038F92C4341F2C0502146C2F201006B
:1018700018F0C0FD45F220101421C0F202001EF045
:1018800029F920461DF09CFA45F23810C0F20200FA
:101890000F211EF01FF94EF24020C2F20000BDE8F9
:1018A00038401AF081BA00BF70B5064645F2604074
:1018B0000C46C0F20200172115461EF00BF9711EEE
:1018C000C9B20F292BD841F67866C2F2010641F061
:1018D000A001B06C03681B689847B06C036804F003
:1018E0007F011B689847B06C036805F07F011B6897
:1018F000984745F28030C0F202000A211EF0EAF853
:1019000045F23810C0F202000F211EF0E3F84EF24B
:101910004020C2F20000BDE870401AF045BA45F21E
:101920008030C0F202000A211EF0D4F8002EE7D168
:10193000681E0002240404F4FE0400F470602043D6
:1019400040F4504040F00D001DF03AFAD8E700BFD7
:1019500070B5064645F2784015460C46C0F20200C6
:1019600012211EF0B7F86B1E1B02240404F4FE04BF
:1019700003F47063234343F45043340143F00D03F5
:10198000E4B21C4341F2C0502146C2F2010018F0FB
:1019900031FD45F22010C0F2020014211EF09AF829
:1019A00016B920461DF00CFA45F23810C0F20200BC
:1019B0000F211EF08FF84EF24020C2F20000BDE869
:1019C00070401AF0F1B900BF38B541F678650446A9
:1019D000C2F2010545F28C401A21C0F202001EF04D
:1019E00079F8A86C0368F3211B689847A86C036812
:1019F00004F07F01DB6C984745F260100F21C0F2C4
:101A000002001EF067F8200400F4FE0040F473406A
:101A100040F002001DF0D4F945F23810C0F2020087
:101A20000F211EF057F84EF24020C2F20000BDE830
:101A300038401AF0B9B900BFF8B54DF6A863C2F244
:101A400000030E461B7C1446054623B1984202D083
:101A5000FFF7BAF938B141F29053C2F201033146AF
:101A600018680DF023FD45F2A8401721013DC0F292
:101A700002001EF02FF8E9B20F2915D841F6786759
:101A8000C2F2010741F08001B86C03681B689847F7
:101A9000B86C036806F07F011B689847B86C036850
:101AA00004F07F011B68984745F260100F21C0F2D7
:101AB00002001EF00FF8230603F0FE43310443F446
:101AC000004301F4FE01280243F008030B4300F435
:101AD000706018431DF074F945F23810C0F202002E
:101AE0000F211DF0F7FF4EF24020C2F20000BDE8CA
:101AF000F8401AF059B900BFF8B54DF6A863C2F224
:101B000000030E461B7C1446054623B1984202D0C2
:101B1000FFF75AF940B141F29053C2F20103224655
:101B2000186831460DF082FA45F2C0401621013D99
:101B3000C0F202001DF0CEFFE9B20F2915D841F620
:101B40007867C2F2010741F09001B86C03681B6826
:101B50009847B86C036806F07F011B689847B86C1B
:101B6000036804F07F011B68984745F260100F215D
:101B7000C0F202001DF0AEFF230603F0FE43310465
:101B800043F4104301F4FE01280243F009030B4320
:101B900000F4706018431DF013F945F23810C0F2DC
:101BA00002000F211DF096FF4EF24020C2F200000D
:101BB000BDE8F8401AF0F8B870B54DF6A863C2F267
:101BC00000030E461B7C1446054623B1984202D002
:101BD000FFF7FAF840B141F29053C2F201032246F6
:101BE000186831460DF022FA45F2D8401121C0F2B2
:101BF00002001DF06FFF230603F0FE43340443F49C
:101C00001043013D43F0090304F4FE042D021C437C
:101C100005F470652C4341F2C0502146C2F2010028
:101C200018F0E8FB45F220101421C0F202001DF06C
:101C300051FF20461DF0C4F845F23810C0F20200F2
:101C40000F211DF047FF4EF24020C2F20000BDE818
:101C500070401AF0A9B800BF38B541F6786504465F
:101C6000C2F2010545F2EC402421C0F202001DF051
:101C700031FFA86C0368F1211B689847A86C0368C2
:101C800021461B68984745F260100F21C0F2020000
:101C900004F00F041DF01EFF44F010044FF2021078
:101CA00040EA04401DF08CF845F23810C0F2020002
:101CB0000F211DF00FFF4EF24020C2F20000BDE8E0
:101CC00038401AF071B800BF70B54DF6A863C2F283
:101CD00000030E461B7C1446054623B1984202D0F1
:101CE000FFF772F838B141F29053C2F20103314666
:101CF00018680DF0DBFB45F214501221C0F202000F
:101D00001DF0E8FE230603F0FE43340443F40043D1
:101D1000013D43F0080304F4FE042D021C4305F4C6
:101D200070652C4341F2C0502146C2F2010018F008
:101D300061FB45F220101421C0F202001DF0CAFE22
:101D400020461DF03DF845F23810C0F202000F2188
:101D50001DF0C0FE4EF24020C2F20000BDE870400F
:101D60001AF022B838B541F678650446C2F201058A
:101D700045F228501521C0F202001DF0ABFEA86C00
:101D80000368F3211B689847A86C036804F07F017F
:101D9000DB6C984745F260100F21C0F202001DF085
:101DA00099FE210401F4FE0141F4734141F2C05057
:101DB00041F00201C2F2010018F01CFB45F22010B4
:101DC000C0F2020014211DF085FE4EF24020C2F246
:101DD0000000BDE8384019F0E7BF00BF38B541F654
:101DE00078650446C2F2010545F240501F21C0F259
:101DF00002001DF06FFEA86C0368F1211B68984774
:101E0000A86C036821461B68984745F260100F21B3
:101E1000C0F2020004F00F041DF05CFE44F0100458
:101E20004FF2021141F2C05041EA0441C2F20100F6
:101E300018F0E0FA45F22010C0F2020014211DF063
:101E400049FE4EF24020C2F20000BDE8384019F0D1
:101E5000ABBF00BF38B541F29053C2F2010301F5A8
:101E600000521B6805460C4645F26050C3F8C0207E
:101E70000D2104F30D04C0F202001DF02BFE04F549
:101E800000536C1E1A04240202F4FE0204F470646F
:101E9000144344F460445B0403F0FE4344F00E0436
:101EA0001C4341F2C0502146C2F2010018F0A2FAD0
:101EB00045F220101421C0F202001DF00BFE204656
:101EC0001CF07EFF45F23810C0F202000F211DF019
:101ED00001FE4EF24020C2F20000BDE8384019F089
:101EE00063BF00BFF8B541F29053C2F2010305464B
:101EF0001B6801F5005645F270500C46013D122159
:101F0000C3F8C060C0F202001DF0E4FDE9B20F2981
:101F100015D841F67867C2F2010741F0E001B86CCC
:101F200003681B689847B86C036806F07F011B685C
:101F30009847B86C0368C6F3C6111B68984745F20A
:101F4000601004F30D040F2104F50054C0F20200E8
:101F50001DF0C0FD2802230403F4FE0300F47060AA
:101F6000184340F46040640404F0FE4440F00E0066
:101F700020431CF025FF45F23810C0F202000F216B
:101F80001DF0A8FD4EF24020C2F20000BDE8F8406E
:101F900019F00ABF4AF28853C2F2010310B4D3F811
:101FA000E0201368506819780478507A137A044254
:101FB00001EA03011AD0937A03F0030309B143F055
:101FC000040343F008039910082B91722AD8072BB9
:101FD00022D2032B2ED011D9042B13D0062B14D1CF
:101FE000D3685DF8044B023BD3607047937A03F0EB
:101FF00003030029E7D043F00403E4E7012B0BD0EF
:10200000022B02D1D368013BD3605DF8044B7047CB
:102010000D2BF7D00E2BF8D1D3685DF8044B0133AC
:10202000D36070470C2B05D0F2D8092BD8D00B2BDE
:10203000E8D0EAE7D3685DF8044B0233D360704719
:102040004AF28853C2F2010310B4D3F8E8201368AF
:10205000506819780478507A137A044201EA03012F
:102060001AD0937A03F0030309B143F0040343F059
:1020700008039910082B91722AD8072B22D2032B20
:102080002ED011D9042B13D0062B14D1D3685DF8B0
:10209000044B023BD3607047937A03F0030300299B
:1020A000E7D043F00403E4E7012B0BD0022B02D16D
:1020B000D368013BD3605DF8044B70470D2BF7D01C
:1020C0000E2BF8D1D3685DF8044B0133D360704711
:1020D0000C2B05D0F2D8092BD8D00B2BE8D0EAE78F
:1020E000D3685DF8044B0233D36070474AF28853DB
:1020F000C2F2010310B4D3F8EC20136850681978C9
:102100000478507A137A044201EA03011AD0937AD0
:1021100003F0030309B143F0040343F008039910EB
:10212000082B91722AD8072B22D2032B2ED011D93B
:10213000042B13D0062B14D1D3685DF8044B023B5B
:10214000D3607047937A03F003030029E7D043F08C
:102150000403E4E7012B0BD0022B02D1D368013B2F
:10216000D3605DF8044B70470D2BF7D00E2BF8D1E0
:10217000D3685DF8044B0133D36070470C2B05D056
:10218000F2D8092BD8D00B2BE8D0EAE7D3685DF85A
:10219000044B0233D36070474AF28853C2F2010302
:1021A00010B4D3F8E4201368506819780478507A92
:1021B000137A044201EA03011AD0937A03F003036D
:1021C00009B143F0040343F008039910082B9172FE
:1021D0002AD8072B22D2032B2ED011D9042B13D0AF
:1021E000062B14D1D3685DF8044B023BD3607047D3
:1021F000937A03F003030029E7D043F00403E4E7F4
:10220000012B0BD0022B02D1D368013BD3605DF8C8
:10221000044B70470D2BF7D00E2BF8D1D3685DF827
:10222000044B0133D36070470C2B05D0F2D8092B37
:10223000D8D00B2BE8D0EAE7D3685DF8044B023323
:10224000D36070474AF28853C2F2010310B41A6A8D
:102250001368506819780478507A137A044201EAB6
:1022600003011AD0937A03F0030309B143F0040386
:1022700043F008039910082B91722AD8072B22D219
:10228000032B2ED011D9042B13D0062B14D1D368D5
:102290005DF8044B023BD3607047937A03F003036D
:1022A0000029E7D043F00403E4E7012B0BD0022B15
:1022B00002D1D368013BD3605DF8044B70470D2B0E
:1022C000F7D00E2BF8D1D3685DF8044B0133D360FF
:1022D00070470C2B05D0F2D8092BD8D00B2BE8D0A7
:1022E000EAE7D3685DF8044B0233D360704700BF60
:1022F0004AF28853C2F2010310B45A6A1368506854
:1023000019780478507A137A044201EA03011AD04A
:10231000937A03F0030309B143F0040343F0080385
:102320009910082B91722AD8072B22D2032B2ED07A
:1023300011D9042B13D0062B14D1D3685DF8044BAC
:10234000023BD3607047937A03F003030029E7D080
:1023500043F00403E4E7012B0BD0022B02D1D36836
:10236000013BD3605DF8044B70470D2BF7D00E2B6B
:10237000F8D1D3685DF8044B0133D36070470C2B60
:1023800005D0F2D8092BD8D00B2BE8D0EAE7D368D8
:102390005DF8044B0233D360704700BF4AF28853A4
:1023A000C2F2010310B49A6A13685068197804786D
:1023B000507A137A044201EA03011AD0937A03F0A7
:1023C000030309B143F0040343F008039910082BF9
:1023D00091722AD8072B22D2032B2ED011D9042B8D
:1023E00013D0062B14D1D3685DF8044B023BD360A5
:1023F0007047937A03F003030029E7D043F0040306
:10240000E4E7012B0BD0022B02D1D368013BD36050
:102410005DF8044B70470D2BF7D00E2BF8D1D36825
:102420005DF8044B0133D36070470C2B05D0F2D814
:10243000092BD8D00B2BE8D0EAE7D3685DF8044B22
:102440000233D360704700BF4AF28853C2F20103DF
:1024500010B4DA6A1368506819780478507A137ADD
:10246000044201EA03011AD0937A03F0030309B18D
:1024700043F0040343F008039910082B91722AD803
:10248000072B22D2032B2ED011D9042B13D0062BCD
:1024900014D1D3685DF8044B023BD3607047937A44
:1024A00003F003030029E7D043F00403E4E7012B22
:1024B0000BD0022B02D1D368013BD3605DF8044BF3
:1024C00070470D2BF7D00E2BF8D1D3685DF8044B75
:1024D0000133D36070470C2B05D0F2D8092BD8D02C
:1024E0000B2BE8D0EAE7D3685DF8044B0233D360E6
:1024F000704700BF4AF28853C2F2010310B41A6B4E
:102500001368506819780478507A137A044201EA03
:1025100003011AD0937A03F0030309B143F00403D3
:1025200043F008039910082B91722AD8072B22D266
:10253000032B2ED011D9042B13D0062B14D1D36822
:102540005DF8044B023BD3607047937A03F00303BA
:102550000029E7D043F00403E4E7012B0BD0022B62
:1025600002D1D368013BD3605DF8044B70470D2B5B
:10257000F7D00E2BF8D1D3685DF8044B0133D3604C
:1025800070470C2B05D0F2D8092BD8D00B2BE8D0F4
:10259000EAE7D3685DF8044B0233D360704700BFAD
:1025A0004AF28853C2F2010310B45A6B13685068A0
:1025B00019780478507A137A044201EA03011AD098
:1025C000937A03F0030309B143F0040343F00803D3
:1025D0009910082B91722AD8072B22D2032B2ED0C8
:1025E00011D9042B13D0062B14D1D3685DF8044BFA
:1025F000023BD3607047937A03F003030029E7D0CE
:1026000043F00403E4E7012B0BD0022B02D1D36883
:10261000013BD3605DF8044B70470D2BF7D00E2BB8
:10262000F8D1D3685DF8044B0133D36070470C2BAD
:1026300005D0F2D8092BD8D00B2BE8D0EAE7D36825
:102640005DF8044B0233D360704700BF4AF28853F1
:10265000C2F2010310B49A6B1368506819780478B9
:10266000507A137A044201EA03011AD0937A03F0F4
:10267000030309B143F0040343F008039910082B46
:1026800091722AD8072B22D2032B2ED011D9042BDA
:1026900013D0062B14D1D3685DF8044B023BD360F2
:1026A0007047937A03F003030029E7D043F0040353
:1026B000E4E7012B0BD0022B02D1D368013BD3609E
:1026C0005DF8044B70470D2BF7D00E2BF8D1D36873
:1026D0005DF8044B0133D36070470C2B05D0F2D862
:1026E000092BD8D00B2BE8D0EAE7D3685DF8044B70
:1026F0000233D360704700BF4AF28853C2F201032D
:1027000010B4DA6B1368506819780478507A137A29
:10271000044201EA03011AD0937A03F0030309B1DA
:1027200043F0040343F008039910082B91722AD850
:10273000072B22D2032B2ED011D9042B13D0062B1A
:1027400014D1D3685DF8044B023BD3607047937A91
:1027500003F003030029E7D043F00403E4E7012B6F
:102760000BD0022B02D1D368013BD3605DF8044B40
:1027700070470D2BF7D00E2BF8D1D3685DF8044BC2
:102780000133D36070470C2B05D0F2D8092BD8D079
:102790000B2BE8D0EAE7D3685DF8044B0233D36033
:1027A000704700BF4AF28853C2F2010310B41A6C9A
:1027B0001368506819780478507A137A044201EA51
:1027C00003011AD0937A03F0030309B143F0040321
:1027D00043F008039910082B91722AD8072B22D2B4
:1027E000032B2ED011D9042B13D0062B14D1D36870
:1027F0005DF8044B023BD3607047937A03F0030308
:102800000029E7D043F00403E4E7012B0BD0022BAF
:1028100002D1D368013BD3605DF8044B70470D2BA8
:10282000F7D00E2BF8D1D3685DF8044B0133D36099
:1028300070470C2B05D0F2D8092BD8D00B2BE8D041
:10284000EAE7D3685DF8044B0233D360704700BFFA
:102850004AF28853C2F2010310B45A6C13685068EC
:1028600019780478507A137A044201EA03011AD0E5
:10287000937A03F0030309B143F0040343F0080320
:102880009910082B91722AD8072B22D2032B2ED015
:1028900011D9042B13D0062B14D1D3685DF8044B47
:1028A000023BD3607047937A03F003030029E7D01B
:1028B00043F00403E4E7012B0BD0022B02D1D368D1
:1028C000013BD3605DF8044B70470D2BF7D00E2B06
:1028D000F8D1D3685DF8044B0133D36070470C2BFB
:1028E00005D0F2D8092BD8D00B2BE8D0EAE7D36873
:1028F0005DF8044B0233D360704700BF4AF288533F
:10290000C2F2010310B49A6C136850681978047805
:10291000507A137A044201EA03011AD0937A03F041
:10292000030309B143F0040343F008039910082B93
:1029300091722AD8072B22D2032B2ED011D9042B27
:1029400013D0062B14D1D3685DF8044B023BD3603F
:102950007047937A03F003030029E7D043F00403A0
:10296000E4E7012B0BD0022B02D1D368013BD360EB
:102970005DF8044B70470D2BF7D00E2BF8D1D368C0
:102980005DF8044B0133D36070470C2B05D0F2D8AF
:10299000092BD8D00B2BE8D0EAE7D3685DF8044BBD
:1029A0000233D360704700BF4AF28853C2F201037A
:1029B00010B4DA6C1368506819780478507A137A76
:1029C000044201EA03011AD0937A03F0030309B128
:1029D00043F0040343F008039910082B91722AD89E
:1029E000072B22D2032B2ED011D9042B13D0062B68
:1029F00014D1D3685DF8044B023BD3607047937ADF
:102A000003F003030029E7D043F00403E4E7012BBC
:102A10000BD0022B02D1D368013BD3605DF8044B8D
:102A200070470D2BF7D00E2BF8D1D3685DF8044B0F
:102A30000133D36070470C2B05D0F2D8092BD8D0C6
:102A40000B2BE8D0EAE7D3685DF8044B0233D36080
:102A5000704700BF4AF28853C2F2010310B41A6DE6
:102A60001368506819780478507A137A044201EA9E
:102A700003011AD0937A03F0030309B143F004036E
:102A800043F008039910082B91722AD8072B22D201
:102A9000032B2ED011D9042B13D0062B14D1D368BD
:102AA0005DF8044B023BD3607047937A03F0030355
:102AB0000029E7D043F00403E4E7012B0BD0022BFD
:102AC00002D1D368013BD3605DF8044B70470D2BF6
:102AD000F7D00E2BF8D1D3685DF8044B0133D360E7
:102AE00070470C2B05D0F2D8092BD8D00B2BE8D08F
:102AF000EAE7D3685DF8044B0233D360704700BF48
:102B00004AF28853C2F2010310B45A6D1368506838
:102B100019780478507A137A044201EA03011AD032
:102B2000937A03F0030309B143F0040343F008036D
:102B30009910082B91722AD8072B22D2032B2ED062
:102B400011D9042B13D0062B14D1D3685DF8044B94
:102B5000023BD3607047937A03F003030029E7D068
:102B600043F00403E4E7012B0BD0022B02D1D3681E
:102B7000013BD3605DF8044B70470D2BF7D00E2B53
:102B8000F8D1D3685DF8044B0133D36070470C2B48
:102B900005D0F2D8092BD8D00B2BE8D0EAE7D368C0
:102BA0005DF8044B0233D360704700BF4AF288538C
:102BB000C2F2010310B49A6D136850681978047852
:102BC000507A137A044201EA03011AD0937A03F08F
:102BD000030309B143F0040343F008039910082BE1
:102BE00091722AD8072B22D2032B2ED011D9042B75
:102BF00013D0062B14D1D3685DF8044B023BD3608D
:102C00007047937A03F003030029E7D043F00403ED
:102C1000E4E7012B0BD0022B02D1D368013BD36038
:102C20005DF8044B70470D2BF7D00E2BF8D1D3680D
:102C30005DF8044B0133D36070470C2B05D0F2D8FC
:102C4000092BD8D00B2BE8D0EAE7D3685DF8044B0A
:102C50000233D360704700BF4AF28853C2F20103C7
:102C600010B4DA6D1368506819780478507A137AC2
:102C7000044201EA03011AD0937A03F0030309B175
:102C800043F0040343F008039910082B91722AD8EB
:102C9000072B22D2032B2ED011D9042B13D0062BB5
:102CA00014D1D3685DF8044B023BD3607047937A2C
:102CB00003F003030029E7D043F00403E4E7012B0A
:102CC0000BD0022B02D1D368013BD3605DF8044BDB
:102CD00070470D2BF7D00E2BF8D1D3685DF8044B5D
:102CE0000133D36070470C2B05D0F2D8092BD8D014
:102CF0000B2BE8D0EAE7D3685DF8044B0233D360CE
:102D0000704700BF4AF28853C2F2010310B41A6838
:102D10001368506819780478507A137A044201EAEB
:102D200003011AD0937A03F0030309B143F00403BB
:102D300043F008039910082B91722AD8072B22D24E
:102D4000032B2ED011D9042B13D0062B14D1D3680A
:102D50005DF8044B023BD3607047937A03F00303A2
:102D60000029E7D043F00403E4E7012B0BD0022B4A
:102D700002D1D368013BD3605DF8044B70470D2B43
:102D8000F7D00E2BF8D1D3685DF8044B0133D36034
:102D900070470C2B05D0F2D8092BD8D00B2BE8D0DC
:102DA000EAE7D3685DF8044B0233D360704700BF95
:102DB0004AF28853C2F2010310B45A68136850688B
:102DC00019780478507A137A044201EA03011AD080
:102DD000937A03F0030309B143F0040343F00803BB
:102DE0009910082B91722AD8072B22D2032B2ED0B0
:102DF00011D9042B13D0062B14D1D3685DF8044BE2
:102E0000023BD3607047937A03F003030029E7D0B5
:102E100043F00403E4E7012B0BD0022B02D1D3686B
:102E2000013BD3605DF8044B70470D2BF7D00E2BA0
:102E3000F8D1D3685DF8044B0133D36070470C2B95
:102E400005D0F2D8092BD8D00B2BE8D0EAE7D3680D
:102E50005DF8044B0233D360704700BF4AF28853D9
:102E6000C2F2010310B49A681368506819780478A4
:102E7000507A137A044201EA03011AD0937A03F0DC
:102E8000030309B143F0040343F008039910082B2E
:102E900091722AD8072B22D2032B2ED011D9042BC2
:102EA00013D0062B14D1D3685DF8044B023BD360DA
:102EB0007047937A03F003030029E7D043F004033B
:102EC000E4E7012B0BD0022B02D1D368013BD36086
:102ED0005DF8044B70470D2BF7D00E2BF8D1D3685B
:102EE0005DF8044B0133D36070470C2B05D0F2D84A
:102EF000092BD8D00B2BE8D0EAE7D3685DF8044B58
:102F00000233D360704700BF4AF28853C2F2010314
:102F100010B4DA681368506819780478507A137A14
:102F2000044201EA03011AD0937A03F0030309B1C2
:102F300043F0040343F008039910082B91722AD838
:102F4000072B22D2032B2ED011D9042B13D0062B02
:102F500014D1D3685DF8044B023BD3607047937A79
:102F600003F003030029E7D043F00403E4E7012B57
:102F70000BD0022B02D1D368013BD3605DF8044B28
:102F800070470D2BF7D00E2BF8D1D3685DF8044BAA
:102F90000133D36070470C2B05D0F2D8092BD8D061
:102FA0000B2BE8D0EAE7D3685DF8044B0233D3601B
:102FB000704700BF4AF28853C2F2010310B41A6985
:102FC0001368506819780478507A137A044201EA39
:102FD00003011AD0937A03F0030309B143F0040309
:102FE00043F008039910082B91722AD8072B22D29C
:102FF000032B2ED011D9042B13D0062B14D1D36858
:103000005DF8044B023BD3607047937A03F00303EF
:103010000029E7D043F00403E4E7012B0BD0022B97
:1030200002D1D368013BD3605DF8044B70470D2B90
:10303000F7D00E2BF8D1D3685DF8044B0133D36081
:1030400070470C2B05D0F2D8092BD8D00B2BE8D029
:10305000EAE7D3685DF8044B0233D360704700BFE2
:103060004AF28853C2F2010310B45A6913685068D7
:1030700019780478507A137A044201EA03011AD0CD
:10308000937A03F0030309B143F0040343F0080308
:103090009910082B91722AD8072B22D2032B2ED0FD
:1030A00011D9042B13D0062B14D1D3685DF8044B2F
:1030B000023BD3607047937A03F003030029E7D003
:1030C00043F00403E4E7012B0BD0022B02D1D368B9
:1030D000013BD3605DF8044B70470D2BF7D00E2BEE
:1030E000F8D1D3685DF8044B0133D36070470C2BE3
:1030F00005D0F2D8092BD8D00B2BE8D0EAE7D3685B
:103100005DF8044B0233D360704700BF4AF2885326
:10311000C2F2010310B49A691368506819780478F0
:10312000507A137A044201EA03011AD0937A03F029
:10313000030309B143F0040343F008039910082B7B
:1031400091722AD8072B22D2032B2ED011D9042B0F
:1031500013D0062B14D1D3685DF8044B023BD36027
:103160007047937A03F003030029E7D043F0040388
:10317000E4E7012B0BD0022B02D1D368013BD360D3
:103180005DF8044B70470D2BF7D00E2BF8D1D368A8
:103190005DF8044B0133D36070470C2B05D0F2D897
:1031A000092BD8D00B2BE8D0EAE7D3685DF8044BA5
:1031B0000233D360704700BF4AF28853C2F2010362
:1031C00010B4DA691368506819780478507A137A61
:1031D000044201EA03011AD0937A03F0030309B110
:1031E00043F0040343F008039910082B91722AD886
:1031F000072B22D2032B2ED011D9042B13D0062B50
:1032000014D1D3685DF8044B023BD3607047937AC6
:1032100003F003030029E7D043F00403E4E7012BA4
:103220000BD0022B02D1D368013BD3605DF8044B75
:1032300070470D2BF7D00E2BF8D1D3685DF8044BF7
:103240000133D36070470C2B05D0F2D8092BD8D0AE
:103250000B2BE8D0EAE7D3685DF8044B0233D36068
:10326000704700BF4AF28853C2F2010310B41A6ECD
:103270001368506819780478507A137A044201EA86
:1032800003011AD0937A03F0030309B143F0040356
:1032900043F008039910082B91722AD8072B22D2E9
:1032A000032B2ED011D9042B13D0062B14D1D368A5
:1032B0005DF8044B023BD3607047937A03F003033D
:1032C0000029E7D043F00403E4E7012B0BD0022BE5
:1032D00002D1D368013BD3605DF8044B70470D2BDE
:1032E000F7D00E2BF8D1D3685DF8044B0133D360CF
:1032F00070470C2B05D0F2D8092BD8D00B2BE8D077
:10330000EAE7D3685DF8044B0233D360704700BF2F
:103310004AF28853C2F2010310B45A6E136850681F
:1033200019780478507A137A044201EA03011AD01A
:10333000937A03F0030309B143F0040343F0080355
:103340009910082B91722AD8072B22D2032B2ED04A
:1033500011D9042B13D0062B14D1D3685DF8044B7C
:10336000023BD3607047937A03F003030029E7D050
:1033700043F00403E4E7012B0BD0022B02D1D36806
:10338000013BD3605DF8044B70470D2BF7D00E2B3B
:10339000F8D1D3685DF8044B0133D36070470C2B30
:1033A00005D0F2D8092BD8D00B2BE8D0EAE7D368A8
:1033B0005DF8044B0233D360704700BF4AF2885374
:1033C000C2F2010310B49A6E136850681978047839
:1033D000507A137A044201EA03011AD0937A03F077
:1033E000030309B143F0040343F008039910082BC9
:1033F00091722AD8072B22D2032B2ED011D9042B5D
:1034000013D0062B14D1D3685DF8044B023BD36074
:103410007047937A03F003030029E7D043F00403D5
:10342000E4E7012B0BD0022B02D1D368013BD36020
:103430005DF8044B70470D2BF7D00E2BF8D1D368F5
:103440005DF8044B0133D36070470C2B05D0F2D8E4
:10345000092BD8D00B2BE8D0EAE7D3685DF8044BF2
:103460000233D360704700BF4AF28853C2F20103AF
:1034700010B4DA6E1368506819780478507A137AA9
:10348000044201EA03011AD0937A03F0030309B15D
:1034900043F0040343F008039910082B91722AD8D3
:1034A000072B22D2032B2ED011D9042B13D0062B9D
:1034B00014D1D3685DF8044B023BD3607047937A14
:1034C00003F003030029E7D043F00403E4E7012BF2
:1034D0000BD0022B02D1D368013BD3605DF8044BC3
:1034E00070470D2BF7D00E2BF8D1D3685DF8044B45
:1034F0000133D36070470C2B05D0F2D8092BD8D0FC
:103500000B2BE8D0EAE7D3685DF8044B0233D360B5
:10351000704700BF4AF28853C2F2010310B41A6F19
:103520001368506819780478507A137A044201EAD3
:1035300003011AD0937A03F0030309B143F00403A3
:1035400043F008039910082B91722AD8072B22D236
:10355000032B2ED011D9042B13D0062B14D1D368F2
:103560005DF8044B023BD3607047937A03F003038A
:103570000029E7D043F00403E4E7012B0BD0022B32
:1035800002D1D368013BD3605DF8044B70470D2B2B
:10359000F7D00E2BF8D1D3685DF8044B0133D3601C
:1035A00070470C2B05D0F2D8092BD8D00B2BE8D0C4
:1035B000EAE7D3685DF8044B0233D360704700BF7D
:1035C0004AF28853C2F2010310B45A6F136850686C
:1035D00019780478507A137A044201EA03011AD068
:1035E000937A03F0030309B143F0040343F00803A3
:1035F0009910082B91722AD8072B22D2032B2ED098
:1036000011D9042B13D0062B14D1D3685DF8044BC9
:10361000023BD3607047937A03F003030029E7D09D
:1036200043F00403E4E7012B0BD0022B02D1D36853
:10363000013BD3605DF8044B70470D2BF7D00E2B88
:10364000F8D1D3685DF8044B0133D36070470C2B7D
:1036500005D0F2D8092BD8D00B2BE8D0EAE7D368F5
:103660005DF8044B0233D360704700BF4AF28853C1
:10367000C2F2010310B49A6F136850681978047885
:10368000507A137A044201EA03011AD0937A03F0C4
:10369000030309B143F0040343F008039910082B16
:1036A00091722AD8072B22D2032B2ED011D9042BAA
:1036B00013D0062B14D1D3685DF8044B023BD360C2
:1036C0007047937A03F003030029E7D043F0040323
:1036D000E4E7012B0BD0022B02D1D368013BD3606E
:1036E0005DF8044B70470D2BF7D00E2BF8D1D36843
:1036F0005DF8044B0133D36070470C2B05D0F2D832
:10370000092BD8D00B2BE8D0EAE7D3685DF8044B3F
:103710000233D360704700BF4AF28853C2F20103FC
:1037200010B4DA6F1368506819780478507A137AF5
:10373000044201EA03011AD0937A03F0030309B1AA
:1037400043F0040343F008039910082B91722AD820
:10375000072B22D2032B2ED011D9042B13D0062BEA
:1037600014D1D3685DF8044B023BD3607047937A61
:1037700003F003030029E7D043F00403E4E7012B3F
:103780000BD0022B02D1D368013BD3605DF8044B10
:1037900070470D2BF7D00E2BF8D1D3685DF8044B92
:1037A0000133D36070470C2B05D0F2D8092BD8D049
:1037B0000B2BE8D0EAE7D3685DF8044B0233D36003
:1037C000704700BF4AF28853C2F2010310B4D3F825
:1037D00080201368506819780478507A137A04426C
:1037E00001EA03011AD0937A03F0030309B143F00D
:1037F000040343F008039910082B91722AD8072B71
:1038000022D2032B2ED011D9042B13D0062B14D186
:10381000D3685DF8044B023BD3607047937A03F0A2
:1038200003030029E7D043F00403E4E7012B0BD0A6
:10383000022B02D1D368013BD3605DF8044B704783
:103840000D2BF7D00E2BF8D1D3685DF8044B013364
:10385000D36070470C2B05D0F2D8092BD8D00B2B96
:10386000E8D0EAE7D3685DF8044B0233D3607047D1
:103870004AF28853C2F2010310B4D3F884201368CB
:10388000506819780478507A137A044201EA0301E7
:103890001AD0937A03F0030309B143F0040343F011
:1038A00008039910082B91722AD8072B22D2032BD8
:1038B0002ED011D9042B13D0062B14D1D3685DF868
:1038C000044B023BD3607047937A03F00303002953
:1038D000E7D043F00403E4E7012B0BD0022B02D125
:1038E000D368013BD3605DF8044B70470D2BF7D0D4
:1038F0000E2BF8D1D3685DF8044B0133D3607047C9
:103900000C2B05D0F2D8092BD8D00B2BE8D0EAE746
:10391000D3685DF8044B0233D36070474AF2885392
:10392000C2F2010310B4D3F88820136850681978E4
:103930000478507A137A044201EA03011AD0937A88
:1039400003F0030309B143F0040343F008039910A3
:10395000082B91722AD8072B22D2032B2ED011D9F3
:10396000042B13D0062B14D1D3685DF8044B023B13
:10397000D3607047937A03F003030029E7D043F044
:103980000403E4E7012B0BD0022B02D1D368013BE7
:10399000D3605DF8044B70470D2BF7D00E2BF8D198
:1039A000D3685DF8044B0133D36070470C2B05D00E
:1039B000F2D8092BD8D00B2BE8D0EAE7D3685DF812
:1039C000044B0233D36070474AF28853C2F20103BA
:1039D00010B4D3F88C201368506819780478507AA2
:1039E000137A044201EA03011AD0937A03F0030325
:1039F00009B143F0040343F008039910082B9172B6
:103A00002AD8072B22D2032B2ED011D9042B13D066
:103A1000062B14D1D3685DF8044B023BD36070478A
:103A2000937A03F003030029E7D043F00403E4E7AB
:103A3000012B0BD0022B02D1D368013BD3605DF880
:103A4000044B70470D2BF7D00E2BF8D1D3685DF8DF
:103A5000044B0133D36070470C2B05D0F2D8092BEF
:103A6000D8D00B2BE8D0EAE7D3685DF8044B0233DB
:103A7000D36070474AF28853C2F2010310B4D3F8FE
:103A800090201368506819780478507A137A0442A9
:103A900001EA03011AD0937A03F0030309B143F05A
:103AA000040343F008039910082B91722AD8072BBE
:103AB00022D2032B2ED011D9042B13D0062B14D1D4
:103AC000D3685DF8044B023BD3607047937A03F0F0
:103AD00003030029E7D043F00403E4E7012B0BD0F4
:103AE000022B02D1D368013BD3605DF8044B7047D1
:103AF0000D2BF7D00E2BF8D1D3685DF8044B0133B2
:103B0000D36070470C2B05D0F2D8092BD8D00B2BE3
:103B1000E8D0EAE7D3685DF8044B0233D36070471E
:103B20004AF28853C2F2010310B4D3F89420136808
:103B3000506819780478507A137A044201EA030134
:103B40001AD0937A03F0030309B143F0040343F05E
:103B500008039910082B91722AD8072B22D2032B25
:103B60002ED011D9042B13D0062B14D1D3685DF8B5
:103B7000044B023BD3607047937A03F003030029A0
:103B8000E7D043F00403E4E7012B0BD0022B02D172
:103B9000D368013BD3605DF8044B70470D2BF7D021
:103BA0000E2BF8D1D3685DF8044B0133D360704716
:103BB0000C2B05D0F2D8092BD8D00B2BE8D0EAE794
:103BC000D3685DF8044B0233D36070474AF28853E0
:103BD000C2F2010310B4D3F8982013685068197822
:103BE0000478507A137A044201EA03011AD0937AD6
:103BF00003F0030309B143F0040343F008039910F1
:103C0000082B91722AD8072B22D2032B2ED011D940
:103C1000042B13D0062B14D1D3685DF8044B023B60
:103C2000D3607047937A03F003030029E7D043F091
:103C30000403E4E7012B0BD0022B02D1D368013B34
:103C4000D3605DF8044B70470D2BF7D00E2BF8D1E5
:103C5000D3685DF8044B0133D36070470C2B05D05B
:103C6000F2D8092BD8D00B2BE8D0EAE7D3685DF85F
:103C7000044B0233D36070474AF28853C2F2010307
:103C800010B4D3F89C201368506819780478507ADF
:103C9000137A044201EA03011AD0937A03F0030372
:103CA00009B143F0040343F008039910082B917203
:103CB0002AD8072B22D2032B2ED011D9042B13D0B4
:103CC000062B14D1D3685DF8044B023BD3607047D8
:103CD000937A03F003030029E7D043F00403E4E7F9
:103CE000012B0BD0022B02D1D368013BD3605DF8CE
:103CF000044B70470D2BF7D00E2BF8D1D3685DF82D
:103D0000044B0133D36070470C2B05D0F2D8092B3C
:103D1000D8D00B2BE8D0EAE7D3685DF8044B023328
:103D2000D36070474AF28853C2F2010310B4D3F84B
:103D3000A0201368506819780478507A137A0442E6
:103D400001EA03011AD0937A03F0030309B143F0A7
:103D5000040343F008039910082B91722AD8072B0B
:103D600022D2032B2ED011D9042B13D0062B14D121
:103D7000D3685DF8044B023BD3607047937A03F03D
:103D800003030029E7D043F00403E4E7012B0BD041
:103D9000022B02D1D368013BD3605DF8044B70471E
:103DA0000D2BF7D00E2BF8D1D3685DF8044B0133FF
:103DB000D36070470C2B05D0F2D8092BD8D00B2B31
:103DC000E8D0EAE7D3685DF8044B0233D36070476C
:103DD0004AF28853C2F2010310B4D3F8A420136846
:103DE000506819780478507A137A044201EA030182
:103DF0001AD0937A03F0030309B143F0040343F0AC
:103E000008039910082B91722AD8072B22D2032B72
:103E10002ED011D9042B13D0062B14D1D3685DF802
:103E2000044B023BD3607047937A03F003030029ED
:103E3000E7D043F00403E4E7012B0BD0022B02D1BF
:103E4000D368013BD3605DF8044B70470D2BF7D06E
:103E50000E2BF8D1D3685DF8044B0133D360704763
:103E60000C2B05D0F2D8092BD8D00B2BE8D0EAE7E1
:103E7000D3685DF8044B0233D36070474AF288532D
:103E8000C2F2010310B4D3F8A8201368506819785F
:103E90000478507A137A044201EA03011AD0937A23
:103EA00003F0030309B143F0040343F0080399103E
:103EB000082B91722AD8072B22D2032B2ED011D98E
:103EC000042B13D0062B14D1D3685DF8044B023BAE
:103ED000D3607047937A03F003030029E7D043F0DF
:103EE0000403E4E7012B0BD0022B02D1D368013B82
:103EF000D3605DF8044B70470D2BF7D00E2BF8D133
:103F0000D3685DF8044B0133D36070470C2B05D0A8
:103F1000F2D8092BD8D00B2BE8D0EAE7D3685DF8AC
:103F2000044B0233D36070474AF28853C2F2010354
:103F300010B4D3F8AC201368506819780478507A1C
:103F4000137A044201EA03011AD0937A03F00303BF
:103F500009B143F0040343F008039910082B917250
:103F60002AD8072B22D2032B2ED011D9042B13D001
:103F7000062B14D1D3685DF8044B023BD360704725
:103F8000937A03F003030029E7D043F00403E4E746
:103F9000012B0BD0022B02D1D368013BD3605DF81B
:103FA000044B70470D2BF7D00E2BF8D1D3685DF87A
:103FB000044B0133D36070470C2B05D0F2D8092B8A
:103FC000D8D00B2BE8D0EAE7D3685DF8044B023376
:103FD000D36070474AF28853C2F2010310B4D3F899
:103FE000B0201368506819780478507A137A044224
:103FF00001EA03011AD0937A03F0030309B143F0F5
:10400000040343F008039910082B91722AD8072B58
:1040100022D2032B2ED011D9042B13D0062B14D16E
:10402000D3685DF8044B023BD3607047937A03F08A
:1040300003030029E7D043F00403E4E7012B0BD08E
:10404000022B02D1D368013BD3605DF8044B70476B
:104050000D2BF7D00E2BF8D1D3685DF8044B01334C
:10406000D36070470C2B05D0F2D8092BD8D00B2B7E
:10407000E8D0EAE7D3685DF8044B0233D3607047B9
:104080004AF28853C2F2010310B4D3F8B420136883
:10409000506819780478507A137A044201EA0301CF
:1040A0001AD0937A03F0030309B143F0040343F0F9
:1040B00008039910082B91722AD8072B22D2032BC0
:1040C0002ED011D9042B13D0062B14D1D3685DF850
:1040D000044B023BD3607047937A03F0030300293B
:1040E000E7D043F00403E4E7012B0BD0022B02D10D
:1040F000D368013BD3605DF8044B70470D2BF7D0BC
:104100000E2BF8D1D3685DF8044B0133D3607047B0
:104110000C2B05D0F2D8092BD8D00B2BE8D0EAE72E
:10412000D3685DF8044B0233D36070474AF288537A
:10413000C2F2010310B4D3F8B8201368506819789C
:104140000478507A137A044201EA03011AD0937A70
:1041500003F0030309B143F0040343F0080399108B
:10416000082B91722AD8072B22D2032B2ED011D9DB
:10417000042B13D0062B14D1D3685DF8044B023BFB
:10418000D3607047937A03F003030029E7D043F02C
:104190000403E4E7012B0BD0022B02D1D368013BCF
:1041A000D3605DF8044B70470D2BF7D00E2BF8D180
:1041B000D3685DF8044B0133D36070470C2B05D0F6
:1041C000F2D8092BD8D00B2BE8D0EAE7D3685DF8FA
:1041D000044B0233D36070474AF28853C2F20103A2
:1041E00010B4D3F8BC201368506819780478507A5A
:1041F000137A044201EA03011AD0937A03F003030D
:1042000009B143F0040343F008039910082B91729D
:104210002AD8072B22D2032B2ED011D9042B13D04E
:10422000062B14D1D3685DF8044B023BD360704772
:10423000937A03F003030029E7D043F00403E4E793
:10424000012B0BD0022B02D1D368013BD3605DF868
:10425000044B70470D2BF7D00E2BF8D1D3685DF8C7
:10426000044B0133D36070470C2B05D0F2D8092BD7
:10427000D8D00B2BE8D0EAE7D3685DF8044B0233C3
:10428000D36070474AF28853C2F2010310B4D3F8E6
:10429000C0201368506819780478507A137A044261
:1042A00001EA03011AD0937A03F0030309B143F042
:1042B000040343F008039910082B91722AD8072BA6
:1042C00022D2032B2ED011D9042B13D0062B14D1BC
:1042D000D3685DF8044B023BD3607047937A03F0D8
:1042E00003030029E7D043F00403E4E7012B0BD0DC
:1042F000022B02D1D368013BD3605DF8044B7047B9
:104300000D2BF7D00E2BF8D1D3685DF8044B013399
:10431000D36070470C2B05D0F2D8092BD8D00B2BCB
:10432000E8D0EAE7D3685DF8044B0233D360704706
:104330004AF28853C2F2010310B4D3F8C4201368C0
:10434000506819780478507A137A044201EA03011C
:104350001AD0937A03F0030309B143F0040343F046
:1043600008039910082B91722AD8072B22D2032B0D
:104370002ED011D9042B13D0062B14D1D3685DF89D
:10438000044B023BD3607047937A03F00303002988
:10439000E7D043F00403E4E7012B0BD0022B02D15A
:1043A000D368013BD3605DF8044B70470D2BF7D009
:1043B0000E2BF8D1D3685DF8044B0133D3607047FE
:1043C0000C2B05D0F2D8092BD8D00B2BE8D0EAE77C
:1043D000D3685DF8044B0233D36070474AF28853C8
:1043E000C2F2010310B4D3F8C820136850681978DA
:1043F0000478507A137A044201EA03011AD0937ABE
:1044000003F0030309B143F0040343F008039910D8
:10441000082B91722AD8072B22D2032B2ED011D928
:10442000042B13D0062B14D1D3685DF8044B023B48
:10443000D3607047937A03F003030029E7D043F079
:104440000403E4E7012B0BD0022B02D1D368013B1C
:10445000D3605DF8044B70470D2BF7D00E2BF8D1CD
:10446000D3685DF8044B0133D36070470C2B05D043
:10447000F2D8092BD8D00B2BE8D0EAE7D3685DF847
:10448000044B0233D36070474AF28853C2F20103EF
:1044900010B4D3F8CC201368506819780478507A97
:1044A000137A044201EA03011AD0937A03F003035A
:1044B00009B143F0040343F008039910082B9172EB
:1044C0002AD8072B22D2032B2ED011D9042B13D09C
:1044D000062B14D1D3685DF8044B023BD3607047C0
:1044E000937A03F003030029E7D043F00403E4E7E1
:1044F000012B0BD0022B02D1D368013BD3605DF8B6
:10450000044B70470D2BF7D00E2BF8D1D3685DF814
:10451000044B0133D36070470C2B05D0F2D8092B24
:10452000D8D00B2BE8D0EAE7D3685DF8044B023310
:10453000D36070474AF28853C2F2010310B4D3F833
:10454000D0201368506819780478507A137A04429E
:1045500001EA03011AD0937A03F0030309B143F08F
:10456000040343F008039910082B91722AD8072BF3
:1045700022D2032B2ED011D9042B13D0062B14D109
:10458000D3685DF8044B023BD3607047937A03F025
:1045900003030029E7D043F00403E4E7012B0BD029
:1045A000022B02D1D368013BD3605DF8044B704706
:1045B0000D2BF7D00E2BF8D1D3685DF8044B0133E7
:1045C000D36070470C2B05D0F2D8092BD8D00B2B19
:1045D000E8D0EAE7D3685DF8044B0233D360704754
:1045E0004AF28853C2F2010310B4D3F8D4201368FE
:1045F000506819780478507A137A044201EA03016A
:104600001AD0937A03F0030309B143F0040343F093
:1046100008039910082B91722AD8072B22D2032B5A
:104620002ED011D9042B13D0062B14D1D3685DF8EA
:10463000044B023BD3607047937A03F003030029D5
:10464000E7D043F00403E4E7012B0BD0022B02D1A7
:10465000D368013BD3605DF8044B70470D2BF7D056
:104660000E2BF8D1D3685DF8044B0133D36070474B
:104670000C2B05D0F2D8092BD8D00B2BE8D0EAE7C9
:10468000D3685DF8044B0233D36070474AF2885315
:10469000C2F2010310B4D3F8D82013685068197817
:1046A0000478507A137A044201EA03011AD0937A0B
:1046B00003F0030309B143F0040343F00803991026
:1046C000082B91722AD8072B22D2032B2ED011D976
:1046D000042B13D0062B14D1D3685DF8044B023B96
:1046E000D3607047937A03F003030029E7D043F0C7
:1046F0000403E4E7012B0BD0022B02D1D368013B6A
:10470000D3605DF8044B70470D2BF7D00E2BF8D11A
:10471000D3685DF8044B0133D36070470C2B05D090
:10472000F2D8092BD8D00B2BE8D0EAE7D3685DF894
:10473000044B0233D36070474AF28853C2F201033C
:1047400010B4D3F8DC201368506819780478507AD4
:10475000137A044201EA03011AD0937A03F00303A7
:1047600009B143F0040343F008039910082B917238
:104770002AD8072B22D2032B2ED011D9042B13D0E9
:10478000062B14D1D3685DF8044B023BD36070470D
:10479000937A03F003030029E7D043F00403E4E72E
:1047A000012B0BD0022B02D1D368013BD3605DF803
:1047B000044B70470D2BF7D00E2BF8D1D3685DF862
:1047C000044B0133D36070470C2B05D0F2D8092B72
:1047D000D8D00B2BE8D0EAE7D3685DF8044B02335E
:1047E000D360704710B445F290040023C0F2020475
:1047F0004172026104600372C36041B1194600E076
:10480000026942F82310427A01339A42F8DC4AF2F4
:104810008863C2F201031A680AB90CE01A465369A8
:10482000002BFBD15061002343618380C3808372DE
:104830005DF8044B70471860F5E700BFF8B541F626
:104840007864C2F2010447F61221A06C0368DB69A8
:10485000984741F6C947032041F6B93346F2E5517E
:1048600044F6295641F6556284F86400C0F200030C
:10487000C0F20007C0F20001C0F20006C0F2000260
:1048800041F6250063602760E1606661A261C0F2C5
:10489000000045F6453340F6057741F6511140F6E4
:1048A000194640F6DD122061C0F20003C0F2000795
:1048B000C0F20001C0F20006C0F2000241F2F15065
:1048C000E3612762A160A662E262C0F2000040F6E6
:1048D000794340F6215740F6CD4140F6755640F6F3
:1048E0002962C0F200022063C0F20003C0F2000798
:1048F000C0F20001C0F200064EF2402545F284509D
:104900006264C2F200056363A76300234FF6FF777A
:10491000E16326641721C0F2020084F84C3084F869
:104920004E3084F84D30A365636584F8E93084F82F
:10493000663084F8653084F8673084F86830E7655D
:1049400027661BF0C7F8284617F02EFA13F022FF4F
:1049500041F2C053C2F2010341F6F92141F6392771
:1049600046F22D5644F6AD5441F6E562C0F2000120
:10497000C0F20007C0F20006C0F20004C0F200025C
:1049800041F28D70C3F86811C3F86471C3F87061A7
:10499000C3F87841C3F87C21C0F2000045F6A53188
:1049A00041F6594741F6A90641F6C91440F6AD62F1
:1049B000C3F87401C0F20001C0F20007C0F20006A3
:1049C000C0F20004C0F2000241F27560C3F8841125
:1049D000C3F88871C3F86C61C3F89041C3F894219F
:1049E000C0F2000040F6312140F6892740F6E1266A
:1049F00040F6393440F69132C0F20002C3F8980113
:104A0000C0F20001C0F20007C0F20006C0F20004CC
:104A100045F29C50C3F89C11C3F8A071C3F8A4617F
:104A2000C3F8A841C3F8AC211D21C0F202001BF05D
:104A300051F8284617F0B8F94AF68811C2F2010178
:104A400041F2E13EC0F2000E4AF68014C1F800E0E7
:104A5000C2F2010441F2193EC0F2000E4AF684137C
:104A6000C4F800E0C2F2010346F26D4EC0F2000E3F
:104A70004AF65817C3F800E0C2F2010744F6456E43
:104A8000C0F2000E4AF64810C7F800E0C2F201007A
:104A900041F2A94EC0F2000E4AF64416C0F800E0FA
:104AA000C2F2010641F2792EC0F2000E4AF66812F7
:104AB000C6F800E0C2F2010245F6294EC0F2000E2F
:104AC0004AF66011C2F800E0C2F2010141F6DD5E73
:104AD000C0F2000E4AF65414C1F800E0C2F201041C
:104AE00041F2D91EC0F2000E4AF67C13C4F800E071
:104AF000C2F2010341F6655EC0F2000E4AF6641789
:104B0000C3F800E0C2F2010741F2791EC0F2000EC4
:104B10004AF62C10C7F800E0C2F2010041F2FD672E
:104B2000C0F200074AF65C160760C2F201064AF6B8
:104B30003C1241F22907C2F20102C0F200074AF614
:104B4000741141F289003760C2F20101C0F2000025
:104B50004AF634144AF6301340F6C977C2F201031C
:104B60001060C2F20104C0F2000740F6697641F21B
:104B7000E90245F2BC500F60C0F20006C0F200022C
:104B8000C0F20200182126601A601AF0A3FF28461E
:104B9000BDE8F84017F008B94DF20A73C3F6234395
:104BA00006EE103A437EC17E07EE103A837CB8EEE3
:104BB000C77A07EE903A70B4F8EEE76A27EE067A05
:104BC00083B067EE267A0022FCEEE77A8273CDEDA1
:104BD000017A42739DF80430027301B10373827E3F
:104BE00002B14373027F02B1837390F8213090F8D1
:104BF000231007EE103A4DF20A73C3F6234306EE74
:104C0000103A037CB8EEC77A07EE903A27EE067AA0
:104C1000F8EEE76A67EE267AFCEEE77ACDED017AE8
:104C20009DF8043021B1017B994238BF19460173C8
:104C300090F8221021B1417B994238BF1946417347
:104C400090F8244024B1817B8B4238BF0B4683739C
:104C5000437FC17F07EE103A4DF20A73C3F6234338
:104C600006EE103A437CB8EEC77A07EE903A27EE8C
:104C7000067AF8EEE76A67EE267AFCEEE77ACDED83
:104C8000017A9DF8043021B1017B994238BF194661
:104C90000173817F21B1417B994238BF194641732D
:104CA00090F8201021B1857BAB4238BF2B4683732F
:104CB00090F8253090F8275007EE103A4DF20A731D
:104CC000C3F6234306EE103AC37BB8EEC77A07EE6D
:104CD000903A27EE067AF8EEE76A67EE267AFCEE5F
:104CE000E77ACDED017A9DF8043025B1057B9D4230
:104CF00038BF1D46057390F8265025B1457B9D426F
:104D000038BF1D46457390F8285025B1867BB342C5
:104D100038BF3346837322B919B914B90DB97F234B
:104D2000837303B070BC704738B541F29053C2F240
:104D300001030C461B680546240483F8CF1003F1D9
:104D4000C00004F4FE04013DFFF726FF44F4504484
:104D500045F2D8502D020D2105F47065C0F2020015
:104D600044F00D041AF0B6FE2C4341F2C050214627
:104D7000C2F2010015F03EFB45F220101421C0F2F2
:104D800002001AF0A7FE20461AF01AF845F2381071
:104D9000C0F202000F211AF09DFE4EF24020C2F236
:104DA0000000BDE8384016F0FFBF00BF41F290534D
:104DB000C2F2010370B51B68054683F8CF1003F1FA
:104DC000C0000C46FFF7E8FE45F2E8501221013D15
:104DD000C0F202001AF07EFEE9B20F290FD841F6A8
:104DE0007866C2F2010641F0D001B06C03681B681E
:104DF0009847B06C036804F07F011B68984745F240
:104E000060100F21C0F202001AF064FE230403F4C4
:104E1000FE03280243F4504343F00D0300F4706096
:104E2000184319F0CDFF45F23810C0F202000F21EF
:104E30001AF050FE4EF24020C2F20000BDE8704071
:104E400016F0B2BF41F29053C2F2010370B51B6875
:104E5000054683F8CF1003F1C0000C46FFF79CFE17
:104E600045F2FC500D21013DC0F202001AF032FE65
:104E7000E9B20F290FD841F67866C2F2010641F077
:104E8000D001B06C03681B689847B06C036804F0ED
:104E90007F011B68984745F260100F21C0F20200A5
:104EA0001AF018FE230403F4FE03290243F45043CE
:104EB00043F00D0301F4706141F2C0501943C2F296
:104EC000010015F097FA45F22010C0F202001421FB
:104ED0001AF000FE4EF24020C2F20000BDE8704021
:104EE00016F062BF10B4036841681A780C78417AF2
:104EF000037A0C4202EA03021AD0837A03F0030316
:104F00000AB143F0040343F008039A10082B82729D
:104F10002AD8072B22D2032B2ED011D9042B13D041
:104F2000062B14D1C3685DF8044B023BC360704785
:104F3000837A03F00303002AE7D043F00403E4E795
:104F4000012B0BD0022B02D1C368013BC3605DF87B
:104F5000044B70470D2BF7D00E2BF8D1C3685DF8CA
:104F6000044B0133C36070470C2B05D0F2D8092BDA
:104F7000D8D00B2BE8D0EAE7C3685DF8044B0233C6
:104F8000C36070471D2810B50B4600F0E983024648
:104F900022D92C2800F064813FD8242800F0EE8329
:104FA00040F2A880282800F0748300F2D6802628DA
:104FB00000F0F58140F2D5824AF28854C2F2010431
:104FC00043F67941C0F2000104222720C4F89C3046
:104FD00017F052FC012010BD0E2800F097833AD83C
:104FE000062800F0A1836CD90A2800F0058300F29E
:104FF0000781082800F07E8140F275824AF28854C9
:10500000C2F2010442F2F121C0F20001042209209F
:10501000636217F031FC012010BD342800F0BD831D
:1050200036D8302800F0638300F2D6802E2800F0B6
:10503000528140F201824AF28854C2F2010444F2E1
:10504000D911C0F2000104222F20C4F8BC3017F09F
:1050500013FC012010BD152800F0748364D91928B1
:1050600000F0FA8100F2A580172800F08A8140F252
:10507000D1824AF28854C2F2010443F26521C0F29F
:10508000000104221820236617F0F6FB012010BD52
:10509000382800F0CE8275D8362800F0398140F2E9
:1050A0007F824AF28854C2F2010444F23971C0F29C
:1050B000000104223720C4F8DC3017F0DDFB0120AA
:1050C00010BD022800F0018240F27881042800F02F
:1050D0004B8140F2BD824AF28854C2F2010443F28D
:1050E0006101C0F2000104220520636117F0C4FBD6
:1050F000012010BD202800F0448240F2898122283E
:1051000000F0238140F2D4824AF28854C2F20104B2
:1051100043F6C911C0F2000104222320C4F88C30E8
:1051200017F0AAFB012010BD112800F0B18140F258
:105130005A81132800F0FB8040F2B8814AF288546B
:10514000C2F2010442F65521C0F2000104221420EB
:10515000236517F091FB012010BD2A2800F0AC80D8
:1051600040F2E0814AF28854C2F2010443F6297108
:10517000C0F2000104222B20C4F8AC3017F07CFBF5
:10518000012010BD3A2800F08880C0F072823B28D0
:1051900040F06D824AF28854C2F2010442F2ED01FD
:1051A000C0F200010422C4F8EC3017F065FB0120C6
:1051B00010BD1B2863D040F28B824AF28854C2F2A1
:1051C000010443F21551C0F2000104221C202367A0
:1051D00017F052FB012010BD322824D040F29281FA
:1051E0004AF28854C2F2010444F28941C0F200013B
:1051F00004223320C4F8CC3017F03EFB012010BD50
:105200000C281FD040F29E814AF28854C2F2010459
:1052100042F2A151C0F2000104220D20636317F095
:105220002BFB012010BD4AF28854C2F2010444F263
:10523000DD31C0F200010422C4F8C83017F01CFBB5
:10524000012010BD4AF28854C2F2010442F2F54135
:10525000C0F200010422236317F00EFB012010BDF1
:105260004AF28854C2F2010443F6D571C0F200013B
:105270000422C4F8B03017F0FFFA012010BD4AF242
:105280008854C2F2010443F26941C0F200010422D1
:10529000E36617F0F1FA012010BD4AF28854C2F219
:1052A000010442F24101C0F200010422C4F8E830D6
:1052B00017F0E2FA012010BD4AF28854C2F201044C
:1052C00043F67D61C0F200010422C4F8A83017F053
:1052D000D3FA012010BD4AF28854C2F2010444F20C
:1052E0002D11C0F200010422C4F8B83017F0C4FA3E
:1052F000012010BD4AF28854C2F2010442F2452155
:10530000C0F200010422236217F0B6FA012010BD9A
:105310004AF28854C2F2010444F28D61C0F20001E5
:105320000422C4F8D83017F0A7FA012010BD4AF2C1
:105330008854C2F2010442F6A911C0F2000104220D
:10534000E36417F099FA012010BD4AF28854C2F2C2
:10535000010443F61D11C0F200010422C4F8883094
:1053600017F08AFA012010BD4AF28854C2F20104F3
:1053700042F6B571C0F20001236117F07DFA0120F9
:1053800010BD4AF28854C2F2010442F65941C0F2FB
:1053900000010422E36517F06FFA012010BD4AF204
:1053A0008854C2F2010443F6CD31C0F20001042258
:1053B000C4F8983017F060FA012010BD002800F002
:1053C000FF80012840F053814AF28854C2F2010460
:1053D00042F6B151C0F2000104220120636017F0CF
:1053E0004BFA012010BD0F2800F0F880102840F083
:1053F0003E814AF28854C2F2010442F2A571C0F221
:10540000000104221020236417F036FA012010BD99
:105410001E282FD01F2840F02A814AF28854C2F259
:10542000010443F21971C0F2000104221F20E36756
:1054300017F022FA012010BD4AF28854C2F201048A
:1054400044F28101C0F2000104222D20C4F8B430DE
:1054500017F012FA012010BD4AF28854C2F201047A
:1054600043F21131C0F200010422636617F004FA1E
:10547000012010BD4AF28854C2F2010443F26D616A
:10548000C0F200010422A36717F0F6F9012010BD55
:105490004AF28854C2F2010442F65101C0F20001FE
:1054A0000422636417F0E8F9012010BD4AF2885421
:1054B000C2F2010442F6FD01C0F2000104221220F2
:1054C000A36417F0D9F9012010BD4AF28854C2F242
:1054D000010442F65D61C0F200010422A36017F0EE
:1054E000CBF9012010BD4AF28854C2F2010443F204
:1054F000B911C0F2000104220720E36117F0BCF9E2
:10550000012010BD4AF28854C2F2010444F2313144
:10551000C0F2000104223120C4F8C43017F0ACF905
:10552000012010BD4AF28854C2F2010443F6D15161
:10553000C0F2000104222920C4F8A43017F09CF91D
:10554000012010BD4AF28854C2F2010442F24941DE
:10555000C0F2000104220B20E36217F08DF9012054
:1055600010BD4AF28854C2F2010443F62131C0F260
:10557000000104222520C4F8943017F07DF90120A1
:1055800010BD4AF28854C2F2010443F2C571C0F260
:1055900000010422C4F8803017F06EF9012010BD1C
:1055A0004AF28854C2F2010444F2E151C0F200010F
:1055B00004223520C4F8D43017F05EF9012010BD64
:1055C0004AF28854C2F2010442F60551C0F20001C9
:1055D0000422236017F050F9012010BD4AF28854CC
:1055E000C2F2010442F2F961C0F200010422E36355
:1055F00017F042F9012010BD4AF28854C2F20104AA
:1056000042F29D31C0F200010422A36217F034F986
:10561000012010BD4AF28854C2F2010442F6AD31B5
:10562000C0F2000104221620A36517F025F901201D
:1056300010BD4AF28854C2F2010441F69571C0F2DD
:1056400000010422C4F8E03017F016F9012010BD63
:105650004AF28854C2F2010442F60971C0F2000114
:1056600004220320E36017F007F9012010BD002099
:1056700010BD4AF28854C2F2010442F29911C0F2FC
:10568000000104223920C4F8E43017F0F5F80120B5
:1056900010BD4AF28854C2F2010443F62551C0F20B
:1056A00000010422C4F8A03017F0E6F8012010BD74
:1056B0004AF28854C2F2010443F67101C0F20001BB
:1056C00004222120C4F8843017F0D6F8012010BD40
:1056D0004AF28854C2F2010443F2BD31C0F2000123
:1056E00004221A20A36617F0C7F8012010BD4AF261
:1056F0008854C2F2010444F28521C0F20001042260
:10570000C4F8C03017F0B8F8012010BD4AF2885430
:10571000C2F2010442F24D61C0F200010422A3630F
:1057200017F0AAF8012010BD4AF28854C2F2010411
:1057300043F20D11C0F200010422A36117F09CF89E
:10574000012010BD4AF28854C2F2010442F6013130
:10575000C0F200010422636517F08EF8012010BD2D
:105760004AF28854C2F2010443F2C151C0F200016E
:105770000422636717F080F8012010BD4AF28854B4
:10578000C2F2010443F67521C0F200010422C4F8FC
:10579000903017F071F8012010BD4AF28854C2F21F
:1057A000010444F23551C0F200010422C4F8D030A3
:1057B00017F062F8012010BDF8B5044615460E46F4
:1057C0000846022117F0D0FA2846022117F0CCFA39
:1057D00046F68403C0F20203012253F83600227217
:1057E00000F50071216053F8351062724DF2C0432C
:1057F00001F5007762F31F4300226760E260013B1E
:10580000FDD190F8003291F8002203F00103D20795
:1058100044BF43F00203DBB2A37221463046FFF7D8
:10582000B1FB214620742846FFF7ACFB237C1844CB
:1058300020742046F8BD00BFF8B5064645F20C605E
:105840000F46C0F202000B211AF044F94EF240203C
:105850003946C2F2000000230A2216F0B7FA45F2D8
:105860001860C0F2020001211AF034F9B7B1002526
:105870002C4645F63C100121C0F202001AF02AF92C
:1058800001344EF24020715DE4B2C2F20000002308
:105890000A2216F09BFAA7422546EAD84EF240208B
:1058A000C2F2000016F080FA4DF6A863C2F20003BF
:1058B0001B7C73B1B07800F00F000130834208D038
:1058C000FBF782FA28B945F21C60C0F202001B21E6
:1058D00007E07378432B0ED045F23860C0F2020027
:1058E0001B211AF0F7F84EF24020C2F20000BDE88A
:1058F000F84016F059BA45F254600C21C0F202008B
:105900001AF0E8F8B1784EF24020C1F30211C2F269
:10591000000016F0EBF945F218600121C0F2020018
:105920001AF0D8F84EF24020C2F2000016F03CFA0D
:10593000072F05D045F2EC60C0F202002021D0E72D
:10594000F378C3F38403002B00F0C680022B40F0F1
:10595000F180B379F72B40F0C28041F29053C2F24C
:10596000010331791B6872794AF6AB2001F07F019F
:10597000C3F6AA5007EE100A581802F07F023171E0
:10598000727180F8C82193F80A4293F8075293F88D
:105990000C0293F80872C3F8C45093F8095293F8B4
:1059A0000E2293F81012C3F8C87083F8D95004F08F
:1059B0000107C4F34005C4F3800493F80BE283F8B5
:1059C000DA7083F8DB5000F0010783F8DC40C0F3A5
:1059D000400593F80D4283F8DDE0C0F3800083F8C2
:1059E000DE7002F0010E83F8DF5083F8E00093F8D8
:1059F0000F5283F8E140C1F3400001F00104C2F30B
:105A00004007C2F3800283F8E42083F8E64083F87D
:105A1000E2E083F8E37083F8E55083F8E70093F859
:105A20001122520607EE902AF8EEE77AC1F38001C0
:105A300067EE877A83F8E810FDEEE77A03F1C0009D
:105A4000C3ED357AFFF7A8F834795C34E4B245F257
:105A50003470C0F20200FAF7A5FFF37813F07C0F60
:105A600005D145F2C460C0F20200FAF79BFF45F28F
:105A7000D060C0F20200FAF795FF4EF24020317973
:105A800000230A22C2F2000016F0A0F945F2E860F5
:105A9000C0F20200FAF786FF4EF24020717900232F
:105AA0000A22C2F2000016F091F945F2DC60C0F261
:105AB0000200FAF777FF4EF2402021460023C2F29F
:105AC00000000A2216F082F94EF24020C2F20000D5
:105AD000BDE8F84016F068B9B379F72B07D045F266
:105AE0009C60C0F20200BDE8F840FAF765BF327969
:105AF000737941F29054C2F2010402F07F0203F084
:105B00007F0320683271737109F0FAFEF2783379FD
:105B10002068717902F0030203EBC213034483F897
:105B20006C1109F0E1FDF478337903EBC41404F04F
:105B3000FF048CE745F26460C0F20200BDE8F84063
:105B4000FAF73ABF38B504460D46FFF775FE45F241
:105B500010701021C0F2020019F0BCFF41F2C050D9
:105B600000232A462146C2F2010014F081FC45F2CE
:105B700020101421C0F2020019F0ACFF2946204683
:105B8000002219F071F945F23810C0F202000F211D
:105B900019F0A0FF4EF24020C2F20000BDE83840EC
:105BA00016F002B92DE9F04141F678650F468046BE
:105BB000C2F20105FFF740FE45F224701521C0F244
:105BC000020019F087FFA86C0368F021DB6C98478E
:105BD00057B1444608EB0706A86C14F8011B03688C
:105BE0001B689847A642F7D1A86C0368F721DB6CC5
:105BF000984745F260100F21C0F2020019F06AFFC9
:105C000039464046002219F02FF945F23810C0F20B
:105C100002000F2119F05EFF4EF24020C2F2000098
:105C2000BDE8F04116F0C0B82DE9F04141F67865C5
:105C30000F468046C2F20105FFF7FEFD45F23C70BB
:105C40001021C0F2020019F045FFA86C0368F02192
:105C5000DB6C984757B1444608EB0706A86C14F86C
:105C6000011B03681B689847A642F7D1A86C03681C
:105C7000F721DB6C984745F260100F21C0F202005B
:105C800019F028FF41F2C0503A464146C2F20100E5
:105C9000002314F0EDFB45F22010C0F202001421A5
:105CA00019F018FF4EF24020C2F20000BDE8F041AA
:105CB00016F07AB8FFFFFFFF38B545F2507010EECE
:105CC000105A4DF6A8642DED048BC2F20004142185
:105CD000C0F20200B0EE608AC4ED030A84ED020A4D
:105CE00019F0F8FE28461DF051FE41EC100B4EF263
:105CF00040200A21C2F2000016F0A8F845F26870B0
:105D00000121C0F2020019F0E5FE40F6DB73C4F297
:105D10004903A06809EE103A1DF038FE41EC100B63
:105D20004EF240200A21C2F2000016F08FF845F230
:105D30006C700621C0F2020019F0CCFE45F26870CA
:105D40000121C0F2020019F0C5FEE0681DF01EFE40
:105D500041EC100B4EF240200A21C2F2000016F076
:105D600075F845F274700221C0F2020019F0B2FE1B
:105D7000E36807EE903A27EE890AF6EE008A20EEF5
:105D8000280A1AF041FEA36807EE903A60EE277ADF
:105D900017EE900A1DF0FAFD9FED511B41EC100B20
:105DA0001AF032FF4EF240200321C2F2000016F03A
:105DB0004DF845F278700121C0F2020019F08AFE18
:105DC000E36807EE903A27EE890A20EE280A1AF0D7
:105DD000CBFDA36807EE903A60EE277A17EE900AA3
:105DE0001DF0D4FD9FED3E1B41EC100B1AF00CFF93
:105DF0004EF240200321C2F2000016F027F84EF2C6
:105E00004020C2F2000015F0CFFF41F2905328EE7F
:105E1000098AC2F2010328EE288A1B68B0EE480AFC
:105E2000C3F868511AF0F0FD4FF47E43C4F2FF63EB
:105E300007EE903AB4EEE70AF1EE10FA0EDC4FF4FA
:105E40007E43CCF2FF6307EE903AB4EEE70AF1EE40
:105E500010FA30D50023C8F2010302E00023C7F690
:105E6000FF7341F23452C2F20102B0EE480A93616C
:105E70001AF07AFD4FF47E43C4F2FF6307EE903AC6
:105E8000B4EEE70AF1EE10FA23DC4FF47E43CCF2D5
:105E9000FF6307EE903AB4EEE70AF1EE10FA11D57F
:105EA0000023C8F20103BDEC048B41F26442C2F24C
:105EB0000102936138BDF0EE407AFEEEC87A17EE2B
:105EC000903ACEE7F0EE407AFEEEC87A17EE903ABE
:105ED000E9E70023C7F6FF73E5E700BFAFF30080F3
:105EE0000000002085EBB13F2DE9F041044645F26A
:105EF0007C700D46C0F20200032119F0EBFD4EF25A
:105F0000402000230A222146C2F2000015F05EFF65
:105F100045F280700121C0F2020019F0DBFD4EF263
:105F20004020294600230A22C2F2000015F04EFF4D
:105F30004EF24020C2F2000015F036FF672C00F050
:105F4000CF8150D9782C00F0A28000F28C80692C8F
:105F500000F0C080C0F09C816A2C00F05D816B2C49
:105F600040F06782002301EE903A05EB45050023DF
:105F7000C4F2482305EB051501EE103AC5F3C7132B
:105F800007EE903A41F67462C2F20102B8EE670A77
:105F9000F0EE610AB7EE002A137003F065FE4FF4CD
:105FA0007E43C4F2FF6307EE903AB4EEE70AF1EEE7
:105FB00010FA00F3D5814FF47E43CCF2FF6307EE75
:105FC000903AB4EEE70AF1EE10FA40F13482002381
:105FD000C8F2010341F2BC42C2F20102BDE8F04145
:105FE000D36106F0E1B9042C00F0A28140F2C9802F
:105FF0000A2C5ED040F2E480202C00F00681402C78
:1060000040F0308241F29056C2F201063F2D94BF1B
:1060100000210121306809F073FB306809F078FB3A
:106020000546002840F0AB803068374609F00CFD8B
:10603000EBB203EB430498424FEA840440F29F80A2
:10604000306803190135DA78002AEFD093F802801E
:10605000B8F1000FEAD198680BF042F838680444B0
:1060600084F80380E2E77B2C1AD040F29D807E2CDE
:1060700000F0C1807F2C40F0F78141F29053C2F2D2
:10608000010300211868BDE8F04109F031BB41F27D
:106090009053C2F20103BDE8F041186809F03CBB1F
:1060A00041F29053C2F20103BDE8F041186809F0D3
:1060B00027BC4DF6A863C2F2000300EE905A9A681E
:1060C000FBEEEC0A00EE102ABDE8F041C3ED030A36
:1060D000FFF7F2BD002301EE903A0023C4F296438D
:1060E00002EE103A05EB45050023C4F2482305EB08
:1060F000051501EE103AC5F3C71307EE903A40F2CA
:106100006C52C2F20102B8EE670AF0EE610A137037
:1061100003F0AAFDB5EEC00AF1EE10FA00F13181EC
:1061200047F67903C4F2302307EE103AF6EE007A10
:10613000E0EE077A49F68073C0F20103FCEEE77ADD
:1061400017EE902A9A4240F284811A464FF450701A
:1061500040F22073C2F20103197ECC0700F11481D2
:10616000DC8B1A62844241F0010138BFD883197672
:10617000BDE8F04106F018B9632D40F2F980BDE8A2
:10618000F081012C00F0E080F6D3022C40F04F812A
:1061900041F29053C2F20103186880F8D050C03029
:1061A000FEF7FAFCBDE8F081792C40F0598141F20C
:1061B0009053C2F20103BDE8F041186809F0C0BA7B
:1061C000072C40F04B8107EE905A0023C4F2FE23C7
:1061D000B8EE677A07EE903A87EE270A4DF6A86385
:1061E000C2F20003BDE8F041DA6800EE902A83EDC8
:1061F000020AFFF761BD41F29053C2F2010301218F
:106200001868BDE8F04109F073BA4DF6A863C2F210
:1062100000031D71BDE8F08105EBC5050022C5F343
:10622000471501EE902A07EE905A41F6F0430022FE
:10623000C2F20103C4F20C22B8EE670A01EE102A82
:10624000F0EE610AB7EE002A1D7003F00DFD4FF469
:106250007E43C4F2FF6307EE903AB4EEE70AF1EE34
:1062600010FA00F381804FF47E43CCF2FF6307EE17
:10627000903AB4EEE70AF1EE10FA40F1E380002321
:10628000C8F2010341F28442C2F20102D3616FE716
:106290002DB205EB850303EB830305EB8305C5F303
:1062A000C71507EE905A0023C4F2C823F8EE676AB8
:1062B00007EE903A86EEA77A41F29052C2F20102BE
:1062C00040F21C03C2F2010312681D70BDE8F041E8
:1062D000F7EE007A77EEC77AC2ED587A06F064B826
:1062E0002DB205EB850303EB830305EB8305C5F3B3
:1062F000C71507EE905A0023C4F2C823F8EE676A68
:1063000007EE903A86EEA77A41F29052C2F201026D
:1063100041F6F143C2F2010312681D70BDE8F0417D
:10632000F7EE007A77EEC77AC2ED597A06F03CB8FC
:1063300041F29053C2F20103186880F8D150C03086
:10634000FEF72AFCBDE8F08141F29053C2F201034E
:10635000186880F8D250C030FEF71EFCBDE8F0810E
:106360000023C7F6FF7335E60023C7F6FF7389E7FE
:106370004DF6A863C2F200031D71BDE8F04106F0BE
:1063800013B801200022E3E61C6AA24205D9D98B8A
:106390001A62884288BFD883EAE602F17F00C0090A
:1063A000013000281A62024638BF0022880706D54D
:1063B000586A7F30C0090130824238BF02464F0719
:1063C00006D5986A7F30C0090130824238BF024644
:1063D0000E0706D5D86A7F30C0090130824238BF27
:1063E0000246CD0606D5186B7F30C00901308242C7
:1063F00038BF02468C0606D5586B7F30C009013085
:10640000824238BF0246480606D5986B7F30C009E5
:106410000130824238BF0246C90906D0D96B7F31AC
:10642000C90901318A4238BF0A46DA83A0E6BDE8CD
:10643000F081BDE8F081F0EE407AFEEEC87A17EE0A
:10644000903AC7E5F0EE407AFEEEC87A17EE903A41
:1064500018E702F17F00C009013079E6BDE8F0815C
:10646000BDE8F081BDE8F081BDE8F081F8B54DF6FA
:10647000A863C2F200030E461B7C1446054623B1F6
:10648000984202D0FAF7A0FC18B121463046FFF737
:106490002BFD45F284700D21013DC0F2020019F080
:1064A00019FBE9B20F2915D841F67867C2F2010746
:1064B00041F0B001B86C03681B689847B86C03687A
:1064C00006F07F011B689847B86C036804F07F01F1
:1064D0001B68984745F260100F21C0F2020019F0C6
:1064E000F9FA230603F0FE43310443F4304301F488
:1064F000FE012D0243F00B030B4341F2C05005F4A3
:1065000070611943C2F2010013F074FF45F22010CC
:10651000C0F20200142119F0DDFA4EF24020C2F25E
:106520000000BDE8F84015F03FBC00BFF8B54DF6DF
:10653000A863C2F200030E461B7C1446054623B135
:10654000984202D0FAF740FC18B121463046FFF7D6
:10655000CBFC45F294701221013DC0F2020019F00B
:10656000B9FAE9B20F2915D841F67867C2F20107E6
:1065700041F0B001B86C03681B689847B86C0368B9
:1065800006F07F011B689847B86C036804F07F0130
:106590001B68984745F260100F21C0F2020019F005
:1065A00099FA230603F0FE43310443F4304301F427
:1065B000FE01280243F00B030B4300F47060184304
:1065C00018F0FEFB45F23810C0F202000F2119F05E
:1065D00081FA4EF24020C2F20000BDE8F84015F00A
:1065E000E3BB00BF70B54DF6A863C2F200030E46D0
:1065F0001B7C1446054623B1984202D0FAF7E4FB0F
:1066000018B121463046FFF76FFC45F2A8700D2106
:10661000C0F2020019F05EFA230603F0FE433404D0
:1066200043F43043013D43F00B0304F4FE042D0218
:106630001C4305F470652C4341F2C0502146C2F260
:10664000010013F0D7FE45F220101421C0F2020021
:1066500019F040FA204618F0B3FB45F23810C0F2AA
:1066600002000F2119F036FA4EF24020C2F200006B
:10667000BDE8704015F098BB4AF23473C2F20103D2
:1066800082B01B68019341F67062C2F2010240F2CF
:10669000CC53C2F201030199116001221A7002B0B9
:1066A000704700BF45F2C8032DE9F04FC0F2020366
:1066B0001C460FCCB1B020AD0FC50FCC0FC50FCC11
:1066C0000FC594E80F0010944DF6A86740F2CC5423
:1066D000C2F20007C2F201044FF0000E84F800E09D
:1066E0001F9585E80F00BD7A0395FD7A3B790495E7
:1066F0003D7B05957D7B06956FEA0309BD7B07957C
:1067000009F00F0930AD05EB8909BA7997F80580D2
:10671000787A02901D1159F8403C11951146FA798A
:10672000139183F070431446DB433A7A019283EA73
:1067300005020DF1C00E02F00F020EEB82024FEACD
:10674000281E52F8402C82EA1313DB4383EA080226
:10675000754602F00F020DF1C00E0EEB82020DF134
:10676000C00E52F8402C129582EA131383EA0502F8
:1067700002F00F020EEB82020DF1C00E52F8402C17
:1067800082EA1313DB4383EA010202F00F020EEBED
:106790008202081152F8402C0199064682EA13132E
:1067A00083EA06020DF1C00E02F00F020EEB820228
:1067B000081114960990029852F8402C159482EA18
:1067C0001313DB4383EA04020DF1C00E02F00F0243
:1067D0000EEB8202251152F8402C039C169582EA9A
:1067E000131383EA05020DF1C00E02F00F020EEB47
:1067F00082020DF1C00E52F8402C82EA13136FEAA8
:10680000030C8CEA010202F00F0205990EEB8202E2
:106810000B1152F8402C0C93099B82EA1C1C8CEA49
:1068200003020DF1C00E02F00F020EEB8202069B76
:1068300052F8402C1B110D9382EA1C13DB4383EAB0
:106840000002061102F00F0207980A960DF1C00E21
:106850000EEB820E02110E925EF8402C82EA1313A8
:106860000A9A5A4002F00F020DF1C00E0EEB820E92
:10687000109AA2F1300C5EF8402C82EA1313DB432D
:1068800083EA04020DF1C00E02F00F020EEB820249
:1068900026110B9652F8402C0B9C049E82EA13138F
:1068A00083EA04020DF1C00A02F00F020AEB820231
:1068B000351152F8402C179582EA1313DB4383EA13
:1068C000060202F00F020AEB82020DF1C00A52F832
:1068D000402C0C9E82EA131383EA050202F00F0299
:1068E0000AEB82020DF1C00A52F8402C82EA13131F
:1068F000DB4383EA010202F00F020AEB82020DF190
:10690000C00A52F8402C82EA131383EA060202F00E
:106910000F020AEB82020DF1C00A52F8402C069ECB
:106920000E9D97F813B082EA1313DB4383EA060245
:1069300002F00F020AEB82020D9E52F8402C82EA0E
:10694000131383EA06020DF1C00A02F00F020AEBEC
:1069500082020DF1C00A52F8402C82EA1313DB4385
:1069600083EA000202F00F020AEB82020DF1C00A74
:1069700052F8402C82EA131383EA050202F00F0258
:106980000AEB820297F80FA052F8402C564697F86F
:1069900010A01896514697F811A01A9182EA131385
:1069A0005046DB4397F812A083EA0602554602F0F0
:1069B0000F020DF1C00A0AEB8202361152F8402C88
:1069C000199682EA131383EA06020DF1C00A02F057
:1069D0000F020AEB82020DF1C00A52F8402C1D95FD
:1069E00082EA1313DB4383EA010202F00F020AEB8F
:1069F00082020E1152F8402C0F9682EA13130F9A5E
:106A00005A400DF1C00A02F00F020AEB820206465C
:106A100052F8402C1B9682EA1313DB4383EA0602EA
:106A20000DF1C00A02F00F020AEB8202011152F8C6
:106A3000402C1C9182EA131383EA01024FEA2B1ABD
:106A4000CDF820A002F00F020DF1C00A0AEB82027D
:106A50000DF1C00A52F8402C82EA1313DB4383EA9B
:106A6000050202F00F020AEB8202281152F8402CB4
:106A70001E9082EA131383EA00020DF1C00A02F0AD
:106A80000F020AEB820230AE52F8402C82EA131356
:106A9000DB438BEA030202F00F020AEB82020DF1E4
:106AA000800E52F8402C82EA131A089B55468AEA57
:106AB000030ABCE80F000AF00F0A06EB8A0A3C46FC
:106AC0005AF840ACAEE80F00BCE80F00AEE80F008B
:106AD000BCE80F00AEE80F0059F8402C8AEA151AFE
:106AE00082F07042119DD24382EA050303F00F0346
:106AF00006EB83030DF1C00E53F8403C83EA1212FB
:106B0000D24382EA080303F00F0306EB83036FEA24
:106B10000A0A53F8403CC7F800A083EA1212129BFD
:106B2000534003F00F030EEB83030DF1C00E53F837
:106B3000403C1398019983EA1212D24382EA00037F
:106B400003F00F030EEB8303149853F8403C83EAE1
:106B5000121282EA00030DF1C00E03F00F030EEBD8
:106B60008303159853F8403C83EA1212D24382EA19
:106B700000030DF1C00E03F00F030EEB8303169814
:106B800053F8403C83EA121282EA00030DF1C00E72
:106B900003F00F030EEB83030DF1C00E53F8403CDE
:106BA000099883EA1212D24382EA010303F00F0329
:106BB0000EEB83030DF1C00E53F8403C059983EAB8
:106BC000121282EA000303F00F030EEB8303029814
:106BD00053F8403C83EA1212D24382EA00030DF1DB
:106BE000C00E03F00F030EEB83030A9853F8403CEA
:106BF00083EA121282EA00030DF1C00E03F00F03C4
:106C00000EEB83030DF1C00E53F8403C0B9883EA62
:106C10001212039BD243534003F00F030EEB830386
:106C20000DF1C00E53F8403C83EA121282EA0003D1
:106C300003F00F030EEB83030DF1C00E53F8403C3D
:106C4000179883EA1212049BD243534003F00F03B8
:106C50000EEB83030DF1C00E53F8403C83EA121291
:106C600082EA000303F00F030EEB83030DF1C00E65
:106C700053F8403C0C9883EA1212D24382EA010393
:106C800003F00F030EEB83030DF1C00E53F8403CED
:106C900083EA121282EA000303F00F030EEB830370
:106CA0000DF1C00E53F8403C0D9883EA1212069B7A
:106CB000D243534003F00F030EEB83030DF1C00EDC
:106CC00053F8403C83EA121282EA000303F00F03F8
:106CD0000EEB83030DF1C00E53F8403C07981A9950
:106CE00083EA1212D24382EA000303F00F030EEB91
:106CF00083030E9853F8403C83EA121282EA0003A1
:106D00000DF1C00E03F00F030EEB83030DF1C00E67
:106D100053F8403C199883EA1212189BD24353400F
:106D200003F00F030EEB83030DF1C00E53F8403C4C
:106D300083EA121282EA000303F00F030EEB8303CF
:106D40000DF1C00E53F8403C1E9883EA1212D24354
:106D500082EA010303F00F030EEB83030F9953F84C
:106D6000403C83EA121282EA01030DF1C00E03F0E7
:106D70000F030EEB83030DF1C00E53F8403C1C993A
:106D800083EA12121B9BD243534003F00F030EEB16
:106D9000830307F1140553F8403C83EA121282EA98
:106DA000010303F00F030EEB8303FE4353F8403C53
:106DB00083EA12121D9BD243534003F00F030EEBE4
:106DC000830353F8403C83EA121282EA000303F083
:106DD0000F030EEB830353F8403C83EA1212D243B5
:106DE0008BEA020303F00F030EEB830353F8403CDE
:106DF00083EA1212089B534003F00F030EEB830348
:106E000053F8403C83EA1213DB433B7014F8018BC8
:106E1000A719384615F01CFA80454146384601D07E
:106E200015F030FAAC42F1D145F2B8702721C0F22A
:106E3000020018F04FFE4EF24020C2F2000031B0C6
:106E4000BDE8F04F14F0B0BFF0B597B001AD2C46DF
:106E500006AE601B15F0FCF904F8010BB442F8D142
:106E600045F2C805C0F202050FCD0FC40FCD0FC407
:106E70000FCD0FC495E80F0084E80F009DF808605F
:106E80009DF809509DF80A409DF80B209DF80C30A4
:106E90009DF80D009DF80E10F7430DF1580E07F008
:106EA0000F070EEB870757F8407C87F07047FF43CA
:106EB00087EA161606F00F060EEB860656F8406CAB
:106EC00086EA1716F64385EA060707F00F070EEB6A
:106ED000870757F8407C87EA161787EA151606F0E9
:106EE0000F060EEB86069DF80F5056F8406C86EAAA
:106EF0001716F64384EA060707F00F070EEB87071D
:106F000057F8407C87EA161787EA141606F00F0632
:106F10000EEB86069DF8104056F8406C86EA171670
:106F2000F64382EA060707F00F070EEB870757F8CC
:106F3000407C87EA161787EA121606F00F060EEB5A
:106F400086069DF8112056F8406C86EA1716F6431F
:106F500083EA060707F00F070EEB870757F8407C18
:106F600087EA161787EA131606F00F060EEB860659
:106F70009DF8123056F8406C86EA1716F64380EA00
:106F8000060707F00F070EEB870757F8407C87EAE4
:106F9000161787EA101606F00F060EEB860645F266
:106FA000E07056F8406C86EA1716F64381EA060749
:106FB00007F00F070EEB8707C0F2020057F8407C7E
:106FC00087EA161787EA111606F00F060EEB8606FB
:106FD000132156F8406C86EA1716F64385EA060731
:106FE00007F00F070EEB870757F8407C87EA161665
:106FF00086EA151505F00F050EEB850555F8405C82
:1070000085EA1615ED4384EA050606F00F060EEB39
:10701000860656F8406C86EA151585EA141404F0C5
:107020000F040EEB840454F8404C84EA1514E44336
:1070300082EA040505F00F050EEB850555F8405C66
:1070400085EA141484EA121202F00F020EEB820297
:1070500052F8402C82EA1412D24383EA020404F06C
:107060000F040EEB840454F8406C86EA121787EA8A
:10707000131303F00F030EEB830353F8406C9DF8DA
:1070800013309DF814509DF815409DF8162086EA9F
:107090001716F64383EA060707F00F070EEB87077C
:1070A00057F8407C87EA161787EA131606F00F0692
:1070B0000EEB86069DF8173056F8406C86EA1716D8
:1070C000F64385EA060707F00F070EEB870757F828
:1070D000407C87EA161686EA151505F00F050EEBBB
:1070E000850555F8405C85EA1615ED4384EA0506EA
:1070F00006F00F060EEB860656F8406C86EA15156C
:1071000085EA141404F00F040EEB840454F8404C88
:1071100084EA1514E44382EA040505F00F050EEB3A
:10712000850555F8405C85EA141484EA121202F0D1
:107130000F020EEB820252F8402C82EA1412D24364
:1071400083EA020404F00F040EEB840454F8404C6C
:1071500084EA121484EA131303F00F030EEB830383
:1071600053F8403C83EA141418F0B4FC019D4EF22D
:107170004020002310222946C2F2000014F026FE0F
:1071800045F2F4700521C0F2020018F0A3FCE443BC
:107190004EF240202146C2F200000023102214F0DB
:1071A00015FEA5421DD14DF6A865C2F2000505F1F8
:1071B00014062C46601B15F04BF804F8010BB44282
:1071C000F8D145F62000C0F202000F2118F082FC31
:1071D0004EF24020C2F2000017B0BDE8F04014F0BB
:1071E000E3BD45F2FC702321C0F2020018F072FCEE
:1071F000FFF758FAECE700BF2DE9F8434AF20E79A1
:10720000C2F2010945F630002DED028B0521C0F2D6
:10721000020018F05FFCB9F8003007EE103A43F2B4
:107220003333C4F2233308EE903AB8EEC77A43F210
:107230003333C4F2A33308EE103A37EE287A4EF215
:107240004024C7EE087AC2F200044AF20877C2F27C
:1072500001074AF20C78C2F201084AF28C66C2F2C7
:10726000010640F22C05C2F2010517EE900A1CF04F
:107270008DFB41EC100B0221204614F0E7FD45F692
:1072800038000D21C0F2020018F024FC3B8807EE04
:10729000903AF8EEE77A77EEA87A87EE887A17EEDA
:1072A000100A1CF073FB41EC100B0221204614F075
:1072B000CDFD45F648000821C0F2020018F00AFC96
:1072C000B8F80010204614F011FD45F654000C21CA
:1072D000C0F2020018F0FEFB3188204614F006FDD3
:1072E00045F664001421C0F2020018F0F3FB29886F
:1072F000204614F0FBFC45F67C000921C0F2020098
:1073000018F0E8FB41F23053C2F201030A22196877
:107310002046002314F05AFD45F688000D21C0F2E6
:10732000020018F0D7FB40F22003C2F201030A2248
:1073300019682046002314F049FD45F698000921FC
:10734000C0F2020018F0C6FB41F6A043C2F20103EE
:107350000A2219682046002314F038FD45F6A400DF
:107360000C21C0F2020018F0B5FB8021204614F079
:10737000BDFC45F6B4001021C0F2020018F0AAFBD3
:1073800041F6CD43C2F201030A22197820460023B8
:1073900014F01CFD204614F007FDBDEC028BB9F87B
:1073A0000030B8F800203B80002332802B80BDE8FD
:1073B000F88300BF70B584B0002441F29055029468
:1073C0000194CDF80B40C2F20105062645F6C8002F
:1073D0000221C0F2020018F07DFB4EF2402031463F
:1073E000C2F2000014F082FC45F628200221C0F20F
:1073F000020018F06FFB4EF24020C2F2000014F0C1
:10740000D3FC45F6CC005621C0F2020018F062FB16
:107410004EF24020C2F2000014F0C6FC2B68234458
:107420004EF2402093F86C110A220023C2F20000B1
:1074300014F0CCFC45F63C100121C0F2020018F01B
:1074400049FB2B6823444EF2402093F86D110A2229
:107450000023C2F2000014F0B9FC45F63C100121F3
:10746000C0F2020018F036FB2B6823444EF2402095
:1074700093F86E110A220023C2F2000014F0A6FC59
:1074800045F63C100121C0F2020018F023FB2B68E6
:1074900023444EF2402093F86F110A220023C2F2D7
:1074A000000014F093FC45F63C100121C0F20200EC
:1074B00018F010FB2B6823444EF2402093F8701113
:1074C0000A220023C2F2000014F080FC45F63C10B2
:1074D0000121C0F2020018F0FDFA2B6823444EF29D
:1074E000402093F871110A220023C2F2000014F028
:1074F0006DFC45F63C100121C0F2020018F0EAFADA
:107500002B6823444EF2402093F872110A22002384
:10751000C2F2000014F05AFC45F63C100121C0F202
:10752000020018F0D7FA2B6823444EF2402093F85B
:1075300073110A220023C2F2000014F047FC45F642
:1075400024100821C0F2020018F0C4FA2B6823446A
:107550004EF2402093F874110A220023C2F2000078
:1075600014F034FC45F630100D21C0F2020018F082
:10757000B1FA2B6823444EF2402093F875110A2289
:107580000023C2F2000014F021FC45F630100D215A
:10759000C0F2020018F09EFA2B6823444EF24020FD
:1075A0000A2293F87611C2F20000002314F00EFCB8
:1075B0004EF24020C2F2000014F0F6FB45F64010F7
:1075C0005C21C0F2020018F085FA4EF24020C2F2AF
:1075D000000014F0E9FB45F6A0100621C0F20200FD
:1075E00018F078FA2B6823444EF2402093F8771174
:1075F0000A220023C2F2000014F0E8FB45F6341022
:107600000921C0F2020018F065FA2B6823444EF2FB
:10761000402093F878110A220023C2F2000014F0EF
:10762000D5FB45F634100921C0F2020018F052FAD9
:107630002B6823444EF2402093F879110A2200234C
:10764000C2F2000014F0C2FB45F624100821C0F27B
:10765000020018F03FFA2B6823444EF2402093F8C2
:107660007A110A220023C2F2000014F0AFFB45F6A3
:1076700038100521C0F2020018F02CFA2B682344C0
:107680004EF2402093F87B110A220023C2F2000040
:1076900014F09CFB45F6A0100621C0F2020018F081
:1076A00019FA2B6823444EF2402093F87C110A22E9
:1076B0000023C2F2000014F089FB45F6A010062159
:1076C000C0F2020018F006FA2B6823444EF2402064
:1076D00093F87D110A220023C2F2000014F076FB19
:1076E00045F628100421C0F2020018F0F3F92B68C7
:1076F00023444EF2402093F87E110A220023C2F266
:10770000000014F063FB45F638100521C0F20200BA
:1077100018F0E0F92B6823444EF2402093F87F11D3
:107720000A220023C2F2000014F050FB45F6381084
:107730000521C0F2020018F0CDF92B6823444EF267
:10774000402093F880110A220023C2F2000014F0B6
:107750003DFB4EF240201534C2F2000014F024FB31
:107760007E2C06F1FF367FF431AE45F6A8102D21B0
:10777000C0F2020018F0AEF94EF24020C2F2000052
:1077800014F012FB45F63C10C0F20200012118F083
:10779000A1F92B6823444EF2402093F86C110A2281
:1077A0000023C2F2000014F011FB45F6A4100134CE
:1077B000C0F20200022141F2905618F08BF9862C9B
:1077C000C2F20106E5D14EF24020C2F2000014F0F0
:1077D000EBFA45F6D8100521C0F2020018F07AF94C
:1077E00033684EF2402093F8F2110A220023C2F2CD
:1077F000000014F0EBFA4EF24020C2F2000014F048
:10780000D3FA45F6E0100421C0F2020018F062F944
:1078100033684EF2402093F8F3110A220023C2F29B
:10782000000014F0D3FA4EF24020C2F2000014F02F
:10783000BBFA45F6E8100521C0F2020018F04AF93B
:1078400033684EF2402093F8F4110A220023C2F26A
:10785000000014F0BBFA4EF24020C2F2000014F017
:10786000A3FA45F6F0100921C0F2020018F032F92F
:1078700033684EF2402093F8F5110A220023C2F239
:10788000000014F0A3FA4EF24020C2F2000014F0FF
:107890008BFA45F6FC100921C0F2020018F01AF923
:1078A00033684EF2402093F8F6110A220023C2F208
:1078B000000014F08BFA4EF24020C2F2000014F0E7
:1078C00073FA45F608200921C0F2020018F002F907
:1078D00033684EF2402093F8F7110A220023C2F2D7
:1078E000000014F073FA4EF24020C2F2000014F0CF
:1078F0005BFA45F614200921C0F2020018F0EAF8FC
:1079000033684EF2402093F8F8110A220023C2F2A5
:10791000000014F05BFA4EF24020C2F2000014F0B6
:1079200043FA45F620200A21C0F2020018F0D2F8EE
:1079300033684EF2402093F8F9110A220023C2F274
:10794000000014F043FA4EF24020C2F2000014F09E
:107950002BFA45F62C200D21C0F2020018F0BAF8DF
:1079600033684EF2402093F8FA110A220023C2F243
:10797000000014F02BFA4EF24020C2F2000014F086
:1079800013FA45F63C200921C0F2020018F0A2F8D3
:1079900033684EF2402093F8FB110A220023C2F212
:1079A000000014F013FA4EF24020C2F2000014F06E
:1079B000FBF945F648200921C0F2020018F08AF8C8
:1079C00033684EF2402093F8FC110A220023C2F2E1
:1079D000000014F0FBF94EF24020C2F2000014F057
:1079E000E3F945F654200621C0F2020018F072F8BF
:1079F00031680A2201F2FD1101A81DF04FF845F28D
:107A000068700121C0F2020018F064F801A81CF0AF
:107A1000D7FF014601A818F05DF845F21860012172
:107A2000C0F2020018F056F84EF24020C2F20000F8
:107A300014F0BAF99B244EF2402000230A2221467A
:107A4000C2F2000014F0C2F945F628200221C0F26B
:107A5000020018F03FF82B6823444EF2402093F8C0
:107A60006C110A220023C2F2000014F0AFF94EF2AA
:107A700040200134C2F2000014F096F9AD2CDAD1A6
:107A80004EF24020C2F2000014F08EF904B070BD36
:107A90002DE9F0412DED028B41F6606086B0C2F217
:107AA000010013F0D3FB41F66060C2F2010013F055
:107AB00049FA41F66060C2F2010013F03BFA41F668
:107AC0006060C2F2010013F0D3F841F66060C2F2C8
:107AD000010013F03FFA41F66060C2F2010013F0BA
:107AE00041FA41F66060C2F2010013F01BFA45F65C
:107AF0005C23C0F2020393E8070000244FF0203714
:107B00006B46029703940494CDF80B708DF81440E3
:107B100003C341F660601A8021462246C2F201008A
:107B200013F0DCF968461CF04BFF024641F660603A
:107B30006946C2F2010014F0C3F84EF24020234619
:107B40000A222146C2F2000014F040F945F2787092
:107B50000121C0F2020017F0BDFF4EF24020234683
:107B60000A222146C2F2000014F030F945F66820DE
:107B70000321C0F2020017F0ADFF68461CF020FFA1
:107B80000146684617F0A6FF45F218600121C0F2D1
:107B9000020017F09FFF45F66C264EF24020C0F21F
:107BA0000206C2F2000014F0FFF896E8030000900D
:107BB00041F66060019722468DF80410C2F2010080
:107BC0000B21029703940494CDF80B708DF81440A8
:107BD00013F084F968461CF0F3FE024641F660603B
:107BE0006946C2F2010014F06BF84EF240202346C1
:107BF0000A222146C2F2000014F0E8F845F278703B
:107C00000121C0F2020017F065FF4EF2402023462A
:107C10000A220B21C2F2000014F0D8F845F66820C1
:107C20000321C0F2020017F055FF68461CF0C8FEA1
:107C30000146684617F04EFF45F218600121C0F278
:107C4000020017F047FF4EF24020C2F2000014F08D
:107C5000ABF845F67423C0F202030FCB8DE80F009A
:107C600041F6606021460122C2F2010004948DF8C1
:107C7000144013F033F968461CF0A2FE024641F6A8
:107C800060606946C2F2010014F01AF84EF240201A
:107C900023460A220121C2F2000014F097F845F2AF
:107CA00078700121C0F2020017F014FF4EF240205C
:107CB0000A2223462146C2F2000014F087F845F656
:107CC00068200321C0F2020017F004FF68461CF090
:107CD00077FE0146684617F0FDFE45F21860012167
:107CE000C0F2020017F0F6FE4EF24020C2F2000091
:107CF00014F05AF80221042015F036F802211E2053
:107D000015F032F8DC2015F093F845F68820342180
:107D1000C0F2020017F0DEFE4EF24020C2F2000078
:107D200014F042F845F6C0202E21C0F2020017F0F0
:107D3000D1FE4EF24020C2F2000014F035F845F6B4
:107D4000F0202921C0F2020017F0C4FE4EF24020BC
:107D5000C2F2000014F028F845F61C300921C0F2E8
:107D6000020017F0B7FE0521304617F0B3FE4EF2C1
:107D70004020C2F2000014F017F845F628300D211B
:107D8000C0F2020017F0A6FE4EF24020C2F2000040
:107D900014F00AF8FFF758F8FCF750FD4EF288137C
:107DA000CEF20003012740F2002040F29855C2F2C3
:107DB00001051F604FF4E171C1F6FF7013F058FA2E
:107DC00028460BF071FA28460AF0BEFDEA88242105
:107DD00022F0100228460AF083FBEA88242122F4CC
:107DE000807228460AF07CFB28460AF02DFDF6EE4C
:107DF000000AB0EE600A28460BF050F84CF6CD466B
:107E00001D2128460AF090FEC3F64C5628460BF07A
:107E1000A3F801EE106A4DF20A76C3F6234600EE8F
:107E2000906A46F26666C3F666763B4600EE106AD6
:107E30003A46394628460BF0D7F828460AF000FCA7
:107E400028460AF07FFC0222072128460AF0F2FDAC
:107E500028460AF073FB4CF6CD43C3F64C6302226E
:107E600000EE903AB7EE000A394628460AF0E0FEE6
:107E700045F638301B21C0F2020017F02BFE4EF2FF
:107E80004020C2F2000013F08FFF4DF6D860C2F21E
:107E900000000B210CF048FC4DF6D860C2F2000047
:107EA0000D210CF0A9FC49F21400C2F20100FE21E0
:107EB0000CF0E0FD002840F0A18045F65430172179
:107EC000C0F2020017F006FE4EF24020C2F200009F
:107ED00013F06AFF45F66C33C0F2020393E8030027
:107EE00041F6A44241F65463C2F20102C2F2010318
:107EF00082E8030083E803004DF6A866C2F200069C
:107F000041F6F044C2F20104002301EE903A2378D6
:107F100000EE103A0023C4F2964302EE103A00231A
:107F2000C4F2482301EE103AB8EE400AF0EE610ABE
:107F300001F09AFEB5EEC00AF1EE10FA00F13383BB
:107F400047F67903C4F2302307EE103AF6EE007AD2
:107F5000E0EE077A49F68073C0F20103FCEEE77A9F
:107F600017EE902A9A4240F221831A464FF450713C
:107F700040F22073C2F20103187EC50700F123818D
:107F8000DD8B1A62A94240F0010088BFD9831876C0
:107F9000237800EE103A002301EE903A41F2844437
:107FA0000023C4F20C23C2F2010401EE103AB8EE31
:107FB000400A4FF48033F0EE610AB7EE002AA36165
:107FC00001F052FE4FF47E43C4F2FF6307EE903A95
:107FD000B4EEE70AF1EE10FA00F3BB804FF47E43F3
:107FE000CCF2FF6307EE903AB4EEE70AF1EE10FA36
:107FF00040F1D2820023C8F20103ADE045F67430AF
:108000000E21C0F2020017F065FD4EF24020C2F2D0
:10801000000013F0C9FE4DF6A86641F25C53C2F2AF
:108020000103C2F200061F7008F0BEFA327941F671
:10803000CC4EC2F2010E02EB420340F2300802EBDA
:108040008302C2F2010841F6A4418EF80000C2F298
:10805000010108EB020008F035F9307908F050F919
:1080600045F684300621C0F2020017F033FD337963
:1080700003EB430503EB850308EB030528461CF0DF
:108080009FFC0146284617F025FD45F27870C0F2A6
:108090000200F8F787FC41F6A440C2F201001CF090
:1080A0008FFC014641F6A440C2F2010017F012FD18
:1080B00045F218603946C0F2020017F00BFD4EF28F
:1080C0004020C2F2000041F6F44513F06DFEC2F20A
:1080D00001052FE045F68C300321C0F2020017F0B5
:1080E000F9FC4EF2402000230A222146C2F2000091
:1080F00013F06CFE45F268700121C0F2020017F027
:10810000E9FC28461CF05CFC0146284617F0E2FC1E
:1081100045F218600121C0F2020017F0DBFC4EF2BC
:1081200040200134C2F2000013F03EFE202C05F185
:108130000B0509D0092CCDD845F63C100121C0F221
:10814000020017F0C7FCC5E77179307908F0C0FB71
:10815000D6E60023C7F6FF7341F67465C2F2010547
:10816000002201EE902A2A78E36100EE102A002214
:10817000C4F2482201EE102AB8EE400AF0EE610A7D
:10818000B7EE002A01F070FD4FF47E43F7EE007A5F
:10819000C4F2FF6337EEC00A07EE903AB4EEE70A86
:1081A000F1EE10FA19DC4FF47E43CCF2FF6307EED8
:1081B000903AB4EEE70AF1EE10FA40F1E6810023BE
:1081C000C8F201030CE01D6AAA4240F29481D88BE8
:1081D0001A62814288BFD983DAE60023C7F6FF73AB
:1081E0002A7800EE102A002201EE902A41F2BC44C7
:1081F0000022C4F24822C2F2010401EE102AB8EEB5
:10820000400AF0EE610AB7EE002AA36101F02CFDEE
:108210004FF47E43C4F2FF6307EE903AB4EEE70AF0
:10822000F1EE10FA0FDC4FF47E43CCF2FF6307EE61
:10823000903AB4EEE70AF1EE10FA40F155810023CE
:10824000C8F2010302E00023C7F6FF732A78E36156
:1082500000EE102A002201EE902A0022C4F24822E9
:1082600001EE102AB8EE400AF0EE610AB7EE002ADD
:1082700001F0FAFC4FF47E43C4F2FF6307EE903A3C
:10828000B4EEE70AF1EE10FA0FDC4FF47E43CCF2C5
:10829000FF6307EE903AB4EEE70AF1EE10FA40F110
:1082A0001C810023C8F2010302E00023C7F6FF731C
:1082B00041F6F14140F21C02C2F20101C2F2010298
:1082C00009781278236207EE901A07EE102A00222E
:1082D000C4F2C82208EE102AF8EE677AB8EE477AA0
:1082E000C7EE886A41F29053F268C2F201031B683C
:1082F000C7EE087AB7EE007A77EE666A77EE677AAD
:1083000000EE902AB268C3ED596A83ED5A7AC3ED44
:10831000587A00EE102AFDF7CFFC0023C4F22C237C
:1083200007EE903A002306EE903AB36807EE103A53
:1083300027EE087A27EE277AC7EE087A77EEA67A34
:10834000FDEEE77A17EE903A9B0072B641F2F444E4
:10835000C2F20104E36062B6237C012B40F22B8160
:1083600072B6E36862B640F22402002BC2F2010248
:10837000B8BF03339B101360737972B69B002362FE
:1083800062B694F82430012B40F21A8172B6236A47
:1083900062B640F22402002BB8BF0333C2F20102DE
:1083A00041F6D0409B10C2F20100536012F000FC75
:1083B00041F6E040C2F2010012F0FAFB4AF20E74FC
:1083C0004AF20C71C2F20104C2F201014AF20872CF
:1083D0004AF28C63C2F20102C2F2010345F6903008
:1083E00025880C8815801821C0F202001C8017F027
:1083F00071FB4EF2402000230A223179C2F20000C4
:1084000013F0E4FC45F278700121C0F2020017F08D
:1084100061FB4EF2402000230A227179C2F2000073
:1084200013F0D4FC45F218600121C0F2020017F0ED
:1084300051FB4EF24020C2F2000013F0B5FCFEF7F3
:10844000B9FF45F6AC301421C0F2020017F042FB30
:108450004EF240208021C2F2000013F047FC45F6A6
:10846000C4301121C0F2020017F034FB4EF240205C
:1084700040F65A31C2F2000013F038FC45F6D8300D
:108480000321C0F2020017F025FB4EF24020C2F299
:10849000000013F089FCFEF7AFFE41F66060C2F207
:1084A000010012F05FFD01F01FFE4EF20813CEF244
:1084B0000003012245F6DC301A600B21C0F20200F5
:1084C00017F008FB4EF24020C2F2000013F06CFCE3
:1084D00006B0BDEC028BBDE8F081F0EE407AFEEE16
:1084E000C87A17EE903AE3E6F0EE407AFEEEC87AEC
:1084F00017EE903AAAE602F17F01C909013100297D
:108500001A620A4638BF0022870706D5596A7F31AA
:10851000C90901318A4238BF0A46450706D5996A1A
:108520007F31C90901318A4238BF0A46010706D5A1
:10853000D96A7F31C90901318A4238BF0A46C70664
:1085400006D5196B7F31C90901318A4238BF0A4605
:10855000850606D5596B7F31C90901318A4238BF7A
:108560000A46410606D5996B7F31C90901318A4215
:1085700038BF0A46C10906D0D96B7F31C90901311C
:108580008A4238BF0A46DA8302E5F0EE407AFEEE10
:10859000C87A17EE903A23E6F0EE407AFEEEC87AFB
:1085A00017EE903AD8E501210022E1E402F17F01C3
:1085B000C9090131DCE472B62046FCF793FCD0E631
:1085C00072B641F20850C2F20100FCF78BFCDEE605
:1085D0002DE9F0479DF82040013CE4B20F2C03D870
:1085E0004EB2002E0D4601DBBDE8F087E0290FD921
:1085F000F729F9D90835EDB2012303FA05F515F08D
:10860000DD0FF1D0806C0368BDE8F0471B681847A8
:108610008146806C1F46036846EA0401C9B21B68A4
:1086200090469847D9F84800036808F07F011B6816
:1086300005F0EF059847C02DD6D0D9F8480003685B
:1086400007F07F011B68BDE8F0471847F8B50446FE
:10865000806C03681B69984708B90020F8BDA06CBE
:1086600003685B699847C3B203F0FB01F929F4D0B2
:10867000A26D82B994F84D2084F84F30150600F1B0
:108680009C8040B20028C0F25081002084F84D0048
:10869000A0656065F8BD010667D494F84F10F02915
:1086A00004EB020140D081F84F30616D4B1E9A42BD
:1086B00040D394F84F20F02AE7D013063DD400238E
:1086C00084F86630B02B4CD0A02B4AD0D02B48D0A9
:1086D000E02B46D0C02B44D0002094F8505084F8B2
:1086E0006750032908BF94F8515084F8650018BFFB
:1086F000002500210120B02B84F86850A165616538
:1087000084F8E90000F0B58000F2AC80902B00F016
:10871000B080A02B00F0AD80802B00F0AA80002359
:1087200084F84D300120F8BD81F86930636D013B5C
:108730009A42AAD20132A2658FE702F10C03DBB2A2
:10874000012BBCD902F0FB03F92BB8D0EF2A00F2C1
:10875000DB8002F0F003802B84F8663001D0902B90
:10876000B0D102F00F000130B7E7A3F1F7010829FB
:1087700093D8012505FA01F010F4DD7F40F09680D2
:1087800000298AD194F86930F02B7FF47EAF561C13
:108790002244F720370A82F8690084F8676084F879
:1087A000687084F8651084F84D10284684F86630A7
:1087B00084F8E950A1656165F8BD02F10C05EEB2DF
:1087C000012E7FF65EAF02F0FB0EBEF1F90F3FF413
:1087D00058AFEF2A2DD802F0F007802F2AD140B2EF
:1087E0000028FFF64FAF012184F84F2084F8503065
:1087F000A165EDB2012D7FF648AFBEF1F90F3FF450
:1088000044AFEF2A5FD802F0F003B02B26D01ED978
:10881000D02B04D0E02B21D0C02B7FF436AF022325
:1088200063650121A36D994227D90133A365002017
:10883000F8BD174607F0DF06902ED0D007F0BF0630
:10884000A02ECCD007F0EF07C02FC8D019E7902B8F
:1088500004D0A02B02D0802B7FF417AF03236365D5
:108860000221DFE7D02B04D0E02B02D0C02B7FF415
:1088700056AF84F84D200120F8BDEF2A94BF02F0D6
:10888000F005154602F00F020023013294F8501053
:1088900084F86520012084F8671084F8683084F833
:1088A0006650A365636584F8E900F8BD002284F88A
:1088B000672084F8682084F8652084F8663084F89E
:1088C000E9502846F8BDF62A0FD007D8F12AA6D0DD
:1088D0001CD9F22AC2D0F32AA1D0D6E6FC2A21D88C
:1088E000FA2A02D2F82A7FF4D0AE0023012084F8BD
:1088F000653084F8673084F8683084F86620A365B2
:10890000636584F8E900F8BD1346D9E6F02A7FF4E0
:10891000BCAE80210023616584F8692084F84D3065
:108920007F217FE7FE2AE0D2AFE61A468E4603F1AA
:108930000C055EE790F86630F12B7CD00ED9FA2B4F
:108940002BD01FD8F32B38D0C0F08180F62B7AD0F3
:10895000F82B40F08B80036BF3B11847B02B6ED02F
:1089600031D9D02B21D03ED9E02B42D0F02B7ED173
:10897000C3698BB1B0F86710802900F1690028BF86
:1089800080211847FC2B0CD051D3FE2B4BD0FF2B52
:108990006BD1436C002BE0D17047436B002BDCD1D3
:1089A000FAE7C36B002BD8D1F6E74369002BF3D06D
:1089B00090F8671090F865001847836A002BEBD099
:1089C00090F867001847902B29D0A02B23D0802B3C
:1089D000E2D10368002BDFD090F8682090F8671090
:1089E00090F865001847C02B42D10369002BDFD1F6
:1089F000D2E78269002ACFD090F8681090F86730EB
:108A000090F86500C90101F47E5103F07F0319431A
:108A1000A1F5005110478368002BDDD1BCE7436806
:108A2000002BD9D1B8E7036C002B96D1B4E7836B48
:108A3000002B92D1B0E7036A002BC1D1ACE7C36829
:108A4000002BC9D1A8E7C36A002B86D1A4E7426AEC
:108A5000002AA1D090F8683090F86700DB0103F499
:108A60007E5300F07F0018431047704770477047EF
:108A7000704700BF90F86430DA0725D513F0FE0F79
:108A800022D070B590F8665085F08002602A82B0DE
:108A900004461AD9F62D6ED067D8F12D7ED04FD965
:108AA000F22D2DD0F32D1AD1806C94F867600368F5
:108AB00029461B689847A06C0368DB6C06F07F01B1
:108AC00002B0BDE870401847704790F865608E426C
:108AD00007D031B15B08012B08D0032B27D002B09F
:108AE00070BD5B08012B01D0022BF8D194F86830DF
:108AF00094F86720009629462046FFF769FDEEE7C7
:108B0000806C94F86730026894F8686012682946AF
:108B100043EAC6159047A06C036805F07F019B6C83
:108B20009847A06C0368C5F3C6119B6CC8E794F81E
:108B3000683094F8672000962946FFF749FDCEE794
:108B4000F02DCCD1B0F86760802E28BF802600F1D0
:108B50006905002EC3D02E44A06C15F8011B0368D4
:108B60001B689847AE42F7D1B9E7FC2D26D8FA2DFD
:108B700001D2F82DB3D105F10803DBB2072BAED833
:108B8000012202FA03F313F0DD0FA8D0A06C0368F2
:108B90001B68294602B0BDE870401847806C94F805
:108BA000672094F8683006681201294603F00F0325
:108BB00002F0700532681D439047E7E7FE2D8ED323
:108BC000D9E700BFF0B540F2D05087B0C2F2010043
:108BD0000BF078FC002840F0FE804AF23474C2F2B8
:108BE000010441F6706223680193C2F20102019B05
:108BF000116841F287325B1A934206D941F6CD43A0
:108C0000C2F201031B78002B43D041F67865C2F213
:108C1000010595F84C60102E4CD9002016F072FB1F
:108C200010F0EEFD41F2C0500021C2F2010011F03F
:108C3000D9FC41F2585322680292C2F20103029A0F
:108C40001868121A4AF23471322AC2F201014ED85F
:108C500041F28C5322680492C2F20103049A19680B
:108C6000521A632A00F2B28040F2B0632268059281
:108C7000C2F20103059A196841F28730521A824202
:108C800005D901F59C5108311960FEF7B5FA07B016
:108C9000F0BD40F2CC53C2F201031B78002BB4D0DC
:108CA00041F67865C2F20105FDF7FCFC95F84C60D1
:108CB000102EB2D82846FFF7C9FC0028ADD095F891
:108CC0006630902B00F00B8183F08003602B40F224
:108CD000098141F67860C2F20100FFF72BFE41F6F0
:108CE00078603146C2F20100FFF7C4FE95E741F219
:108CF00090560A680392C2F2010641F26055039A47
:108D000030681A60C2F2010506F0A2FE41F6CD43BA
:108D1000C2F20103AA881870002A40F03D8140F297
:108D20004455C2F20105AB88002B40F0ED8040F2C3
:108D3000F065C2F20105AB88002B89D03268D2F809
:108D4000601107EE901A296807EE101A77EE877AFD
:108D500045F66040C2ED587A013BC0F20200AB809C
:108D6000F7F720FE3368D3F860011AF00FFE41ECEC
:108D7000100B4EF240200521C2F2000013F066F8FD
:108D800045F67040C0F20200F7F70CFE4EF24020AC
:108D9000A988C2F2000012F0A9FF45F68840C0F28F
:108DA0000200F7F7FFFD28681AF0F0FD41EC100B08
:108DB0004EF240200521C2F2000013F047F84EF2B7
:108DC0004020C2F2000012F0EFFF41E76431196069
:108DD00003F0EAFA48E740F2A454C2F2010413F0A7
:108DE000FFFF2368C01AB0F5356F7FF6F6AE13F0BB
:108DF000F7FF206040F2D050C2F201000BF072FB8E
:108E0000044613F0EDFF41F29053C2F20103054610
:108E100022461868802106F00FF813F0E1FF40F6B3
:108E20005A33401B984252D840F22C0413F0D8FF1A
:108E3000C2F20104401B2388834260D372B640F221
:108E4000A853C2F201031A7F02F0FF010AB1002207
:108E50001A7762B6A1B372B647F6FF744FF40040BA
:108E6000B3F91E50B3F92020DC83188462B685EA7A
:108E7000E57182EAE273A3EBE273A1EBE5718B4249
:108E8000B8BF0B4607EE903A4FF47E43C4F2FF633F
:108E900006EE103AF8EEE77A47F2A403C7EE866AC8
:108EA000C3F67D7307EE103AF4EEC76AF1EE10FADE
:108EB00006DD41F6A043C2F201031A6801321A60CE
:108EC00040F2D050C2F201000BF01EFB85E641F2E9
:108ED0003053C2F201031A6801321A60A4E795F810
:108EE000683043B195F865309E423FF4F2AE002EF3
:108EF0003FF4EFAEF3E6802385F86630F2E713F037
:108F00006FFF401B208099E73268D2F8641107EEAA
:108F1000901A296807EE101A77EE877A45F6144002
:108F2000C2ED597A013BC0F20200AB80F7F73AFD7F
:108F30003368D3F864011AF029FD41EC100B4EF2AE
:108F400040200521C2F2000012F080FF45F62840C3
:108F5000C0F20200F7F726FD4EF24020A988C2F2C7
:108F6000000012F0C3FE45F64440C0F20200F7F7DD
:108F700019FD28681AF00AFD41EC100B4EF2402052
:108F80000521C2F2000012F061FF4EF24020C2F251
:108F9000000012F009FFCAE64DF6A867C2F200070A
:108FA000013AFB68AA8000EE903ABB6807EE903A5F
:108FB0002B6807EE103A37EE870AFCF77DFE45F680
:108FC000E830C0F20200F7F7EDFCB8681AF0DEFCFA
:108FD00041EC100B4EF240200521C2F2000012F0CD
:108FE00035FF45F6F430C0F20200F7F7DBFC4EF235
:108FF0004020A988C2F2000012F078FE45F6044035
:10900000C0F20200F7F7CEFC28681AF0BFFC41EC72
:10901000100B4EF240200521C2F2000012F016FFA4
:109020004EF24020C2F2000012F0BEFE77E600BF12
:109030002DE9F04F41F67865C2F201058DB013F0CD
:10904000B5F895F86430002401264EF2600743F02D
:1090500001034FF6FF7E66F34703214685F865401E
:1090600085F8664085F8674085F8684085F8E940EE
:10907000C2F2000705F169008022C5F85CE0C5F87E
:1090800060E085F86430AF6485F84C4085F84D4069
:1090900085F84E406C65AC651BF062FB4DF6A02276
:1090A00040F695112846C2F20002C0F2000141F2DA
:1090B000C057C2F201072C606C60AC60EC602C61A0
:1090C0006C61AC61EC612C626C62AC62EC622C6332
:1090D0006C63AC63EC632C646C641AF0F3FF46F2CF
:1090E000C872C0F2020207F59B6307F5B36107F58A
:1090F000A36007F5AB653A607B61402250237C603A
:10910000BC60B861FD61384679627A85BB8511F033
:109110002DF941F6606845F29C03C2F20108C0F2E5
:1091200002033B60102202232721404611F090FDEC
:1091300041F2F44045F2B803C0F2020302220321D7
:10914000C2F20100C8F80030FCF736FB41F20850CB
:109150001D221C21C2F20100FCF72EFB4AF23473DF
:1091600041F6D040C2F2010314220421C2F20100F0
:109170001D46029311F004FD41F6E04014221E2129
:10918000C2F2010011F0FCFC2B68069341F28C53F3
:10919000C2F2010340F2D059C2F20109069A1A60E4
:1091A0002146224640F2A85B4846FBF71BFBC2F271
:1091B000010B46F25863C0F202030BF1180231466C
:1091C000584689F89C40C9F8984089F89D40C9F8EC
:1091D000003040F22075FBF705FB4FF40041C2F26E
:1091E000010547F6FF7246F20063ABF8201045F226
:1091F0009001C0F20203ABF81E20C0F2020105F597
:109200005462CBF800302C722346EC6020466E721C
:109210002A6129602C4600E0226942F82300697A1D
:10922000013340F220729942C2F20102F4DC4AF2A8
:109230008863C2F201030393196809B9A8E21946C9
:109240004B69002BFBD14D614FF00004002141F22E
:10925000844846F2286340F26070C2F20108C0F20E
:10926000020369614FF45062AC80EC80AC722C76E2
:10927000C2F201004FF000042B606C83AC83EC83DE
:109280001BF06EFA08F1280204214046FBF7AAFA07
:109290004FF4803341F2644441F2BC47C2F201070B
:1092A000C8F81830C8F81C30C8F82030C8F8243086
:1092B000059341F23456234646F2406AC2F2010653
:1092C000C2F20103C0F2020A07F128020421384663
:1092D0001C46C8F800A00493FBF784FA059B01968E
:1092E00006F11C0230460121C7F800A0BB61FB61FA
:1092F0003B627B62FBF776FA019B46F2346A9E463C
:109300002246059BCEF81830C0F2020A1C32012119
:10931000204640F24C56CEF800A0FBF763FA059BBE
:10932000A361C2F2010645F29003C0F2020306F106
:1093300018010022022033604FF000033372707274
:1093400031610B46C4F800A0F2601146304600E0DF
:10935000036943F82210747A013240F24C5394426C
:10936000C2F20103F4DC039A12684AF28861C2F285
:1093700001010AB90EE21A465369002BFBD156616E
:10938000002440F24C5040F2746A46F68C23C0F23E
:109390000203C2F2010A7461B480F480B472C2F2B2
:1093A0000100336014F024FC50468AE8000A8AF871
:1093B00008408AF80940CAF80C408AF8104040F288
:1093C000886B12F0B3F84DF6A02240F69911C2F264
:1093D000010BC2F20002C0F2000150461AF072FE08
:1093E0005846CBF80090CBF804808BF808408BF8F7
:1093F0000940CBF80C408BF8104040F29C6A12F008
:1094000095F84DF6A02240F69911C2F2010AC2F277
:109410000002C0F2000158461AF054FE5046CAF845
:1094200000908AF808408AF80940CAF80C408AF887
:109430001040CAF8047041F21C5912F077F84DF64A
:10944000A02240F69911C2F20109C2F20002C0F254
:10945000000150461AF036FE4FF0010B484689E8ED
:10946000200189F80840C9F80C4089F8104089F8B3
:1094700009B040F2B46A12F059F84DF6A02240F655
:109480009911C2F2010AC2F20002C0F2000148467C
:109490001AF018FE022350468AF8093005938AE82C
:1094A000A0008AF80840CAF80C408AF8104040F240
:1094B000C86912F03BF84DF6A02240F69911C2F2AD
:1094C0000109C2F20002C0F2000150461AF0FAFD92
:1094D0004846C9F80080C9F8045089F8084089F85E
:1094E0000940C9F80C4089F8104040F2DC6512F0E0
:1094F0001DF84DF6A02240F69911C2F20105C2F204
:109500000002C0F2000148461AF0DCFD2846C5F80A
:1095100000802C72EC602C746F6085F809B041F209
:10952000945812F003F84DF6A02240F69911C2F2B9
:109530000108C2F20002C0F2000128461AF0C2FD82
:10954000019BC8F80430404688F8084088F8094074
:10955000C8F80C4088F81040C8F8007040F2F86570
:1095600011F0E4FF4DF6A02240F69911C2F2010578
:10957000C2F20002C0F2000140461AF0A3FD049BB3
:109580006B6028462C726C72EC602C742F6040F279
:109590000C7811F0CBFF4DF6A02240F69911C2F2E3
:1095A0000108C2F20002C0F2000128461AF08AFD4A
:1095B0004046C8F8046088F8084088F80940C8F8B0
:1095C0000C4088F81040C8F8007040F2705511F057
:1095D000ADFF4DF6A02240F69911C2F20105C2F28C
:1095E0000002C0F2000140461AF06CFD28466E6091
:1095F0002C72EC602C7485F809B02F6041F268562B
:1096000011F094FF4DF6A02240F69911C2F2010626
:10961000C2F20002C0F2000128461AF053FD059B79
:10962000737245F2900306F11801C0F2020322465C
:1096300033603472F460204631610B46344600E0FA
:10964000236943F82200717A013241F26853914252
:10965000C2F20103F4DC039A12684AF28861C2F292
:1096600001010AB998E01A465369002BFBD15661F3
:10967000002441F2685046F24C63C0F20203746168
:10968000B480F480B472C2F2010040F28457C2F296
:10969000010733600AF096FD019B3C72384687E86B
:1096A00048007C72FC603C7411F040FF4DF6A02233
:1096B00040F69911C0F200013846C2F2000241F6AC
:1096C000B8451AF0FFFCC2F20105049A2C7201237E
:1096D000284685E844006B72EC602C7411F026FF7C
:1096E0004DF6A02240F69911C0F200012846C2F2C0
:1096F00000021AF0E7FC40F29853C2F2010346F26E
:109700000C62C0F202021A604FF419700A221A7237
:1097100013F07EF84AF64441064605F00FF9029F21
:109720003B680793079D3B680893089C3B68099337
:1097300041F29050C2F2010041F6706140F2706255
:1097400041F6B443C2F20101C2F20102C2F20103C6
:10975000066009980D601460186013F041FB029FC9
:109760003B680A930A9D3B680B9340F2A45141F277
:10977000585240F2B063C2F20101C2F20102C2F2D9
:1097800001030B9C086015601C600DB0BDE8F08FF4
:109790001A6059E50B60F3E50B6069E74FF07E5204
:1097A0000021416702678267704700BF70B507EE0E
:1097B000901A2DED048BB8EEE79AB7EE008A88EE8A
:1097C000097A4FF46043C4F22B7300250026044647
:1097D000866305638561C561C56085604560056018
:1097E00007EE903A80ED057A87EE897A0562456347
:1097F00080ED049A17EE100A1AF0C8F841EC100B2D
:1098000017F09EFB51EC100B1AF00CFC49F6AB0361
:10981000C3F6B44308EE900A07EE903A68EEA77AD2
:1098200040F6DB7388EE277AC4F2490306EE903ADD
:109830002369C4ED097A05EE903AB6EE006ABAEEF5
:10984000040AA5EE860A636907EE903A20EE260A1E
:1098500084ED0A7A20EE270A17F020F94BF60B4325
:10986000C3F6324307EE103A0023C4F2FC2307EE9E
:10987000903A68EE878A87EE897A0123236600236F
:10988000CBF6807384F854606566A566E364A364D0
:10989000C8EE287A38EE478AC4ED168A84ED1B8A12
:1098A000BDEC048B84ED0B0AC4ED177A70BD00BFCC
:1098B000F8B50B6806EE903A436E07EE903AC36E29
:1098C00007EE103A836E76EEE77A06EE103AE7EE90
:1098D000067A02F18047012A2DED108B07F1FF3740
:1098E000C1ED007AC0ED196A19DD01EB87040B4662
:1098F0005D6807EE905A37EEE67A06EE905AC56E2E
:1099000006EE105A1D6805EE905AA6EE257A17EE5F
:10991000105A43F8045FA342C0ED197AE8D1846F6E
:10992000BF0007EE904ACB19B7EE007AF4EE477A03
:109930001B688366F1EE10FA11D0002A0FDD3C1D82
:109940000C440B4602E0856F07EE905A1D6807EE47
:10995000105A67EE277AE3EC017AA342F3D1036F42
:1099600007EE903AB7EE007AF4EE477AF1EE10FA8D
:1099700000F0FB80C36C07EE103A436FF4EE477AB9
:10998000F1EE10FA16460D46044600EE103A40F08D
:10999000EF80836C07EE903AB4EE670AF1EE10FAAE
:1099A00040F0E680C36B0CEE903AF7EE00BA3CEE66
:1099B000ABDA002E8CEE8DBA40F3D78040F6DB7325
:1099C000C4F249030437A66B2F440AEE103A2BEE7B
:1099D0000B8A46F26663C3F6E6630DEE903A28EE14
:1099E0000B8A4CF67743C3F22B2309EE903A8BEEA9
:1099F0008D9AF2EE0E8A28EE0B8A10E0022E00F00D
:109A00002981032E40F02281F0EE6B7AECEE2D7A64
:109A100067EEAA7AE5EC017AAF4200F0A6802B68E7
:109A200007EE903AE36905EE903AA36906EE103A24
:109A3000E36A04EE103A23680AEE903A63680EEE89
:109A4000103AA3680FEE103AE3680EEE903A236ADC
:109A50000CEE103A636907EE103A27EE287A37EEDB
:109A6000E55A27EE0A7AF0EE4E3A25EE075A37EE1F
:109A70002B7AEBEE2A3A636AC5EE076AB0EE4F7AAC
:109A800075EEA65AABEE237AE5EEED7A74EE2B4A2C
:109A900077EEC67AB0EE6E5A67EE847AABEE075A6E
:109AA00087EEA47A29EE455A36EE076AF0EE6B3A55
:109AB000F0EE467AE5EE0C7AECEE083A76EEA55A30
:109AC000C7EEA36A37EE066A76EEA96A07EE903A09
:109AD00076EEEA6AC4ED075AEBEE26AA84ED066A32
:109AE000B0EE6A0AABEE260A20EE270A16F060FEF8
:109AF0007AEECE7AA36A67EEAC7A07EE103A27EEDA
:109B0000000A87EE8D7A012E84ED000A77EE0E7A38
:109B100037EECF6A37EE277A26EE2C6A84ED017A8B
:109B2000C6EE0D6A36EE8F7A77EE6E5A76EE876A5B
:109B300065EEAC5AC4ED026A85EE8D6A76EE2E6A49
:109B400036EE266A84ED036A74D03FF757AF002ED5
:109B50007CD1636B06EE103A66EE077A3BEEC66A7E
:109B6000E6EE267AF0EE67AA4EE7BDEC108BF8BD64
:109B70004BF61423B7EE008AC4F23F0309EE103A05
:109B800038EE400AF3EE038A20EE090A17F038FA9D
:109B900030EE480A4BF22D2380EE286AC3F67D731F
:109BA00007EE103A002307EE903AE6EE077A236FAD
:109BB000F0EE0C6A77EE677A06EE103A27EEA67A98
:109BC00026EE090AC4ED107A84ED087A17F018FA27
:109BD00030EE480A4FF4784380EE286AC4F293636B
:109BE00006EE903A0023C4F2702307EE903A40F656
:109BF000DB73C4F24903E6EE267A07EE103A636996
:109C000006EE903A27EEA60A20EE070A16F046FF67
:109C1000216C226F636F84ED0F0A07EE901A38EE05
:109C2000678AF0EE40CABDEEC88AE264A36484EDA0
:109C3000188ABAE6636B06EE903A66EEA77A7BEE78
:109C4000E66AE6EE877AF0EE67AADDE600230AEE22
:109C5000903AD9E6636B06EE903A6AEEA6AA7BEEDE
:109C6000E66AE6EEA7AACFE630EE600A32EE612A97
:109C700031EE601A20EE022A82EE010A30EE210A4D
:109C8000704700BF00B583B012F090FA4AF2347208
:109C9000C2F2010241F6647312680192C2F201033A
:109CA000019A1A6003B05DF804FB00BF2DE9F04390
:109CB0004DF6A868C2F200082DED028BD8ED027AAD
:109CC0009FED748A9FED746AF6EE008AF0EE686A82
:109CD000E7EE886A4AF23473C2F20103B2EE0E7AFA
:109CE00026EE877A40F21D07C7EE087A91B0C2F2DD
:109CF00001071B6803933A78039941F66473C2F233
:109D00000103012A196077EE867AFCEEE77ACDED41
:109D1000017A9DF8046000F0E08141F66060C2F2D3
:109D2000010011F01FF945F6A043C0F2020393E8C9
:109D300003000AAC00254FF020336360A360E560A8
:109D40002561A38125750A9041F660602A46ADF829
:109D50002C10C2F20100294611F0C0F820461AF07A
:109D60002FFE024641F660602146C2F2010011F06A
:109D7000A7FF4EF240202B460A222946C2F20000DD
:109D800012F024F845F278700121C0F2020015F0BB
:109D9000A1FE4EF240202B460A222946C2F20000C4
:109DA00012F014F845F668200321C0F2020015F005
:109DB00091FE20461AF004FE0146204615F08AFE68
:109DC00045F218600121C0F2020015F083FE4EF248
:109DD0004020C2F2000011F0E7FF41F660602A2344
:109DE00001223146C2F201000A956560A560E56076
:109DF000256125758DF8283011F070F820461AF08D
:109E0000DFFD024641F660602146C2F2010011F01A
:109E100057FF4EF240202B460A220121C2F20000D9
:109E200011F0D4FF45F278700121C0F2020015F064
:109E300051FE4EF240202B460A223146C2F200006B
:109E400011F0C4FF45F668200321C0F2020015F0AE
:109E500041FE20461AF0B4FD0146204615F03AFEB8
:109E600045F218600121C0F2020015F033FE4EF2F7
:109E70004020C2F2000011F097FFD8ED027AF0EE18
:109E8000686A41F66878E7EE886AC2F2010888F8E5
:109E9000006003E00000C84200000000FDEEE67A2A
:109EA0000A2217EE900A04A91AF05EF905461AF084
:109EB00087FDC0B20328024628BF0322C2F1030077
:109EC00043F23003C0F230032946204400250A95AE
:109ED0006560A560E56025612575ADF82830A37043
:109EE0001AF0DCFD41F660602A460D21C2F2010045
:109EF00010F0F4FF20461AF063FD024641F6606060
:109F00002146C2F2010011F0DBFE4EF240202B464A
:109F10000A222946C2F2000011F058FF45F278707B
:109F20000121C0F2020015F0D5FD4EF240202B4673
:109F30000A220D21C2F2000011F048FF45F6682008
:109F40000321C0F2020015F0C5FD20461AF038FDCD
:109F50000146204615F0BEFD45F218600121C0F211
:109F6000020015F0B7FD4EF24020C2F2000011F0E1
:109F70001BFF98F8003041F66878B342C2F201083E
:109F800000F0A48041F660602A2301223146C2F22B
:109F900001000A956560A560E560256125758DF86D
:109FA000283010F09BFF20461AF00AFD024641F6C9
:109FB00060602146C2F2010011F082FE4EF24020A4
:109FC0002B460A220121C2F2000011F0FFFE45F2E9
:109FD00078700121C0F2020015F07CFD4EF24020A5
:109FE0002B460A223146C2F2000011F0EFFE45F680
:109FF00068200321C0F2020015F06CFD20461AF023
:10A00000DFFC0146204615F065FD45F21860012190
:10A01000C0F2020015F05EFD4EF24020C2F20000D8
:10A0200011F0C2FE98F800900A9541F66060202376
:10A0300049460122C2F201006560A560E560256124
:10A0400025758DF8283010F049FF20461AF0B8FC2D
:10A05000024641F660602146C2F2010011F030FE76
:10A060004EF240202B460A220121C2F2000011F0DC
:10A07000ADFE45F278700121C0F2020015F02AFD14
:10A080004EF240202B460A224946C2F2000011F04F
:10A090009DFE45F668200321C0F2020015F01AFD6E
:10A0A00020461AF08DFC0146204615F013FD45F2BE
:10A0B00018600121C0F2020015F00CFD4EF24020A4
:10A0C000C2F2000011F070FE88F8006001233B70BE
:10A0D00011B0BDEC028BBDE8F08341F66878C2F2A6
:10A0E00001080AACDAE600BF2DE9F04340F21D0793
:10A0F000C2F201078DB03B78002B40F094854DF6FD
:10A10000A866C2F2000669460A2230791AF02CF8D5
:10A1100004461AF055FCC0B20228024628BF0222AB
:10A12000C2F1020006AB21461844002443F230037A
:10A1300006940794ADF81830089409940A948DF8A1
:10A140002C401AF0ABFC41F6606022462146C2F278
:10A15000010010F0C3FE06A81AF032FC024641F6D8
:10A16000606006A9C2F2010011F0AAFD4EF2402083
:10A1700023460A222146C2F2000011F027FE45F2D2
:10A1800078700121C0F2020015F0A4FC4EF24020CC
:10A1900023460A222146C2F2000011F017FE45F6BE
:10A1A00068200321C0F2020015F094FC06A81AF002
:10A1B00007FC014606A815F08DFC45F21860012148
:10A1C000C0F2020015F086FC4EF24020C2F2000000
:10A1D00011F0EAFD41F6606022460221C2F2010060
:10A1E0004FF0200906940794089409940A948DF876
:10A1F0002C408DF8189010F071FE06A81AF0E0FBC4
:10A20000024641F6606006A9C2F2010011F058FD55
:10A210004EF2402023460A222146C2F2000011F0ED
:10A22000D5FD45F278700121C0F2020015F052FC14
:10A230004EF2402023460A220221C2F2000011F011
:10A24000C5FD45F668200321C0F2020015F042FC6E
:10A2500006A81AF0B5FB014606A815F03BFC45F22E
:10A2600018600121C0F2020015F034FC4EF24020CB
:10A27000C2F2000011F098FD337940F2300003EB98
:10A2800043024DF6A66803EB8203C2F2010041F6D9
:10A29000A441C2F200081844C2F2010106F012F80B
:10A2A00098F8005041F6606015F0FD05C2F201001B
:10A2B00000F0D08222460221069407940894099463
:10A2C0000A948DF82C408DF8189010F007FE06A81F
:10A2D0001AF076FB024641F6606006A9C2F2010060
:10A2E00011F0EEFC4EF2402023460A222146C2F233
:10A2F000000011F06BFD45F278700121C0F2020000
:10A3000015F0E8FB4EF2402023460A220221C2F259
:10A31000000011F05BFD45F668200321C0F2020049
:10A3200015F0D8FB06A81AF04BFB014606A815F05D
:10A33000D1FB45F218600121C0F2020015F0CAFB02
:10A340004EF24020C2F2000011F02EFD41F6A44072
:10A35000C2F201001AF034FBC2B2082A41F6A4414D
:10A3600028BF08224FF02033C2F2010106A806934D
:10A3700007940894CDF81B3009940A948DF82C406A
:10A380001AF08CFB41F6606022460321C2F2010004
:10A3900010F0A4FD06A81AF013FB024641F6606017
:10A3A00006A9C2F2010011F08BFC4EF240202346B8
:10A3B0000A222146C2F2000011F008FD45F2787031
:10A3C0000121C0F2020015F085FB4EF24020234629
:10A3D0000A220321C2F2000011F0F8FC45F66820C1
:10A3E0000321C0F2020015F075FB06A81AF0E8FA86
:10A3F000014606A815F06EFB45F218600121C0F277
:10A40000020015F067FB4EF24020C2F2000011F08E
:10A41000CBFC41F6606022460B21C2F2010006949B
:10A420000794089409940A948DF82C408DF818909C
:10A4300010F054FD06A81AF0C3FA024641F6606017
:10A4400006A9C2F2010011F03BFC4EF24020234667
:10A450000A222146C2F2000011F0B8FC45F27870E1
:10A46000C0F20200012115F035FB23464EF24020D8
:10A470000A220B21C2F2000011F0A8FC45F6682068
:10A480000321C0F2020015F025FB06A81AF098FA85
:10A49000014606A815F01EFB45F218600121C0F226
:10A4A000020015F017FB4EF24020C2F2000011F03E
:10A4B0007BFC707969460A22013019F055FE04468A
:10A4C0001AF07EFAC0B20228024628BF0222C2F168
:10A4D000020006AB21461844002443F230030694E0
:10A4E0000794ADF81830089409940A948DF82C401C
:10A4F0001AF0D4FA41F6606021460122C2F201004E
:10A5000010F0ECFC06A81AF05BFA024641F6606017
:10A5100006A9C2F2010011F0D3FB4EF240202346FF
:10A520000A220121C2F2000011F050FC45F27870BD
:10A530000121C0F2020015F0CDFA4EF24020234670
:10A540000A222146C2F2000011F040FC45F66820C4
:10A550000321C0F2020015F0BDFA06A81AF030FA85
:10A56000014606A815F0B6FA45F218600121C0F2BE
:10A57000020015F0AFFA4EF24020C2F2000011F0D6
:10A5800013FC41F6606001220221C2F20100202585
:10A5900006940794089409940A948DF82C408DF839
:10A5A000185010F09BFC06A81AF00AFA024641F671
:10A5B000606006A9C2F2010011F082FB4EF2402059
:10A5C00023460A220121C2F2000011F0FFFB45F2EE
:10A5D00078700121C0F2020015F07CFA4EF24020A2
:10A5E00023460A220221C2F2000011F0EFFB45F6D9
:10A5F00068200321C0F2020015F06CFA06A81AF0D8
:10A60000DFF9014606A815F065FA45F21860012148
:10A61000C0F2020015F05EFA4EF24020C2F20000D5
:10A6200011F0C2FB98F8008008F0FD084DF6A8660E
:10A6300041F66060B8F1010FC2F20006C2F20100FB
:10A6400000F0E781012202210694079408940994FE
:10A650000A948DF82C408DF8185010F03FFC06A895
:10A660001AF0AEF9024641F6606006A9C2F2010096
:10A6700011F026FB4EF2402023460A220121C2F2AD
:10A68000000011F0A3FB45F278700121C0F2020036
:10A6900015F020FA4EF2402023460A220221C2F28F
:10A6A000000011F093FB45F668200321C0F2020080
:10A6B00015F010FA06A81AF083F9014606A815F05D
:10A6C00009FA45F218600121C0F2020015F002FA01
:10A6D0004EF24020C2F2000011F066FB727941F6A2
:10A6E000F44302EB820602EB4606C2F201031E446B
:10A6F00030461AF065F9C2B20A2A28BF0A224FF082
:10A700002033314606A806930793089409940A94C7
:10A710008DF82C408DF820501AF0C0F941F6606099
:10A7200001220321C2F2010010F0D8FB06A81AF0A2
:10A7300047F9024641F6606006A9C2F2010011F035
:10A74000BFFA4EF2402023460A220121C2F2000045
:10A7500011F03CFB45F278700121C0F2020015F0C7
:10A76000B9F94EF2402023460A220321C2F200002A
:10A7700011F02CFB45F668200321C0F2020015F011
:10A78000A9F906A81AF01CF9014606A815F0A2F9C5
:10A7900045F218600121C0F2020015F09BF94EF25B
:10A7A0004020C2F2000011F0FFFA41F66060012281
:10A7B0000E21C2F2010006940794089409940A94A9
:10A7C0008DF82C408DF8185010F088FB06A81AF070
:10A7D000F7F8024641F6606006A9C2F2010011F0E6
:10A7E0006FFA4EF2402023460A220121C2F20000F5
:10A7F00011F0ECFA45F278700121C0F2020015F078
:10A8000069F94EF2402023460A220E21C2F20000CE
:10A8100011F0DCFA45F668200321C0F2020015F0C1
:10A8200059F906A81AF0CCF8014606A815F052F915
:10A8300045F218600121C0F2020015F04BF94EF20A
:10A840004020C2F2000011F0AFFA00233B700DB0BF
:10A85000BDE8F0835B232A460221069507958DF813
:10A860001830089509950A958DF82C5010F036FB94
:10A8700006A81AF0A5F8024641F6606006A9C2F2E1
:10A88000010011F01DFA4EF240202B460A22294603
:10A89000C2F2000011F09AFA45F278700121C0F27C
:10A8A000020015F017F94EF240202B460A22022131
:10A8B000C2F2000011F08AFA45F668200321C0F2C6
:10A8C000020015F007F906A81AF07AF8014606A862
:10A8D00015F000F945F218600121C0F2020015F0F0
:10A8E000F9F84EF24020C2F2000011F05DFA41F694
:10A8F000A440C2F201001AF063F8C2B2082A41F67D
:10A90000A44128BF08224FF02033C2F2010106A85B
:10A91000069307950895CDF81B3009950A958DF893
:10A920002C501AF0BBF841F660602A460321C2F2AF
:10A93000010010F0D3FA06A81AF042F8024641F6D8
:10A94000606006A9C2F2010011F0BAF94EF240208F
:10A950002B460A222946C2F2000011F037FA45F2CE
:10A9600078700121C0F2020015F0B4F84EF24020D8
:10A970002B460A220321C2F2000011F027FA45F605
:10A9800068200321C0F2020015F0A4F806A81AF00E
:10A9900017F8014606A815F09DF845F21860012148
:10A9A000C0F2020015F096F84EF24020C2F200000C
:10A9B00011F0FAF941F660605D232A460B21C2F2DC
:10A9C0000100069507958DF81830089509950A95A8
:10A9D0008DF82C5010F082FA06A819F0F1FF02460B
:10A9E00041F6606006A9C2F2010011F069F94EF269
:10A9F00040202B460A222946C2F2000011F0E6F957
:10AA000045F27870C0F20200012115F063F82B4680
:10AA10002CE55B2342460221069407948DF81830FA
:10AA2000089409940A948DF82C4010F057FA06A85F
:10AA300019F0C6FF024641F6606006A9C2F20100A5
:10AA400011F03EF94EF2402023460A224146C2F25E
:10AA5000000011F0BBF945F278704146C0F20200E7
:10AA600015F038F84EF2402023460A220221C2F2A5
:10AA7000000011F0ABF945F668200321C0F2020096
:10AA800015F028F806A819F09BFF014606A815F056
:10AA900021F845F218604146C0F2020015F01AF89C
:10AAA0004EF24020C2F2000011F07EF9727941F6B8
:10AAB000F44302EB820602EB4606C2F201031E4497
:10AAC000304619F07DFFC2B20A2A28BF0A224FF091
:10AAD0002033314606A806930793089409940A94F4
:10AAE0008DF82C408DF8205019F0D8FF41F66060A9
:10AAF00042460321C2F2010010F0F0F906A819F055
:10AB00005FFF024641F6606006A9C2F2010011F043
:10AB1000D7F84EF2402023460A224146C2F20000F6
:10AB200011F054F945F278704146C0F2020014F079
:10AB3000D1FF4EF2402023460A220321C2F2000038
:10AB400011F044F945F668200321C0F2020014F028
:10AB5000C1FF06A819F034FF014606A814F0BAFF99
:10AB600045F218604146C0F2020014F0B3FF4EF205
:10AB70004020C2F2000011F017F941F660605D2339
:10AB800042460E21C2F20100069407948DF8183057
:10AB9000089409940A948DF82C4010F09FF906A8A7
:10ABA00019F00EFF024641F6606006A9C2F20100EC
:10ABB00011F086F84EF2402023460A224146C2F2A6
:10ABC000000011F003F945F278704146C0F202002E
:10ABD00014F080FF4EF2402023460A220E21C2F2DA
:10ABE000000011F0F3F845F668200321C0F20200DE
:10ABF00014F070FF06A819F0E3FE014606A814F051
:10AC000069FF45F218604146C0F2020014F062FF8D
:10AC10004EF24020C2F2000011F0C6F800233B7053
:10AC20000DB0BDE8F08341F66060C2F2010010F0A3
:10AC300099F9FFF764BA00BF2DE9F04140F21D0613
:10AC4000C2F201068CB03378032B00F03E8341F64C
:10AC50006060C2F2010010F085F945F6A843C0F229
:10AC6000020393E8030006AC00254FF02033A360F5
:10AC70006360E5602561C4F80B302575069041F6E8
:10AC800060602A46ADF81C10C2F20100294610F09F
:10AC900025F9204619F094FE024641F660602146EF
:10ACA000C2F2010011F00CF84EF240202B460A22AD
:10ACB0002946C2F2000011F089F845F278700121AE
:10ACC000C0F2020014F006FF4EF240202B460A228A
:10ACD0002946C2F2000011F079F845F668200321F8
:10ACE000C0F2020014F0F6FE204619F069FE01469B
:10ACF000204614F0EFFE45F218600121C0F2020078
:10AD000014F0E8FE4EF24020C2F2000011F04CF8C0
:10AD100046F2525341F66060C3F67323294601227E
:10AD2000C2F201006560A560E560256125750693A6
:10AD300010F0D4F8204619F043FE024641F6606058
:10AD40002146C2F2010010F0BBFF4EF240202B461C
:10AD50000A220121C2F2000011F038F845F27870A1
:10AD60000121C0F2020014F0B5FE4EF240202B4645
:10AD70000A222946C2F2000011F028F845F66820A0
:10AD80000321C0F2020014F0A5FE204619F018FEBF
:10AD90000146204614F09EFE45F218600121C0F2E3
:10ADA000020014F097FE4EF24020C2F2000010F0B4
:10ADB000FBFF47F2435341F66060C3F67423012260
:10ADC0000821C2F201006560A560E5602561257576
:10ADD000069310F083F8204619F0F2FD024641F682
:10ADE00060602146C2F2010010F06AFF4EF240207E
:10ADF0002B460A220121C2F2000010F0E7FF45F2C3
:10AE000078700121C0F2020014F064FE4EF240207E
:10AE10002B460A220821C2F2000010F0D7FF45F6A7
:10AE200068200321C0F2020014F054FE204619F0FD
:10AE3000C7FD0146204614F04DFE45F21860C0F2F1
:10AE40000200012114F046FE4EF24020C2F2000042
:10AE500010F0AAFF41F6F143C2F201034FF2CB0812
:10AE60001B7803EB830303EB8303C2F68D089B007F
:10AE700088FB0320DB17C3EB201069460A2219F078
:10AE800073F9054619F09CFDC0B20228024628BF9E
:10AE90000222C2F10200294643F230070025204475
:10AEA00006956560A560E56025612575ADF81870AB
:10AEB00019F0F4FD41F6606001220521C2F20100A3
:10AEC00010F00CF8204619F07BFD024641F6606058
:10AED0002146C2F2010010F0F3FE4EF240202B4654
:10AEE0000A220121C2F2000010F070FF45F27870D2
:10AEF0000121C0F2020014F0EDFD4EF240200A22C2
:10AF00002B460521C2F2000010F060FF45F66820D4
:10AF10000321C0F2020014F0DDFD204619F050FDBF
:10AF20000146204614F0D6FD45F218600121C0F21A
:10AF3000020014F0CFFD4EF24020C2F2000010F0EB
:10AF400033FF40F21C03C2F2010369461B7803EB96
:10AF5000830303EB83039B0088FB0320DB17C3EB16
:10AF600020100A2219F000F9804619F029FDC0B21C
:10AF70000228024628BF0222C2F1020041462044B4
:10AF800006956560A560E56025612575ADF81870CA
:10AF900019F084FD41F6606001220D21C2F201002A
:10AFA0000FF09CFF204619F00BFD024641F6606051
:10AFB0002146C2F2010010F083FE4EF240202B46E3
:10AFC0000A220121C2F2000010F000FF45F2787061
:10AFD0000121C0F2020014F07DFD4EF240202B460C
:10AFE0000A220D21C2F2000010F0F0FE45F66820A2
:10AFF0000321C0F2020014F06DFD204619F0E0FCC0
:10B000000146204614F066FD45F218600121C0F2A9
:10B0100002004DF6A66714F05DFDC2F200074EF285
:10B020004020C2F2000010F0BFFE97F8008041F609
:10B030006060B8F1040FC2F2010000F04881012203
:10B0400004214FF0200806956560A560E560256144
:10B0500025758DF818800FF041FF204619F0B0FCDF
:10B06000024641F660602146C2F2010010F028FE5F
:10B070004EF240202B460A220121C2F2000010F0BD
:10B08000A5FE45F278700121C0F2020014F022FD05
:10B090004EF240200A222B460421C2F2000010F09A
:10B0A00095FE45F668200321C0F2020014F012FD5F
:10B0B000204619F085FC0146204614F00BFD45F2B0
:10B0C00018600121C0F2020014F004FD4EF240208D
:10B0D000C2F2000010F068FE41F660600695C2F210
:10B0E00001006560A560E5602561257501220721E5
:10B0F0008DF818800FF0F2FE204619F061FC024630
:10B1000041F660602146C2F2010010F0D9FD4EF216
:10B1100040202B460A220121C2F2000010F056FE08
:10B1200045F278700121C0F2020014F0D3FC4EF217
:10B1300040202B460A220721C2F2000010F046FEF2
:10B1400045F668200321C0F2020014F0C3FC20463B
:10B1500019F036FC0146204614F0BCFC45F218609C
:10B160000121C0F2020014F0B5FC4EF24020C2F200
:10B17000000010F019FE3B7841F66060052B4FF09F
:10B180000005C2F2010000F0FE8001220C21202700
:10B1900006956560A560E560256125758DF81870D8
:10B1A0000FF09CFE204619F00BFC024641F6606051
:10B1B0002146C2F2010010F083FD4EF240202B46E2
:10B1C0000A220121C2F2000010F000FE45F2787060
:10B1D0000121C0F2020014F07DFC4EF240200A2250
:10B1E0002B460C21C2F2000010F0F0FD45F668205D
:10B1F0000321C0F2020014F06DFC204619F0E0FBC0
:10B200000146204614F066FC45F218600121C0F2A8
:10B21000020014F05FFC4EF24020C2F2000010F079
:10B22000C3FD41F660600695C2F201006560A5604D
:10B23000E5602561257501220F218DF818700FF04A
:10B240004DFE204619F0BCFB024641F660602146E7
:10B25000C2F2010010F034FD4EF240202B460A22CB
:10B260000121C2F2000010F0B1FD45F27870012119
:10B27000C0F2020014F02EFC4EF240202B460A22AF
:10B280000F21C2F2000010F0A1FD45F66820032155
:10B29000C0F2020014F01EFC204619F091FB01469A
:10B2A000204614F017FC45F218600121C0F202009C
:10B2B00014F010FC4EF24020C2F2000010F074FDB9
:10B2C000032333700CB0BDE8F08106ACC2E55B230C
:10B2D0000122414606956560A560E56025612575FA
:10B2E0008DF818300FF0FAFD204619F069FB024680
:10B2F00041F660602146C2F2010010F0E1FC4EF21E
:10B3000040202B460A220121C2F2000010F05EFD0F
:10B3100045F278700121C0F2020014F0DBFB4EF21E
:10B3200040202B460A224146C2F2000010F04EFD9A
:10B3300045F668200321C0F2020014F0CBFB204642
:10B3400019F03EFB0146204614F0C4FB45F218609C
:10B350000121C0F2020014F0BDFB4EF24020C2F207
:10B36000000010F021FD41F660605D230695C2F2F9
:10B3700001006560A560E560256125750122072152
:10B380008DF81830B6E65B2301220C210695656026
:10B39000A560E560256125758DF818300FF09EFDDC
:10B3A000204619F00DFB024641F660602146C2F2CC
:10B3B000010010F085FC4EF240202B460A220121AC
:10B3C000C2F2000010F002FD45F278700121C0F2D7
:10B3D000020014F07FFB4EF240202B460A220C2183
:10B3E000C2F2000010F0F2FC45F668200321C0F222
:10B3F000020014F06FFB204619F0E2FA01462046E5
:10B4000014F068FB45F218600121C0F2020014F04C
:10B4100061FB4EF24020C2F2000010F0C5FC41F684
:10B4200060605D230695C2F201006560A560E5607D
:10B430002561257501220F218DF81830FFE600BF28
:10B44000F0B54AF23473C2F2010340F21D068FB028
:10B45000C2F201061B6801933278019941F66473C8
:10B46000C2F20103022A196000F0D18041F6606047
:10B47000C2F201000FF076FD45F6B043C0F20203C0
:10B4800093E8070008AC00254FF02033E560C4F8CE
:10B490000B3084E8070041F660602A462946C2F274
:10B4A0000100256125750FF019FD204619F088FA75
:10B4B000024641F660602146C2F2010010F000FC35
:10B4C0004EF240202B4629460A22C2F2000010F01C
:10B4D0007DFC45F278700121C0F2020014F0FAFA06
:10B4E0004EF240202B460A222946C2F2000010F0FC
:10B4F0006DFC45F668200321C0F2020014F0EAFA60
:10B50000204619F05DFA0146204614F0E3FA45F2B0
:10B5100018600121C0F202004DF6A86714F0DAFAB3
:10B52000C2F200074EF24020C2F2000010F03CFCD4
:10B530003D7C002D73D00A2202A9284618F014FE83
:10B54000054619F03DFAC0B20228024628BF022281
:10B55000C2F1020043F23003294620440025089539
:10B560006560A560E56025612575ADF8203019F0AE
:10B5700095FA41F6606029460122C2F201000FF0FF
:10B58000ADFC204619F01CFA024641F660602146E7
:10B59000C2F2010010F094FB4EF240202B460A222A
:10B5A0000121C2F2000010F011FC45F27870012177
:10B5B000C0F2020014F08EFA4EF240202B460A220E
:10B5C0002946C2F2000010F001FC45F66820032174
:10B5D000C0F2020014F07EFA204619F0F1F901469B
:10B5E000204614F077FA45F218600121C0F20200FB
:10B5F00014F070FA4EF24020C2F2000010F0D4FBBA
:10B600003F7C012F60D0022333700FB0F0BD4DF6A8
:10B61000A867C2F2000708AC3D7C002D8BD144F630
:10B620004F5341F66060C4F64E1329460122C2F220
:10B6300001006560A560E5602561257508930FF040
:10B640004DFC204619F0BCF9024641F660602146E7
:10B65000C2F2010010F034FB4EF240202B460A22C9
:10B660000121C2F2000010F0B1FB45F27870012117
:10B67000C0F2020014F02EFA4EF240202B460A22AD
:10B680002946C2F2000010F0A1FB45F66820032114
:10B69000C0F2020014F01EFA204619F091F901469A
:10B6A000204614F017FA45F218600121C0F202009A
:10B6B00014F010FA4EF24020C2F2000010F074FBB9
:10B6C000022333700FB0F0BD41F6606042F22003F8
:10B6D0003A460221C2F2010008956560A560E56066
:10B6E00025612575ADF820300FF0F8FB204619F0E4
:10B6F00067F9024641F660602146C2F2010010F08F
:10B70000DFFA4EF240202B460A223946C2F20000F0
:10B7100010F05CFB45F278703946C0F2020014F07C
:10B72000D9F94EF240202B460A220221C2F2000033
:10B7300010F04CFB45F668200321C0F2020014F023
:10B74000C9F9204619F03CF90146204614F0C2F927
:10B7500045F218603946C0F2020014F0BBF94EF20F
:10B760004020C2F2000010F01FFB022333700FB024
:10B77000F0BD00BF2DE9F04140F21D06C2F2010606
:10B780008CB03378042B00F0F88441F66060C2F28C
:10B7900001000FF0E7FB45F6C043C0F2020393E857
:10B7A000030006AC00256560A560E5602561257590
:10B7B000069041F660602A468DF81C10C2F2010026
:10B7C00029460FF08BFB204619F0FAF8024641F6A5
:10B7D00060602146C2F2010010F072FA4EF2402081
:10B7E0002B460A222946C2F2000010F0EFFA45F279
:10B7F00078700121C0F2020014F06CF94EF2402082
:10B800002B460A222946C2F2000010F0DFFA45F664
:10B8100068200321C0F2020014F05CF9204619F000
:10B82000CFF80146204614F055F945F21860012181
:10B83000C0F2020014F04EF94EF24020C2F20000B5
:10B8400010F0B2FA41F6606043F654232A4606210E
:10B85000C2F2010006956560A560E5602561257569
:10B86000ADF818300FF03AFB204619F0A9F802465F
:10B8700041F660602146C2F2010010F021FA4EF25A
:10B8800040202B460A222946C2F2000010F09EFA00
:10B8900045F278700121C0F2020014F01BF94EF25B
:10B8A00040202B460A220621C2F2000010F08EFA38
:10B8B00045F668200321C0F2020014F00BF920467F
:10B8C00019F07EF80146204614F004F945F218609C
:10B8D0000121C0F2020014F0FDF84EF24020C2F245
:10B8E000000010F061FA41F6606047F26D332A46BD
:10B8F0000E21C2F2010006956560A560E560256134
:10B900002575ADF818300FF0E9FA204619F058F80F
:10B91000024641F660602146C2F2010010F0D0F903
:10B920004EF240202B460A222946C2F2000010F0B7
:10B930004DFA45F278700121C0F2020014F0CAF805
:10B940004EF240202B460A220E21C2F2000010F0D7
:10B950003DFA45F668200321C0F2020014F0BAF85F
:10B96000204619F02DF80146204614F0B3F845F2B0
:10B9700018600121C0F2020014F0ACF84EF2402031
:10B98000C2F2000010F010FA45F6C843C0F20203FC
:10B9900041F660601B6806951F0C29460122C2F221
:10B9A00001006560A560E56025612575ADF818307A
:10B9B0008DF81A700FF092FA204619F001F802463D
:10B9C00041F660602146C2F2010010F079F94EF2B2
:10B9D00040202B460A220121C2F2000010F0F6F9A5
:10B9E00045F278700121C0F2020014F073F84EF2B3
:10B9F00040202B460A222946C2F2000010F0E6F948
:10BA000045F668200321C0F2020014F063F82046D6
:10BA100018F0D6FF0146204614F05CF845F2186095
:10BA20000121C0F2020014F055F84EF24020C2F29B
:10BA3000000010F0B9F946F6567341F66060C3F69F
:10BA40006C2301220821C2F201006560A560E56057
:10BA50002561257506930FF041FA204618F0B0FFD6
:10BA6000024641F660602146C2F2010010F028F95A
:10BA70004EF240202B460A220121C2F2000010F0B3
:10BA8000A5F945F278700121C0F2020014F022F805
:10BA90004EF240202B460A220821C2F2000010F08C
:10BAA00095F945F668200321C0F2020014F012F85F
:10BAB000204618F085FF0146204614F00BF845F2A9
:10BAC0001860C0F20200012114F004F84EF2402088
:10BAD000C2F2000010F068F940F26C52C2F20102AA
:10BAE0004FF49663107848F21F57C5F2EB1703FB2B
:10BAF00000F387FB0320DB17C3EB201069460A2203
:10BB000018F032FB054618F05BFFC0B2042802466D
:10BB100028BF0422C2F104004FF0303329462044EC
:10BB200000256560A560E56025612575069318F020
:10BB3000B5FF41F660602A460921C2F201000FF00C
:10BB4000CDF9204618F03CFF024641F660602146E0
:10BB5000C2F2010010F0B4F84EF240202B460A2247
:10BB60002946C2F2000010F031F945F27870012147
:10BB7000C0F2020013F0AEFF4EF240200A222B4624
:10BB80000921C2F2000010F021F945F668200321D6
:10BB9000C0F2020013F09EFF204618F011FF01468C
:10BBA000204613F097FF45F218600121C0F2020011
:10BBB00013F090FF4EF24020C2F2000010F0F4F8B3
:10BBC00041F6F043C2F201034AF2EB001B7803EBAB
:10BBD000430303EB4313CEF60E2080FB03201844EF
:10BBE000DB17C3EB601069460A2218F0BDFA8046E5
:10BBF00018F0E6FEC0B20228024628BF0222C2F1B7
:10BC000002004146204443F2300806956560A56075
:10BC1000E56025612575ADF8188018F03FFF41F605
:10BC2000606001220421C2F201000FF057F92046A2
:10BC300018F0C6FE024641F660602146C2F20100DD
:10BC400010F03EF84EF240202B460A220121C2F2AB
:10BC5000000010F0BBF845F278700121C0F202003C
:10BC600013F038FF4EF240200A222B460421C2F284
:10BC7000000010F0ABF845F668200321C0F2020086
:10BC800013F028FF204618F09BFE0146204613F0D3
:10BC900021FF45F218600121C0F2020013F01AFFE3
:10BCA0004EF24020C2F2000010F07EF841F67463BC
:10BCB000C2F2010369461B7803EB430303EB431312
:10BCC00087FB0320DB17C3EB20100A2218F04CFA85
:10BCD000074618F075FEC0B20228024628BF0222AD
:10BCE000C2F102003946204406956560A560E56012
:10BCF00025612575ADF8188018F0D0FE41F660601A
:10BD000001220D21C2F201000FF0E8F8204618F0E0
:10BD100057FE024641F660602146C2F201000FF074
:10BD2000CFFF4EF240202B460A220121C2F2000032
:10BD300010F04CF845F278700121C0F2020013F0C7
:10BD4000C9FE4EF240202B460A220D21C2F200000D
:10BD500010F03CF845F668200321C0F2020013F011
:10BD6000B9FE204618F02CFE0146204613F0B2FE24
:10BD700045F218600121C0F202004DF6A66713F0EB
:10BD8000A9FEC2F200074EF24020C2F2000010F0FD
:10BD90000BF83B7841F66060062BC2F2010000F020
:10BDA0004A822A4608214FF0200806956560A56062
:10BDB000E560256125758DF818800FF08FF8204615
:10BDC00018F0FEFD024641F660602146C2F2010015
:10BDD0000FF076FF4EF240202B460A222946C2F28F
:10BDE00000000FF0F3FF45F278700121C0F202006D
:10BDF00013F070FE4EF240200A222B460821C2F2B8
:10BE000000000FF0E3FF45F668200321C0F20200B6
:10BE100013F060FE204618F0D3FD0146204613F0D3
:10BE200059FE45F218600121C0F2020013F052FEE3
:10BE30004EF24020C2F200000FF0B6FF41F6606003
:10BE40000695C2F201006560A560E5602561257573
:10BE50002A460D218DF818800FF040F8204618F082
:10BE6000AFFD024641F660602146C2F201000FF0CC
:10BE700027FF4EF240202B460A222946C2F200003C
:10BE80000FF0A4FF45F278700121C0F2020013F018
:10BE900021FE4EF240202B460A220D21C2F2000064
:10BEA0000FF094FF45F668200321C0F2020013F062
:10BEB00011FE204618F084FD0146204613F00AFECC
:10BEC00045F218600121C0F2020013F003FE4EF2A9
:10BED0004020C2F200000FF067FF3B7841F660603F
:10BEE000072B4FF00005C2F2010000F0488101224B
:10BEF00003214FF0200806956560A560E560256187
:10BF000025758DF818800EF0E9FF204618F058FDD1
:10BF1000024641F660602146C2F201000FF0D0FEF9
:10BF20004EF240202B460A220121C2F200000FF0FF
:10BF30004DFF45F278700121C0F2020013F0CAFDF6
:10BF40004EF240200A222B460321C2F200000FF0DD
:10BF50003DFF45F668200321C0F2020013F0BAFD50
:10BF6000204618F02DFD0146204613F0B3FD45F2A2
:10BF700018600121C0F2020013F0ACFD4EF2402027
:10BF8000C2F200000FF010FF41F660600695C2F2A9
:10BF900001006560A560E560256125750122062127
:10BFA0008DF818800EF09AFF204618F009FD024621
:10BFB00041F660602146C2F201000FF081FE4EF2B0
:10BFC00040202B460A220121C2F200000FF0FEFEA3
:10BFD00045F278700121C0F2020013F07BFD4EF2B1
:10BFE00040202B460A220621C2F200000FF0EEFE8E
:10BFF00045F668200321C0F2020013F06BFD2046D5
:10C0000018F0DEFC0146204613F064FD45F218608E
:10C010000121C0F2020013F05DFD4EF24020C2F299
:10C0200000000FF0C1FE3B7841F66060082B4FF036
:10C030000005C2F2010000F05A8101220C212027E4
:10C0400006956560A560E560256125758DF8187019
:10C050000EF044FF204618F0B3FC024641F6606043
:10C060002146C2F201000FF02BFE4EF240202B467B
:10C070000A220121C2F200000FF0A8FE45F27870FA
:10C080000121C0F2020013F025FD4EF240200A22E9
:10C090002B460C21C2F200000FF098FE45F66820F6
:10C0A0000321C0F2020013F015FD204618F088FCB1
:10C0B0000146204613F00EFD45F218600121C0F242
:10C0C000020013F007FD4EF24020C2F200000FF014
:10C0D0006BFE41F660600695C2F201006560A560E6
:10C0E000E5602561257501220F218DF818700EF08D
:10C0F000F5FE204618F064FC024641F660602146D9
:10C10000C2F201000FF0DCFD4EF240202B460A2265
:10C110000121C2F200000FF059FE45F278700121B2
:10C12000C0F2020013F0D6FC4EF240202B460A2249
:10C130000F21C2F200000FF049FE45F668200321EE
:10C14000C0F2020013F0C6FC204618F039FC01468C
:10C15000204613F0BFFC45F218600121C0F2020036
:10C1600013F0B8FC4EF24020C2F200000FF01CFEAB
:10C17000042333700CB0BDE8F08106ACACE45B2363
:10C180000122032106956560A560E560256125759E
:10C190008DF818300EF0A2FE204618F011FC024671
:10C1A00041F660602146C2F201000FF089FD4EF2B7
:10C1B00040202B460A220121C2F200000FF006FEA9
:10C1C00045F278700121C0F2020013F083FC4EF2B8
:10C1D00040202B460A220321C2F200000FF0F6FD98
:10C1E00045F668200321C0F2020013F073FC2046DC
:10C1F00018F0E6FB0146204613F06CFC45F218608F
:10C200000121C0F2020013F065FC4EF24020C2F2A0
:10C2100000000FF0C9FD41F660605D230695C2F293
:10C2200001006560A560E560256125750122062194
:10C230008DF81830B6E65B232A460821069565601E
:10C24000A560E560256125758DF818300EF046FE75
:10C25000204618F0B5FB024641F660602146C2F266
:10C2600001000FF02DFD4EF240202B460A222946F8
:10C27000C2F200000FF0AAFD45F278700121C0F271
:10C28000020013F027FC4EF240202B460A22082120
:10C29000C2F200000FF09AFD45F668200321C0F2BB
:10C2A000020013F017FC204618F08AFB01462046D6
:10C2B00013F010FC45F218600121C0F2020013F0E7
:10C2C00009FC4EF24020C2F200000FF06DFD41F675
:10C2D00060605D230695C2F201006560A560E560BF
:10C2E000256125752A460D218DF81830B4E55B23AC
:10C2F00001220C2106956560A560E5602561257524
:10C300008DF818300EF0EAFD204618F059FB024671
:10C3100041F660602146C2F201000FF0D1FC4EF2FE
:10C3200040202B460A220121C2F200000FF04EFDF0
:10C3300045F278700121C0F2020013F0CBFB4EF2FF
:10C3400040202B460A220C21C2F200000FF03EFDD5
:10C3500045F668200321C0F2020013F0BBFB204623
:10C3600018F02EFB0146204613F0B4FB45F218608E
:10C370000121C0F2020013F0ADFB4EF24020C2F2E8
:10C3800000000FF011FD41F660605D230695C2F2DA
:10C3900001006560A560E5602561257501220F211A
:10C3A0008DF81830A3E600BF2DE9F04F2DED068B78
:10C3B0004AF23477C2F2010789B041F664723B68F1
:10C3C0000493C2F20102049B116840F6B7325B1A73
:10C3D000934207D940F21D03C2F201031B78002BE0
:10C3E00040F0488141F2F448C2F2010841F670631E
:10C3F0003A680592C2F2010341F287321968059B3F
:10C400005B1A934208D94DF6A663C2F200031A786C
:10C41000911E012940F2E28041F2F444C2F201048B
:10C4200041F6D04340F224064BF6836A04F10C0235
:10C43000C2F201039FEDD08A9FEDD09ADFEDD08A42
:10C440009FEDD0AADFEDD09ACDF80480C2F20106AC
:10C450000093C2F6A07A0025904603EB051B5846D0
:10C460000EF0A6FB58465FFA85F90EF0E7FB38B1EF
:10C470003B68069341F6B443C2F20103069A1A6080
:10C4800058460EF0D1FBA0B341F6B4433A68079288
:10C49000C2F201031A68079B9B1AB3F5FA7F00F2F8
:10C4A000238140F21D03C2F20103B9F1010F1B7891
:10C4B00000F0D580012B00F07284C0F01183022BB4
:10C4C00000F08784AB4645F6F8400721C0F2020031
:10C4D00013F000FB4EF240205946C2F20000002348
:10C4E0000A220FF073FC4EF24020C2F200000FF05F
:10C4F0005BFC237C012B40F2498172B6E36862B693
:10C50000002B56F8042BB8BF0333B2EBA30F5CD05B
:10C51000B9F1010F6DD140F21D02C2F20102137890
:10C52000012B00F0AE82C0F06983032B00F0FA818A
:10C53000042B0FD14DF6A663C2F200031B78072B24
:10C5400000F0E986082B00F0CB84062B00F053871F
:10C55000FFF710F945F644600821C0F2020013F01D
:10C56000B9FA4EF2402000230A222946C2F2000006
:10C570000FF02CFC45F62820C0F20200022113F037
:10C58000A9FA237C012B40F2068372B6E16862B6F9
:10C590000029B8BF03314EF240208910C2F20000DA
:10C5A0000FF0A4FB4EF24020C2F200000FF0FCFBA3
:10C5B000237C012B40F2C48272B6E36862B6002B82
:10C5C000B8BF03339B1046F8043C0135022D04F13B
:10C5D000140408F1140807D0009B3EE7032A40F03A
:10C5E000008101221A7017E709B0BDEC068BBDE887
:10C5F000F08F40F21D03C2F201031B78012B40F2C1
:10C60000F380022BA6D1237C012B40F2D28772B695
:10C61000E36862B6032B40F35185237C012B41F282
:10C62000508072B6E36862B63F2B03DD72B64023DA
:10C63000E36062B6237C012B40F28F8772B6E36819
:10C6400062B64DF6A862002BC2F20002B8BF0333F7
:10C650009B101374FAF710F8FEF7F2FE7AE7002B3E
:10C6600000F02982033B012B4FF0040140F2388394
:10C67000CB4628E7033B012B7FF6B4AE4DF6A8630B
:10C68000C2F2000393ED027ADFED3B6ADFED3B7A05
:10C690009FED3B6A27EE267A27EE277AC7EE267AA9
:10C6A00077EE867AFDEEE77A17EE903A9B0072B647
:10C6B00041F2F448C2F20108C8F80C3062B698F8AA
:10C6C0001030012B40F2388372B6D8F80C3062B6C5
:10C6D00040F22402002BC2F20102B8BF03339B10C8
:10C6E0001360FDF701FD81E645F6CC402921C0F23B
:10C6F000020013F0EFF94EF2402000230A222946EF
:10C70000C2F200000FF062FB4EF24020C2F20000C5
:10C710000FF04AFBB9F1010FAB467FF4D4AE40F203
:10C720001D03C2F201031B78032B00F0FC84042BD1
:10C7300000F0DA84002B7FF4C6AE4DF6A66241F617
:10C74000F143C2F20002C2F20103042111701B780E
:10C7500072B69B00E36062B6237C012B41F2158325
:10C7600072B6E36862B6002BB8BF03339B10336028
:10C77000FEF762FAA7E600BF0000C84200002C42A4
:10C780000000000000000C4200FEFF4672B694E874
:10C790000C0010781978637A227A194202EA0002B2
:10C7A00000F0B780A37A03F003030AB143F0040357
:10C7B00043F008039A10082BA27200F21482072B90
:10C7C00080F03483032B00F0368340F2AF81042BDA
:10C7D00000F0B281062B7FF491AEE368023BE36088
:10C7E0008DE600221A7017E6237C012B40F2898621
:10C7F00072B6E36862B6032B40F36684237C012B98
:10C8000040F28B8772B6E36862B6AB2B03DD72B67B
:10C81000AC23E36062B6237C012B40F2228772B620
:10C82000E36862B6002B227CB8BF03339B10012A59
:10C8300046F8043C40F2E98672B6E36862B6002B23
:10C84000B8BF03339A10642303FB02F38AFB03127D
:10C85000DB17C3EBE20307EE903AF8EEE77A4DF60A
:10C86000A86387EE887AC2F2000341F26059C2F2EF
:10C87000010945F6005014221C21C0F20200A9F85B
:10C8800004200293D3ED027A77EE677AF3EE046A1E
:10C8900087EEA67A89ED007A13F01CF9029B98685E
:10C8A00017F074F841EC100B4EF240200521C2F253
:10C8B00000000FF0CBFA45F620500E21C0F2020026
:10C8C00013F008F94EF24020B9F80410C2F200004B
:10C8D0000FF00CFA45F630500E21C0F2020013F0B2
:10C8E000F9F8D9F8000017F051F841EC100B4EF2AE
:10C8F00040200521C2F200000FF0A8FA4EF24020BD
:10C90000C2F200000FF050FAF9F7B6FEFDF7CEF9CB
:10C9100020E6A37A03F00303002A3FF44BAF43F071
:10C92000040347E74DF6A663C2F200031B78042B0D
:10C9300000F02084052B40F0A180237C012B41F2E4
:10C94000E68272B6E36862B6032B40F3E887237C85
:10C95000012B41F2AB8472B6E36862B6B3F5C87FCF
:10C9600004DB72B64FF4C873E36062B6237C012B1C
:10C9700041F2A18272B6E36862B6002B227CB8BF96
:10C9800003339B10012A46F8043C41F2688272B6D8
:10C99000E36862B640F21C02002B217CB8BF03336F
:10C9A000C2F201029B100129137041F2528272B649
:10C9B000E36862B6002BB8BF03339B1007EE903AD2
:10C9C000B8EEE77A41F2905BC7EE087AC2F2010B4B
:10C9D00040F2F069DBF80030C2F2010945F6A050E0
:10C9E00014222321C0F20200A9F80420B7EE007A35
:10C9F00037EE677AD3ED587A77EE677AF3EE046A0A
:10CA000087EEA67A89ED007A13F064F8DBF800303F
:10CA1000D3F8600116F0BAFF41EC100B4EF2402043
:10CA20000521C2F200000FF011FA45F6C45015219D
:10CA3000C0F2020013F04EF84EF24020B9F8041094
:10CA4000C2F200000FF052F945F6DC50C0F20200CD
:10CA5000152113F03FF8D9F8000016F097FF41ECCC
:10CA6000100B4EF24020C2F2000005210FF0EEF94B
:10CA70004EF24020C2F200000FF096F9FEF7DCF80B
:10CA800068E54DF6A86341F66060C2F2000300213C
:10CA9000C2F201000293039311700EF063FA029B3D
:10CAA0005B7972B6019A9B00136262B6F9F7E4FDF6
:10CAB000FDF71AFB4EE54DF6A662C2F200021378AE
:10CAC000012B00F01484C0F0E182022B00F0DE8222
:10CAD000032B00F00C84FDF707FB4FF0010BF2E491
:10CAE0004DF6A863C2F2000393ED027A27EE087AAE
:10CAF00027EE097AC7EE087A77EEA87AFDEEE77A94
:10CB000017EE903A9B0072B6E36062B6237C012B6D
:10CB100040F2108772B6E36862B6002BB8BF0333E9
:10CB20009B103360AB46FDF7C1F8CCE4012B00F05D
:10CB30007D81022B7FF4E2ACE368013BE360DEE43D
:10CB400072B694E80C0010781978637A227A194248
:10CB500002EA000200F09680A37A03F003030AB110
:10CB600043F0040343F008039A10082BA27200F26A
:10CB7000A880072B80F0AF81032B00F0B08240F239
:10CB80006681042B00F0A880062B7FF416ADE368C5
:10CB9000023BE36012E572B694E80C001078197855
:10CBA000637A227A194202EA000274D0A37A03F06F
:10CBB00003030AB143F0040343F008039A10082B5F
:10CBC000A27270D8072B80F07B81032B00F0828249
:10CBD00040F23681042B70D0062B7FF4D7ACE1688D
:10CBE0000239E160D3E40C2B00F0258100F21881BA
:10CBF000092B3FF4F2AD0B2B9ED07FE44DF6A663DC
:10CC0000C2F200031A78012A00F05785C0F0FB81B8
:10CC1000022A00F0FA81032A31D1237C012B40F251
:10CC2000B18772B6E36862B6032B40F31586237CA6
:10CC3000012B41F2A38272B6E36862B67F2B4DF6F8
:10CC4000A863C2F2000307DD1A79622A41F2A681C5
:10CC500072B67C22E26062B6227C012A40F2BC8776
:10CC600072B6E26862B6002AB8BF0332C2F3870226
:10CC7000114618795A7103F02BFEF9F7FDFCFDF708
:10CC800033FA67E4A37A03F00303002A3FF46CAF9E
:10CC900043F0040368E7A37A03F00303002A8DD06E
:10CCA00043F004038AE70C2B00F0148200F20281A7
:10CCB000092B94D00B2B7FF469ACE1680139E1605A
:10CCC00065E40C2B00F00B8200F2FF80092B3FF48F
:10CCD0005EAF0B2B7FF471ACE368013BE3606DE466
:10CCE0004DF6A663C2F200031A78062A00F05585B5
:10CCF00000F2BD80042A00F05785052A40F0F38237
:10CD000041F6F142C2F201021970137872B69B002B
:10CD1000E36062B6237C012B41F25B8272B6E3686A
:10CD200062B6002BB8BF03339B1033604FF0010B8A
:10CD3000FDF782FFFFF7C7BB72B6D8F80030D8F80E
:10CD400004101A78087898F8091098F80830084202
:10CD500002EA030200F0828098F80A3003F003032D
:10CD60000AB143F0040343F008039A10082B88F833
:10CD70000A2000F28D82072B80F00185032B00F042
:10CD8000058540F23585042B00F08D82062B7FF45B
:10CD90009CACD8F80C30023BC8F80C3097E44DF648
:10CDA000A863C2F200031B7C72B69B00E36062B60C
:10CDB000237C012B40F2218672B6E36862B6002B19
:10CDC000B8BF03339B103360AB46FEF739FBFFF768
:10CDD0007ABB4DF6A863C2F2000393ED027A27EE08
:10CDE000087A27EE097AC7EE087A77EEA87AFDEE80
:10CDF000E77A17EE903A9B0072B6E36062B6237C46
:10CE0000012B40F2CD8572B6E36862B6002BB8BF45
:10CE100003339B103360AB46FDF766F9FFF753BB56
:10CE20000D2B3FF489AE0E2B7FF468ABE368013322
:10CE3000E360FFF764BBE3680233E360FFF75FBBC7
:10CE4000012B3DD0022B3FF438AFFFF79FBB012BE6
:10CE500041D0022B3FF440AFFFF7AFBB98F80A3048
:10CE600003F00303002A80D043F004037DE7072A80
:10CE700000F02082082A40F0368240F26C52C2F262
:10CE8000010206211278197072B69300E36062B64F
:10CE9000237C012B41F2808172B6E36862B6002BDD
:10CEA000B8BF03339B1033604FF0010BFEF762FCF9
:10CEB000FFF709BB0D2B3FF400AF0E2B7FF466ABE1
:10CEC000E1680131E160FFF762BB0D2B3FF404AF75
:10CED0000E2B7FF472ABE3680133E360FFF76EBBA8
:10CEE000237C012B41F2CC8172B6E36862B6032B3E
:10CEF00040F3DE85237C012B41F2308272B6E36879
:10CF000062B6CB2B03DD72B6C823E36062B6237C26
:10CF1000012B41F2AF8172B6E36862B6002BB8BF55
:10CF20000333C3F3870307EE903A9FED907AF8EE50
:10CF3000676A41F67469C6EE877AC2F2010989F818
:10CF40000030B7EE007A77EEA87A37EE677AB4EE63
:10CF5000E97AF1EE10FA00F33B84DFED826AB4EE79
:10CF6000E67AF1EE10FA00F1F585F0EE476AFEEE92
:10CF7000C86A16EE903A41F2BC42C2F20102F4EEE7
:10CF8000E97AF1EE10FA936100F31D849FED757A52
:10CF9000F4EEC77AF1EE10FA00F1EA85B0EE677AA6
:10CFA000BEEEC87A17EE103AF4EEE97AF1EE10FA16
:10CFB000D36101F39E849FED6B7AF4EEC77AF1EEB4
:10CFC00010FA00F1D085B0EE677ABEEEC87A17EE9F
:10CFD000103A45F628601921C0F20200136212F0DF
:10CFE00079FD4EF2402099F8001000230A22C2F287
:10CFF00000000EF0EBFE4EF24020C2F200000EF0F8
:10D00000D3FEFFF7A5BA02221A70237C012B40F24F
:10D01000388672B6E36862B6032B40F32A8441F681
:10D02000CC49237CC2F20109012B99F800B041F2EE
:10D03000F68072B6E36862B6002BB8BF0333BBEB71
:10D04000A30F06DC99F80030013B9B0072B6E36049
:10D0500062B6237C012B40F2EA8572B6E36862B6C1
:10D060001A1EB8BF03324DF6A863C2F38702C2F29C
:10D07000000310461A71029303F042F9029B59799A
:10D08000187903F025FCF9F7F7FAF8E54DF6A863EF
:10D09000C2F2000301215B79117072B69B00E3605C
:10D0A00062B6237C8B4240F2318172B6E36862B68D
:10D0B000002BB8BF03339B1033600CE572B600231E
:10D0C000E36062B6FFF7B6BA72B60023E36062B6F9
:10D0D000FFF7A1BBE1680231E160FFF758BAE368EE
:10D0E0000233E360FFF76ABA4DF6A6624DF6A86315
:10D0F000C2F20002C2F2000382F800905B7972B6BD
:10D100009B00E36062B6237C012B40F2118672B66D
:10D11000E36862B6002BB8BF03339B103360FCF7A3
:10D12000E3FFFFF7D0B94DF6A66240F26C53C2F2AE
:10D130000002C2F20103062111701B7872B69B0037
:10D14000E36062B6237C012B40F2C58572B6E368CA
:10D1500062B6002BB8BF03339B103360FEF70AFBA7
:10D16000FFF7B1B900FEFFC6000096440000484238
:10D1700079783042237C012B40F23F8672B6E36817
:10D1800062B6032B40F3D183237C012B41F24D8007
:10D1900072B6E36862B6B3F5C87F04DB72B64FF4CB
:10D1A000C873E36062B6237C012B40F2788772B6C5
:10D1B000E36862B6002B227CB8BF03339B10012AC0
:10D1C00046F8043C40F2138772B6E36862B641F653
:10D1D000F142002B217CB8BF0333C2F201029B1045
:10D1E0000129137040F22F8772B6E36862B6002BF4
:10D1F000B8BF03339B1007EE903AF8EEE77A41F29E
:10D20000905B87EE887AC2F2010B40F24459DBF85A
:10D210000030C2F2010945F6405014222621C0F226
:10D220000200A9F80420F7EE007A37EEC77AD3EDB2
:10D23000597A77EE677AF3EE046A87EEA67A89ED7B
:10D24000007A12F047FCDBF80030D3F8640116F0E6
:10D250009DFB41EC100B4EF240200521C2F2000074
:10D260000EF0F4FD45F668501821C0F2020012F0ED
:10D2700031FC4EF24020B9F80410C2F200000EF06A
:10D2800035FD45F68450C0F202001821FFF7E1BBDE
:10D290000C2B00F07B8200F26C82092B3FF479ADFD
:10D2A0000B2B7FF412AAD8F80C30013BC8F80C30D5
:10D2B000FFF70DBA41F67462C2F20102082112783A
:10D2C000197072B69300E36062B6237C012B41F2C1
:10D2D0007F8172B6E36862B6002BB8BF03339B1040
:10D2E0003360FEF747FA4FF0010BFFF7ECB84DF64D
:10D2F000A863C2F2000300211B79117072B69B0073
:10D30000E36062B6237C012B3FF6CFAE72B62046B7
:10D31000F7F7E8FDCAE6237C012B40F28C8772B652
:10D32000E36862B6032B40F3CD83237C012B41F2EB
:10D330003D8072B6E36862B68F2B03DD72B68C2334
:10D34000E36062B6237C012B40F28E8772B6E368FD
:10D3500062B6002BB8BF0333C3F3870307EE903ADE
:10D36000B8EE677A41F6F049C7EE0A7AC2F20109CF
:10D3700089F8003077EEA87AF4EEE97AF1EE10FA47
:10D3800000F31D821FED897AF4EEC77AF1EE10FAF0
:10D3900000F1E583B0EE677ABEEEC87A17EE103A78
:10D3A00041F28442C2F2010245F60C601B21C0F238
:10D3B0000200D36112F08EFB99F8003007EE903A2C
:10D3C000F8EE677A87EE8A7A77EE287A17EE900A77
:10D3D00016F0DCFA41EC100B4EF240200221C2F2B2
:10D3E00000000EF033FD4EF24020C2F200000EF0BD
:10D3F000DBFCFFF7ADB8237C012B40F22F8772B620
:10D40000E36862B6032B40F34E83237C012B40F28A
:10D41000DC8772B6E36862B6CB2B03DD72B6C82335
:10D42000E36062B6237C012B40F2128772B6E36898
:10D4300062B6002BB8BF0333C3F3870307EE903AFD
:10D44000B8EE677A5FEDB87A5FEDB86A67EE277A73
:10D4500040F26C5987EEA67AC2F2010989F80030D1
:10D4600077EE287AF5EEC07AF1EE10FA00F1268315
:10D470005FEDC16AB6EE007AA7EEA67A49F6807330
:10D48000C0F20103FCEEC77A17EE90EA9E4540F227
:10D4900074839E464FF4507040F22073C2F2010331
:10D4A0001A7ED10700F19981D98BC3F820E081421F
:10D4B00042F0010238BFD8831A7645F6F45017219E
:10D4C000C0F2020012F006FB99F800104FF49663C8
:10D4D00048F21F5203FB01F3C5F2EB1282FB031269
:10D4E0004EF24020D917C1EB2211C2F200000EF01B
:10D4F000FDFB4EF24020C2F200000EF055FCFFF79B
:10D5000027B872B694E80C0010781978637A227AFA
:10D51000194202EA000200F08481A37A03F00303B7
:10D520000AB143F0040343F008039A10082BA272D7
:10D5300000F2A581072B80F02785032B00F0528590
:10D5400040F21486042B00F0A581062B7FF451A92C
:10D55000E368023BE360FFF74DB972B694E80C0054
:10D5600010781978637A227A194202EA000200F0F0
:10D570004F81A37A03F003030AB143F0040343F09D
:10D5800008039A10082BA27200F29981072B80F0F1
:10D59000F084032B00F0BA8540F2F685042B00F0EE
:10D5A0009981062B7FF44BA8E368023BE360FFF709
:10D5B00047B872B694E80C0010781978637A227A2A
:10D5C000194202EA000200F03E81A37A03F003034D
:10D5D0000AB143F0040343F008039A10082BA27227
:10D5E00000F27D81072B80F0F384032B00F0E584AB
:10D5F00040F20586042B00F07D81062B7FF408A8FD
:10D60000E368023BE360FFF704B872B694E80C00ED
:10D6100010781978637A227A194202EA000200F03F
:10D620000981A37A03F003030AB143F0040343F032
:10D6300008039A10082BA27200F23181072B80F0A8
:10D640006085032B00F0A58440F2AC85042B00F02C
:10D650003181062B7FF4F1A8E368023BE360FFF71A
:10D66000EDB872B694E80C0010781978637A227AD3
:10D67000194202EA000200F0C280A37A03F0030319
:10D68000002A41F03B8143F008039A10082BA27254
:10D6900000F23581072B80F0AB83032B00F09D84D3
:10D6A00040F2B585042B00F03581062B7FF4B8A835
:10D6B000E368023BE360FFF7B4B803221A70FFF798
:10D6C000ACBA72B694E80C0010781978637A227AB2
:10D6D000194202EA000200F0BD81A37A03F00303BD
:10D6E0000AB143F0040343F008039A10082BA27216
:10D6F00000F2B981072B80F0E585032B00F0E78568
:10D7000040F2FC85042B00F0B981062B7EF48AAF31
:10D71000E368023BE360FEF786BF72B694E80C0054
:10D7200010781978637A227A194202EA000200F02E
:10D730002E81A37A03F003030AB143F0040343F0FC
:10D7400008039A10082BA27200F29D81072B80F02B
:10D75000A385032B00F0A58540F2D785042B00F0AC
:10D760009D81062B7FF44FA8E368023BE360FFF73F
:10D770004BB80D2B3FF497AD0E2B7EF4A6AFD8F827
:10D780000C300133C8F80C30FEF7A1BFD8F80C30CC
:10D790000233C8F80C30FEF79ABF41F6F042C2F2ED
:10D7A00001020721FFF76EBB40F21C02C2F2010228
:10D7B00005211278197072B69300FFF7A9BA0023F9
:10D7C000C7F6FF73ECE50023C7F6FF73D36100E4EF
:10D7D0000023C7F6FF73FFF7CEBB196A8E4540F2F0
:10D7E0007681DA8BC3F820E0824238BFD88364E6C2
:10D7F000012BC4D0022B3FF456ADFEF766BFA37ACF
:10D8000003F00303002A3FF440AF43F004033CE776
:10D81000A37A03F00303002A3FF4B3AE43F00403FA
:10D82000AFE6A37A03F00303002A3FF47EAE43F091
:10D8300004037AE6A37A03F00303002A3FF4F9AE67
:10D8400043F00403F5E6A37A03F00303002A3FF450
:10D85000C4AE43F00403C0E64DF6A863C2F2000371
:10D860001A79002A40F0ED8472B6E26062B6FFF7E2
:10D87000F3B972B60023E36062B6FFF7EABB0C2B84
:10D8800000F0B08300F27A83092B3FF461AE0B2BDA
:10D890007EF4AFAFE368013BE360FEF7ABBF0C2B58
:10D8A00000F0778300F22784092B3FF4D5AE0B2BD1
:10D8B0007EF4C3AFE368013BE360FEF7BFBF0C2B10
:10D8C00000F0248400F24F83092B3FF46DAE0B2B44
:10D8D0007EF4B5AEE368013BE360FEF7B1BE0C2B0E
:10D8E00000F06B8300F26E83092B3FF489AE0B2BA3
:10D8F0007EF48EAEE368013BE360FEF78ABE0C2B3C
:10D9000000F06B8300F26E82092B3FF4D1AE0B2B3B
:10D910007EF486AFE368013BE360FEF782BF72B638
:10D920000023E36062B6FFF721B872B60023E3601C
:10D9300062B638E472B658F80C2C6368107819781F
:10D94000637A227A194202EA000200F0ED83A37A98
:10D9500003F00303002A40F0E58743F008039A1020
:10D96000082BA27200F2F283072B80F05586032B5E
:10D9700000F03B8640F23286042B00F0F283062B47
:10D980007FF4C9A8E368023BE360FFF7C5B8A37A58
:10D9900003F00303002A3FF4D4AE43F00403D0E6BF
:10D9A00072B658F80C2C636810781978637A227A6A
:10D9B000194202EA000200F0AE83A37A03F00303E7
:10D9C0000AB143F0040343F008039A10082BA27233
:10D9D00000F20584072B80F04186032B00F033868C
:10D9E00040F22A86042B00F00584062B7FF40CAA53
:10D9F000E368023BE360FFF708BA72B658F80C2CF4
:10DA0000636810781978637A227A194202EA000270
:10DA100000F09383A37A03F003030AB143F00403F5
:10DA200043F008039A10082BA27200F2C283072B5E
:10DA300080F0FD85032B00F0E48540F2DB85042BAC
:10DA400000F0C283062B7FF4B8A9E368023BE360D1
:10DA5000FFF7B4B9A37A03F00303002A3FF445AEFD
:10DA600043F0040341E60C2B00F0318400F22484DF
:10DA7000092B3FF44DAE0B2B7EF4D4ADE368013B94
:10DA8000E360FEF7D0BD0C2B00F00B8400F2FE83A8
:10DA9000092B3FF469AE0B2B7EF4B5AEE368013B76
:10DAA000E360FEF7B1BE72B60023E36062B6B9E48C
:10DAB00072B60023E36062B6FFF729BA01204FF087
:10DAC000000EE9E472B60023E36062B63AE491071F
:10DAD000C3F820E006D5596A7F31C909013188426F
:10DAE00038BF0846510706D5996A7F31C909013107
:10DAF000884238BF0846110706D5D96A7F31C9095F
:10DB00000131884238BF0846D10606D5196B7F31EE
:10DB1000C9090131884238BF0846910606D5596BBC
:10DB20007F31C9090131884238BF0846510606D500
:10DB3000996B7F31C9090131884238BF0846D20943
:10DB400006D0DA6B7F32D2090132904238BF1046DC
:10DB5000D883B2E40023C8F20103FFF70CBA002314
:10DB6000C8F201031CE40023C8F20103FFF731BA35
:10DB70000023C8F20103FFF717BA0EF17F00C009B6
:10DB8000013089E472B694E80C0010781978637A51
:10DB9000227A194202EA000240F0BE83A37A03F01F
:10DBA0000303002A40F0C2869A10082BA27200F2EA
:10DBB0001284072B80F01086032B00F0DC8540F2E6
:10DBC000D385042B00F01284062B7FF42BA8E36886
:10DBD000023BE360FFF727B872B694E8060091F8BD
:10DBE00000E01078627A217A10420EEA010140F0DA
:10DBF0007383A27A02F00302002940F08386911019
:10DC0000082AA17200F2F783072A80F0CF85032A41
:10DC100000F0358640F22C86042A00F0F783062AAD
:10DC20007FF41FA8E268023AE260FFF71BB872B601
:10DC300094E80C0010781978637A227A194202EA83
:10DC4000000240F05283A37A03F00303002A40F05D
:10DC50005D869A10082BA27200F27083072B80F069
:10DC60007285032B00F07B8540F27285042B00F057
:10DC70007083062B7FF4F2A9E368023BE360FFF7B1
:10DC8000EEB972B694E80C0010781978637A227AAB
:10DC9000194202EA000240F04883A37A03F003032A
:10DCA000002A40F047869A10082BA27200F26E8379
:10DCB000072B80F0B185032B00F0238540F21985F6
:10DCC000042B00F06E83062B7FF4A4A9E368023BCB
:10DCD000E360FFF7A0B972B658F80C2C63681078AF
:10DCE0001978637A227A194202EA000200F0458329
:10DCF000A37A03F003030AB143F0040343F00803DB
:10DD00009A10082BA27200F22384072B80F0C084A3
:10DD1000032B00F0C98440F2C084042B00F023845C
:10DD2000062B7FF414AAE368023BE360FFF710BA06
:10DD300072B658F80C2C636810781978637A227AD6
:10DD4000194202EA000200F00F83A37A03F00303F2
:10DD50000AB143F0040343F008039A10082BA2729F
:10DD600000F2CD83072B80F07385032B00F06585CF
:10DD700040F25C85042B00F0CD83062B7FF4C8A90C
:10DD8000E368023BE360FFF7C4B972B658F80C2CA5
:10DD9000636810781978637A227A194202EA0002DD
:10DDA00000F00A83A37A03F003030AB143F00403EB
:10DDB00043F008039A10082BA27200F24583072B48
:10DDC00080F0AA84032B00F0B38440F2AA84042BD1
:10DDD00000F04583062B7EF4C4ACE368023BE360AD
:10DDE000FEF7C0BC0D2B3FF495AD0E2B7EF418ADA5
:10DDF000E3680133E360FEF714BD72B694E80C00EB
:10DE000010781978637A227A194202EA000200F047
:10DE1000BF83A37A03F00303002A40F07B8543F01D
:10DE200008039A10082BA27200F2A283072B80F03D
:10DE30004684032B00F0F58440F22685042B00F085
:10DE4000A283062B7FF49BA9E368023BE360FFF704
:10DE500097B972B62046F7F745F8FEF7A9BD72B636
:10DE600094E80C0010781978637A227A194202EA51
:10DE7000000200F0D082A37A03F00303002A40F0EE
:10DE80004D8543F008039A10082BA27200F2CC8251
:10DE9000072B80F07B84032B00F07D8440F20A8501
:10DEA000042B00F0CC82062B7EF472ADE368023BBB
:10DEB000E360FEF76EBD72B694E80C001078197836
:10DEC000637A227A194202EA000200F03883A37AC8
:10DED00003F003030AB143F0040343F008039A106C
:10DEE000082BA27200F21B83072B80F08584032B82
:10DEF00000F0878440F2D084042B00F01B83062BB3
:10DF00007EF439ADE368023BE360FEF735BD72B6DF
:10DF100094E80C0010781978637A227A194202EAA0
:10DF2000000200F0E382A37A03F003030AB143F096
:10DF3000040343F008039A10082BA27200F2C68271
:10DF4000072B80F03E84032B00F04B8440F2AB841F
:10DF5000042B00F0C682062B7EF4F4ACE368023B8F
:10DF6000E360FEF7F0BC0D2B3FF4B4AC0E2B7EF457
:10DF700066ABE3680133E360FEF762BB0D2B3FF451
:10DF800089AC0E2B7EF435ACE3680133E360FEF719
:10DF900031BCE3680233E360FEF750BC72B6002286
:10DFA000E26062B61A790132D2B210461A71029357
:10DFB00002F0A6F9029BFEF74FBEE3680233E3606E
:10DFC000FEF727BB0D2B3FF495AC0E2B7EF420AB58
:10DFD000E3680133E360FEF71CBBE3680233E360F0
:10DFE000FEF71FBCE3680233E360FEF703BC72B6C2
:10DFF00094E80C0010781978637A227A194202EAC0
:10E00000000200F0CE82A37A03F003030AB143F0CA
:10E01000040343F008039A10082BA27200F2248232
:10E02000072B80F05783032B00F0598340F2518473
:10E03000042B00F02482062B7FF4C7A8E368023B80
:10E04000E360FFF7C3B872B694E80C001078197853
:10E05000637A227A194202EA000200F02E82A37A41
:10E0600003F003030AB143F0040343F008039A10DA
:10E07000082BA27200F29E82072B80F0FE82032BF7
:10E0800000F0F18240F22D84042B00F09C82062BDC
:10E090007FF4ABA8E368023BE360FFF7A7B872B672
:10E0A00094E80C0010781978637A227A194202EA0F
:10E0B000000200F0F981A37A03F003030AB143F0F0
:10E0C000040343F008039A10082BA27200F2DC81CB
:10E0D000072B80F0C883032B00F0068340F2F28305
:10E0E000042B00F0DC81062B7FF462A8E368023B7E
:10E0F000E360FFF75EB80D2B3FF4DCAB0E2B7EF434
:10E100009CABE3680133E360FEF798BBE36802333E
:10E11000E360FEF795BAA37A03F00303002A3FF405
:10E1200054AC43F0040350E4A37A03F00303002A41
:10E130003FF415AC43F0040311E4A37A03F00303A6
:10E14000002A3FF46FAC43F004036BE40C2B00F0A7
:10E150004C8200F25B82092B3FF414AC0B2B7EF453
:10E16000DAACE368013BE360FEF7D6BC012B3FF479
:10E170000BAF022B3FF48EABFEF73BBB72B62046D3
:10E18000F6F7B0FEFEF758BD012B3FF4F2AE022BBE
:10E190003FF4A0ABFEF753BA72B62046F6F7A2FEE4
:10E1A000FEF77BBE012BACD0022B3FF483ABFEF716
:10E1B00044BB0C2B00F0258200F23382092B3FF484
:10E1C00044AC0B2B7EF4F9ADE368013BE360FEF752
:10E1D000F5BD72B62046F6F785FEFEF7A0BD0C2B06
:10E1E00000F0318200F23482092B3FF401AC0B2B9A
:10E1F0007EF40AAEE368013BE360FEF706BE012B46
:10E200003FF4E6AE022B3FF475ABFEF701BA012BEB
:10E210003FF4EEAD022B3FF47DABFEF701BB72B6CF
:10E220002046F6F75FFEFEF705BF72B62046F6F70A
:10E2300059FEFEF7AEBF72B62046F6F753FEFFF763
:10E240006FB872B67C22E26062B61A79013AABE628
:10E2500072B62046F6F746FEFFF7E9B872B62046DA
:10E26000F6F740FEFFF7CCB872B62046F6F73AFE56
:10E27000FFF76DB872B62046F6F734FEFEF74CBED7
:10E2800072B62046F6F72EFEFEF72FBE0D2B3FF49A
:10E2900005AC0E2B7EF4B7AAE3680133E360FEF70A
:10E2A000B3BAE3680233E360FEF7AEBA72B6204653
:10E2B000F6F718FEFEF750BB0D2B3FF4DFAB0E2B2D
:10E2C0007EF4B0A9E3680133E360FEF7ACB9E3681C
:10E2D0000233E360FEF7A7B9A27A02F0030209B1A4
:10E2E00042F0040242F0080289E4A37A03F0030337
:10E2F0000AB143F0040343F00803AAE4012BE1D080
:10E30000022B3FF4BBABFEF78DB9012BC4D0022B1F
:10E310003FF4C4ABFEF777BAA37A03F003030AB164
:10E3200043F0040343F008033EE4A37A03F003033D
:10E330000AB143F0040343F00803B4E40C2B00F0EB
:10E340000E8200F2FA81092B3FF496AC0B2B7EF47F
:10E3500085AEE368013BE360FEF781BE72B62046FE
:10E36000F6F7C0FDFEF7CBBDA37A03F00303002A46
:10E370003FF4F3AC43F00403EFE4A37A03F00303A8
:10E38000002A3FF4BDAC43F00403B9E40C2B00F0C9
:10E39000B88100F23B82092B3FF498AC0B2B7EF442
:10E3A00039AEE368013BE360FEF735BE72B6204646
:10E3B000F6F798FDFEF7BEBFA37A03F00303002A29
:10E3C0003FF4F8AC43F00403F4E472B62046F6F7E9
:10E3D00089FDFFF71FB80C2B00F0CD8100F2F6810C
:10E3E000092B3FF4F4AB0B2B7EF41CACE368013B30
:10E3F000E360FEF718BC0C2A00F0418200F2D081E5
:10E40000092A3FF40FAC0B2A7EF42BACE268013AE8
:10E41000E260FEF727BCA37A03F00303002A3FF46F
:10E4200032AD43F004032EE50C2B00F0B48100F272
:10E43000A781092B3FF43AAD0B2B7EF4A9AAE36820
:10E44000013BE360FEF7A5BA0C2B00F0718100F2EE
:10E450005D81092B3FF4C1AC0B2B7EF482A9E368EC
:10E46000013BE360FEF77EB90C2B00F0388100F22F
:10E470002B81092B3FF4E2AD0B2B7EF4A6AEE368B3
:10E48000013BE360FEF7A2BE0C2B00F02D8100F2F1
:10E49000E481092B3FF42AAE0B2B7EF489AEE368AE
:10E4A000013BE360FEF785BEA37A03F00303002A75
:10E4B0003FF409AE43F0040305E6A37A03F0030337
:10E4C000002A3FF4D4AD43F00403D0E50C2B00F058
:10E4D000888100F27081092B3FF440AD0B2B7EF454
:10E4E00031AAE368013BE360FEF72DBAA37A03F09B
:10E4F0000303002A3FF41FAD43F004031BE50C2B7C
:10E5000000F09B8100F29E81092B3FF439AC0B2B6C
:10E510007EF4FEADE368013BE360FEF7FABD0C2B31
:10E5200000F06F8100F26281092B3FF4EBAC0B2B02
:10E530007EF421AAE368013BE360FEF71DBAA37AEB
:10E5400003F00303002A3FF4CAAC43F00403C6E41B
:10E550000C2B00F0A98000F29580092B3FF4E3AB6F
:10E560000B2B7EF4F4ADE368013BE360FEF7F0BDF6
:10E570000C2B00F0568100F29C80092B3FF464AC18
:10E580000B2B7EF4FCADE368013BE360FEF7F8BDC6
:10E59000A37A03F00303002A3FF443AC43F00403DF
:10E5A0003FE4A37A03F00303002A3FF434AD43F0C1
:10E5B000040330E50C2B56D05AD8092B3FF46AAD32
:10E5C0000B2B7EF412AEE368013BE360FEF70EBE58
:10E5D00072B62046F6F786FCFEF77CBE012B1BD0F8
:10E5E000022B3FF4BEADFEF796BAE3680233E36058
:10E5F000FEF792BA012B1AD0022B3FF4E5ADFEF7DD
:10E60000DCBBE3680233E360FEF7D8BB0D2B3FF4BD
:10E61000A8AD0E2B7EF47FAAE3680133E360FEF71A
:10E620007BBA0D2B3FF4D0AD0E2B7EF4C6ABE36866
:10E630000133E360FEF7C2BB012B0FD0022B3FF486
:10E64000D9ADFEF7E1BBE3680233E360FEF7DDBB63
:10E650000D2B3FF4CFAD0E2B7EF4D6ABE368013328
:10E66000E360FEF7D2BBE3680233E360FEF7BEBDB2
:10E670000D2BA8D00E2B7EF4B8ADE3680133E36018
:10E68000FEF7B4BD0D2B3FF46EAF0E2B7EF45FADE5
:10E69000E3680133E360FEF75BBD012BF8D0022B8A
:10E6A0003FF461AFFEF753BDE3680233E360FEF76A
:10E6B0004FBD0D2B3FF467AF0E2B7EF460ADE368CA
:10E6C0000133E360FEF75CBD0D2B3FF4D8AE0E2B9B
:10E6D0007EF47BADE3680133E360FEF777BDE3686A
:10E6E0000233E360FEF772BDE3680233E360FEF7D6
:10E6F00060BD012B00F09080022B3FF452AEFEF77C
:10E7000089BCE3680233E360FEF785BC0D2B3FF460
:10E71000A6AE0E2B7EF425A8E3680133E360FEF776
:10E7200021B8012BF8D0022B3FF499AEFEF719B8AF
:10E73000E3680233E360FEF715B80D2B3FF409AE32
:10E740000E2B7EF48BACE3680133E360FEF787BCED
:10E75000012BF8D0022B3FF4FCADFEF77FBCE36841
:10E760000233E360FEF77BBC012B35D0022B3FF474
:10E770003DAEFEF757BAE3680233E360FEF753BAE3
:10E780000D2B3FF45CAE0E2B7EF402A9E36801333F
:10E79000E360FEF7FEB8E3680233E360FEF7F9B822
:10E7A0000D2A3FF433AE0E2A7EF45BAAE2680132F2
:10E7B000E260FEF757BA0D2B3FF493AE0E2B7EF4BA
:10E7C000C1A8E3680133E360FEF7BDB80D2B3FF449
:10E7D0000DAE0E2B7EF426AAE3680133E360FEF74C
:10E7E00022BAE3680233E360FEF7ADB80D2B3FF4C5
:10E7F000A1AE0E2B7EF4BFA8E3680133E360FEF701
:10E80000BBB8E3680233E360FEF7B6B80D2B3FF404
:10E81000C8AD0E2B7EF4FEABE3680133E360FEF778
:10E82000FABBE3680233E360FEF7AABC012B0FD00A
:10E83000022B3FF46FAEFEF76BBCE3680233E3607C
:10E84000FEF767BC0D2B3FF465AE0E2B7EF460AC7B
:10E85000E3680133E360FEF75CBC0D2B3FF41FAEB1
:10E860000E2B7EF4A5ACE3680133E360FEF7A1BC98
:10E87000012A9BD0022A3FF4C9ADFEF7F2B9E26843
:10E880000232E260FEF7EEB9012B3FF418AF022B23
:10E890003FF479AEFEF773BC012BADD0022B3FF4F1
:10E8A00049AEFEF768B8012B8BD0022B3FF419AEAE
:10E8B000FEF748B8012B3FF469AF022B3FF4BFAD20
:10E8C000FEF766B8012BCED0022B3FF4E8ADFEF781
:10E8D0006FBC012B3FF4FEAE022B3FF4D0ADFEF730
:10E8E00074BC012B3FF4C9AE022B3FF46CAEFEF7B3
:10E8F0007CBC0023C7F6FF73FEF76BBB43F0040339
:10E90000FEF7C1BE42F00402FFF779B943F00403F9
:10E91000FFF79FB943F00403FFF781BA43F0040304
:10E92000FFF7AFBA43F00403FFF717B843F004034F
:10E93000FFF73AB943F00403FFF7B5B92DE9F04307
:10E940002DED028B0546002783B000F1F004204630
:10E9500085F8D97085F8DA7085F8DB7085F8DC7099
:10E9600085F8DD7085F8DE7085F8DF7085F8E07079
:10E9700085F8E17085F8E27085F8E37085F8E47059
:10E9800085F8E57085F8E67085F8E77085F8E87039
:10E9900085F8CC7085F8CD7085F8CE700191FAF7C6
:10E9A000FDFE45F65061AD22C0F2020105F5B670DC
:10E9B0000DF0A0FC102385F8193202F0F7FF03F0E8
:10E9C00045F803F00BFDDDED017AB8EEE78A2E463F
:10E9D000B0EE480A03F002FBB0EE480A03F04AFB2F
:10E9E000B0EE480A03F026FCB0EE480A02F0E0FD63
:10E9F00001992046FAF7DAFE4FF409700DF008FF8E
:10EA00000446F1F73DFDC5F85C424FF409700DF086
:10EA1000FFFE45F27803C0F202030360C5F860020E
:10EA20004FF409700DF0F4FE46F22423C0F2020305
:10EA3000C5F85802036005F1C0092C464FF4257053
:10EA40000DF0E6FE80460C3402F03EF844F8048CEB
:10EA500004F80A7C04F8097C04F8087CA1454FF00E
:10EA60000003EBD195F8D9209FEDD06ADFEDCE6A97
:10EA700085F81A3207EE902AB8EEE77A95F8DB208F
:10EA8000C5F8C43067EE067A102067EEA67A4FF418
:10EA90000051FCEEE77AC5F8C830CDED017A85F873
:10EAA000D23085F8D13085F8D03085F8CF3085F870
:10EAB000CE3085F8CD3085F8CC3085F819029DF838
:10EAC0000430C5F8C0100AB185F8CC3095F8DA20CA
:10EAD0000AB185F8CD3095F8DC200AB185F8CE3042
:10EAE00095F8E1309FEDB16ADFEDAF6A95F8E3107C
:10EAF00007EE903AB8EEE77A67EE067A67EEA67A06
:10EB0000FCEEE77ACDED017A9DF8043031B195F84D
:10EB1000CC10994238BF194685F8CC1095F8E21010
:10EB200031B195F8CD10994238BF194685F8CD100E
:10EB300095F8E40030B195F8CE108B4238BF0B4603
:10EB400085F8CE3095F8DD309FED986ADFED966A56
:10EB500095F8DF1007EE903AB8EEE77A67EE067A9E
:10EB600067EEA67AFCEEE77ACDED017A9DF80430E7
:10EB700031B195F8CC10994238BF194685F8CC10C0
:10EB800095F8DE1031B195F8CD10994238BF19468D
:10EB900085F8CD1095F8E01031B195F8CE40A3423C
:10EBA00038BF234685F8CE3095F8E5309FED7F6A73
:10EBB000DFED7D6A95F8E74007EE903AB8EEE77A28
:10EBC00067EE067A67EEA67AFCEEE77ACDED017A7B
:10EBD0009DF8043034B195F8CC409C4238BF1C46B7
:10EBE00085F8CC4095F8E64034B195F8CD409C428C
:10EBF00038BF1C4685F8CD4095F8E84034B195F80B
:10EC0000CE70BB4238BF3B4685F8CE302AB921B919
:10EC100018B914B97F2385F8CE303F23002485F836
:10EC2000D830C5F8D44005F2F51105F5107003F0A1
:10EC300037FA95F81C320BB185F81C4295F81E3254
:10EC4000002485F81B42002B00F0EF80D5F85832E5
:10EC500085F81E42C5F8EC3033793BB1B368B47027
:10EC600018463471F4700BB102F088FC0C36B145D3
:10EC7000F2D195F8D9309FED4D6A95F8DB1007EE8B
:10EC8000903A95F8D230B8EEE77A06EE903A67EE11
:10EC9000067AF8EEE66A002267EEA67A85F8CE20BC
:10ECA000FCEEE77A85F8CD20CDED017A9DF80430B1
:10ECB00085F8CC2009B185F8CC3095F8DA200AB176
:10ECC00085F8CD3095F8DC200AB185F8CE3095F87E
:10ECD000E1309FED366A95F8E31007EE903A95F82B
:10ECE000D030B8EEE77A06EE903A67EE067AF8EEA4
:10ECF000E66A67EEA67AFCEEE77ACDED017A9DF83A
:10ED0000043031B195F8CC10994238BF194685F8D6
:10ED1000CC1095F8E21031B195F8CD10994238BF7A
:10ED2000194685F8CD1095F8E40030B195F8CE106D
:10ED30008B4238BF0B4685F8CE3095F8DD309FED1D
:10ED40001B6A95F8DF1007EE903A95F8D130B8EECF
:10ED5000E77A06EE903A67EE067AF8EEE66A67EE34
:10ED6000A67AFCEEE77ACDED017A9DF8043031B158
:10ED700095F8CC10994238BF194685F8CC1095F813
:10ED8000DE1031B195F8CD10994238BF194685F89B
:10ED9000CD1095F8E01059B195F8CE40A34238BF98
:10EDA000234685F8CE3003E0000000000AD7233C5C
:10EDB00095F8E5301FED036A95F8E74007EE903AC5
:10EDC00095F8CF30B8EEE77A06EE903A67EE067A1D
:10EDD000F8EEE66A67EEA67AFCEEE77ACDED017A08
:10EDE0009DF8043034B195F8CC409C4238BF1C46A5
:10EDF00085F8CC4095F8E64034B195F8CD409C427A
:10EE000038BF1C4685F8CD4095F8E84034B195F8F8
:10EE1000CE60B34238BF334685F8CE302AB921B927
:10EE200018B914B97F2385F8CE30284603B0BDEC5D
:10EE3000028BBDE8F08300BF2DE9F04F2DED028B72
:10EE40008B00CDB00A3302AF23F007037961ADEB3D
:10EE5000030D90F81D127A6002AB06463B6139B390
:10EE600090F81932DBB1002400F5B67503E00134E7
:10EE7000A4B2A34213D904EB440206EB8201087941
:10EE80000028F4D04B78886816F82220294602F032
:10EE90003BF9013496F81932A4B2A342EBD806F23A
:10EEA000F51106F5107003F0FBF8002386F81D320B
:10EEB0007B69002B00F0AB8007F1270840F22004AB
:10EEC00006F510739FED588ABB6028F00F08C2F258
:10EED00001044FF0000A3B694FF4807203EB8A098A
:10EEE0000021404615F03CFC00214FF4807248465A
:10EEF00015F036FCBD68284603F014F98346284611
:10EF000003F06AF996F81912002955D0C7F80CA039
:10EF10000025824603E00135EDB28D424AD205EB71
:10EF2000450306EB83031A79002AF4D0986806F1AA
:10EF3000C00300935A465346414601F09DFFA8F195
:10EF4000040308F1FC0E4A46F7EE006ABFEE006AC1
:10EF500000200DE0216801312160B7EE007AD2ED8A
:10EF6000007A186037EE877A7345A2EC017A1BD0DD
:10EF700053F8041F091121F35721491007EE901A85
:10EF8000F8EEE77A87EE887AB4EEE67AF1EE10FAD8
:10EF9000E0DCB4EEC67AF1EE10FAE0D5216801317A
:10EFA0002160BFEE007ADAE796F819120135EDB26A
:10EFB0008D42B4D3D7F80CA07B690AF1400A1FFA3E
:10EFC0008AFA534587D83C691D4606F1F0001A4677
:10EFD0002146FAF76DFC7A689FED137A681E80B2BD
:10EFE00002EB40002146023AF1EC017A67EE877AA3
:10EFF000FDEEE77A17EE903A22F8023F8242F3D113
:10F0000007F59677BD46BDEC028BBDE8F08F3969F8
:10F010001A4606F1F000FAF74BFC07F59677BD4665
:10F02000BDEC028BBDE8F08F00FEFF462DE9F843F2
:10F03000054690F8FC3190F81962002A00F0D6805D
:10F04000183BCF1890F81A82FFB2002E00F0C5804E
:10F050004FEA480909EB080300EB830341469C781B
:10F06000CE46002C00F09380002403E08378002B30
:10F0700000F08D800131013491FBF6F306FB131192
:10F08000E4B24FEA410E0EEB0100B44205EB800002
:10F090005FFA81F8EAD195F81C32002B6ED095F812
:10F0A0001932002B6AD02A79002A40F0CF81012B37
:10F0B00064D92A7C002A40F0D781022B5ED02A7FB7
:10F0C000002A40F0CD81032B58D095F82820002A43
:10F0D00040F0C881042B51D095F83420002A40F02C
:10F0E000B781052B4AD095F84020002A40F0B28124
:10F0F000062B43D095F84C20002A40F0AD81072B19
:10F100003CD095F85820002A40F0A881082B35D033
:10F1100095F86420002A40F0AB81092B2ED095F899
:10F120007020002A40F0A6810A2B27D095F87C2079
:10F13000002A40F0A1810B2B20D095F88820002ACE
:10F1400040F09C810C2B19D095F89420002A40F0B7
:10F1500097810D2B12D095F8A020002A40F09281C3
:10F160000E2B0BD095F8AC20002A40F07F810F2B9E
:10F1700004D095F8B830002B40F032814FEA4809AE
:10F18000C84405EB880501232B71BDE8F8838E4444
:10F190004FEA8E0E013105EB0E0991FBF6F306FBEB
:10F1A000131685F81A6205F80E7089F8012095F893
:10F1B0001B3289F803300121134689F80210D9F86F
:10F1C00008003A4605F5B67101F098FC95F8F4315F
:10F1D000002B78D1002C7FF45EAF05F5107003F0A2
:10F1E00021F895F81C32002BC8D058E7183BCF18EF
:10F1F000FBB2002E65D00178994200F0BB80012E51
:10F200005FD92A7B9A4200F0AF80022E59D02A7E25
:10F210009A4200F0A380032E53D095F824209A42FE
:10F2200000F09580042E4CD095F830209A4200F0E2
:10F230008780052E45D095F83C209A427AD0062E3C
:10F240003FD095F848209A426ED0072E39D095F8D5
:10F2500054209A4262D0082E33D095F860209A420A
:10F2600056D0092E2DD095F86C209A424AD00A2EFD
:10F2700027D095F878209A423ED00B2E21D095F8D1
:10F2800084209A4232D00C2E1BD095F890209A42BE
:10F2900026D00D2E15D095F89C209A421AD00E2E0D
:10F2A0000FD095F8A8209A4200F093800F2E08D036
:10F2B00095F8B4209A4204D195F8B630002B40F06E
:10F2C000A780BDE8F883D9F8080002F057F9002CB0
:10F2D00083D0E0E695F89E20002AE0D00D2798E044
:10F2E00095F89220002AD4D00C2792E095F8862039
:10F2F000002AC8D00B278CE095F87A20002ABCD0D1
:10F300000A2786E095F86E20002AB0D0092780E011
:10F3100095F86220002AA4D008277AE095F85620B4
:10F32000002A98D0072774E095F84A20002A8CD04C
:10F3300006276EE095F83E20002A80D0052768E079
:10F3400095F83220002A3FF474AF042761E095F865
:10F350002620002A3FF466AF03275AE0AA7E002A3F
:10F360003FF459AF022754E0AA7B002A3FF44DAF87
:10F3700001274EE0817800293FF441AF82701746A3
:10F38000804695F81C32E3B14FF0000E734671468B
:10F390004FF0FF3203EB430305EB8304481CA478D2
:10F3A0002CB115F823309342C4BF5AB28E4641B2F5
:10F3B000B1420B46EEDB013203D098F80430002B4B
:10F3C00062D195F81B32C3B3012388F80330BDE83E
:10F3D000F88395F8AA20002A3FF468AF0E2718E0BA
:10F3E0000F2303EB43039B00EA189178C9B1EB5C50
:10F3F000BB42BFF466AF4FEA480909EB080305EBCF
:10F400008303002111719868916802F063F8B7E6F0
:10F410000F2707EB470805EB8808002388F8023020
:10F42000AFE74FEA480909EB080305EB83031171C5
:10F430009868916802F06EF8A2E607EB470205EBC8
:10F440008205A868BDE8F84301F04ABE0023C8E77A
:10F450000423C6E70523C4E70623C2E70723C0E762
:10F460000223BEE70323BCE70123BAE70E23B8E774
:10F470000823B6E70923B4E70A23B2E70B23B0E772
:10F480000C23AEE70D23ACE70EEB4E0E07EB470265
:10F4900005EB8E03002105EB820288F804100121A0
:10F4A00019719868916802F015F88AE7F8B590F834
:10F4B000FC3190F81972183B1944002F63D003787F
:10F4C000C9B28B4260D0012F5DD9037B8B4200F023
:10F4D000EA80022F57D0037E8B4200F0DE80032F9C
:10F4E00051D090F824308B4200F0D080042F4AD0C5
:10F4F00090F830308B4200F0C280052F43D090F856
:10F500003C308B4200F0B480062F3CD090F848305D
:10F510008B4200F0A680072F35D090F854308B42F4
:10F5200000F09880082F2ED090F860308B4200F0C9
:10F530008A80092F27D090F86C308B427CD00A2F1C
:10F5400021D090F878308B4270D00B2F1BD090F8E0
:10F5500084308B4264D00C2F15D090F890308B42C1
:10F5600058D00D2F0FD090F89C308B424CD00E2FDE
:10F5700009D090F8A8308B4240D00F2F03D090F8DC
:10F58000B4308B422ED0F8BD8378002B9BD0002561
:10F590008570064690F81C320446E3B100231A46F3
:10F5A0009C464FF0FF3E03EB430304EB8300511CEA
:10F5B000807830B114F823307345C4BF4FFA83FE0E
:10F5C00094464AB2BA421346EDDBBEF1FF3F02D089
:10F5D0003379002B76D194F81B32002B69D00123AC
:10F5E000F370F8BD90F8B630002BCCD00F2505EBAA
:10F5F000450600EB86060023B370CBE790F8AA30EF
:10F60000002BBAD00E25F2E790F89E30002BAED03A
:10F610000D25ECE790F89230002BA2D00C25E6E700
:10F6200090F88630002B96D00B25E0E790F87A30E2
:10F63000002B8AD00A25DAE790F86E30002B3FF4D1
:10F640007EAF0925D3E790F86230002B3FF471AF0D
:10F650000825CCE790F85630002B3FF463AF072520
:10F66000C5E790F84A30002B3FF455AF0625BEE7BA
:10F6700090F83E30002B3FF447AF0525B7E790F8F0
:10F680003230002B3FF439AF0425B0E790F8263034
:10F69000002B3FF42BAF0325A9E7837E002B3FF41B
:10F6A0001EAF0225A3E7837B002B3FF412AF012599
:10F6B0009DE705EB450504EB8500BDE8F840806853
:10F6C00001F00EBD0CEB4C0C05EB450204EB8C037A
:10F6D000002104EB8202317101211971986891684F
:10F6E00001F0F8FE77E700BF012380F81D32704774
:10F6F00090F81C328B4218BF80F81C12704700BF74
:10F7000090F81B328B4218BF80F81B12704700BF65
:10F7100090F81B02704700BF70B5044600F1C006A8
:10F72000002523793BB1A368A57018462571E570C3
:10F730000BB101F023FF0C34B442F2D170BD00BF15
:10F7400090F8D9309FED6C6ADFED6C6A90F8DB10B1
:10F7500007EE903AB8EEE77A70B467EE067A83B0B7
:10F7600067EEA67A0023FCEEE77A4FF40052CDED67
:10F77000017AC0F8C020C0F8C4309DF80420C0F859
:10F78000C83080F8D23080F8D13080F8D03080F89E
:10F79000CF3080F8CE3080F8CD3080F8CC3009B151
:10F7A00080F8CC2090F8DA300BB180F8CD2090F8BA
:10F7B000DC1009B180F8CE2090F8E1309FED4E6A60
:10F7C000DFED4E6A90F8E32007EE903AB8EEE77A64
:10F7D00067EE067A67EEA67AFCEEE77ACDED017A5F
:10F7E0009DF8043032B190F8CC209A4238BF1A46C6
:10F7F00080F8CC2090F8E22032B190F8CD209A42E7
:10F8000038BF1A4680F8CD2090F8E44034B190F823
:10F81000CE20934238BF134680F8CE3090F8DD30CA
:10F820009FED356ADFED356A90F8DF2007EE903AFC
:10F83000B8EEE77A67EE067A67EEA67AFCEEE77A2C
:10F84000CDED017A9DF8043032B190F8CC209A4287
:10F8500038BF1A4680F8CC2090F8DE2032B190F8FC
:10F86000CD209A4238BF1A4680F8CD2090F8E0208B
:10F8700032B190F8CE50AB4238BF2B4680F8CE3034
:10F8800090F8E5309FED1C6ADFED1C6A90F8E750B8
:10F8900007EE903AB8EEE77A67EE067A67EEA67A58
:10F8A000FCEEE77ACDED017A9DF8043035B190F8A1
:10F8B000CC509D4238BF1D4680F8CC5090F8E650A1
:10F8C00035B190F8CD509D4238BF1D4680F8CD50DF
:10F8D00090F8E85035B190F8CE60B34238BF334667
:10F8E00080F8CE3029B922B91CB915B97F2380F828
:10F8F000CE3003B070BC70470AD7233C0000000034
:10F9000003791BB18378002B40F09A80037C1BB1F4
:10F91000837B002B40F09180037F1BB1837E002B03
:10F9200040F0888090F828301BB190F82630002BEA
:10F930007CD190F834301BB190F83230002B71D16B
:10F9400090F840301BB190F83E30002B66D190F813
:10F950004C301BB190F84A30002B5BD190F85830F6
:10F960001BB190F85630002B50D190F864301BB189
:10F9700090F86230002B45D190F8703013B190F8B8
:10F980006E30DBBB90F87C3013B190F87A308BBBD3
:10F9900090F8883013B190F886303BBB90F89430E3
:10F9A00013B190F89230EBB990F8A03013B190F801
:10F9B0009E309BB990F8AC3013B190F8AA304BB997
:10F9C00090F8B8302BB190F8B63013B1002380F81E
:10F9D000B6307047002380F8AA30F1E7002380F8A2
:10F9E0009E30E7E7002380F89230DDE7002380F8BF
:10F9F0008630D3E7002380F87A30C9E7002380F807
:10FA00006E30BFE7002380F86230B5E7002380F84E
:10FA10005630AAE7002380F84A309FE7002380F899
:10FA20003E3094E7002380F8323089E7002380F8E5
:10FA300026307EE70023837674E7002383736BE729
:10FA40000023837062E700BF90F81902704700BF7F
:10FA50002DE9F04F054690F8F211D0F8EC0085B092
:10FA600002F030F995F81912002900F0C780C0F3B0
:10FA7000C0030093C0F3001300260193C0F34013AA
:10FA8000344600F00108C0F3400BC0F3800A029333
:10FA900005F5087703E00134E4B2A1427CD904EB18
:10FAA000440305EB830999F80420002AF3D00021D0
:10FAB0002022384614F054FE3946D9F8080001F0E7
:10FAC000CBFCB8F1000F6BD0D5F8201240F22D42DC
:10FAD000914269D895F83812A1F10401B1FA81F187
:10FAE000022049090122BBF1000F0AD0D5F82422D7
:10FAF00040F22D4E724503D895F83922042A57D08A
:10FB00000246BAF1000F0DD0D5F8280240F22D4E72
:10FB100001327045D2B205D895F83A02042804BFE4
:10FB20000131C9B2009B6BB1D5F82C0240F22D4EC9
:10FB300001327045D2B205D895F83B02042804BFC3
:10FB40000131C9B2019B6BB1D5F8300240F22D4EA4
:10FB500001327045D2B205D895F83C02042804BFA2
:10FB60000131C9B2029B6BB1D5F8340240F22D4E7F
:10FB700001327045D2B205D895F83D02042804BF81
:10FB80000131C9B2914217D095F819120134E4B28B
:10FB90000136A142F6B282D8304605B0BDE8F08FFA
:10FBA0000120424641469EE70220012200219AE7B9
:10FBB0000131C9B20246A4E7002245F6007089F877
:10FBC000042089F8032089F802201021C0F20200E5
:10FBD00003920FF07FFF039A4EF240201346214616
:10FBE0000A22C2F200000CF0F1F84EF24020C2F2FC
:10FBF00000000CF0D9F895F819124CE70E46CBE747
:10FC00002DE9F04100F5B67384B004460A4600F5CC
:10FC1000F575106856685E6018601089967A9E7255
:10FC20001881D07A00F00306C0F38100DE721873E9
:10FC3000107BC0F3C30600F007001E755873507B9D
:10FC4000C0F3820600F00300DE739873907B187493
:10FC5000D07BC0F3440600F001009E745874107C01
:10FC6000D87415339D4202F11102D2D10B460A46D7
:10FC700053F8660FDFEDD25A5B68C4F8EA016B6097
:10FC800091F86E3003F01F0384F8F23191F86F3071
:10FC9000C3F3C00003F0070384F8F40184F8F331E0
:10FCA0000B6FC4F8F53191F87430C3F30115C3F349
:10FCB000420003F0010384F8FB5184F8FA0184F850
:10FCC000F93191F8753084F8FC3152F8761F04F25E
:10FCD000FD175368C4F8FD117B6013893B816322D3
:10FCE0000123072184F8073284F8083284F80922B6
:10FCF00084F80B2284F80D2284F80F2284F80A126B
:10FD000084F80C1284F80E1284F8101294F8D010B3
:10FD100084F8123206EE101A94F8D21084F81332D6
:10FD200006EE901A94F8D11084F81432B8EEC66A30
:10FD3000F8EEE66A07EE101A26EE256A94F8CF1060
:10FD400084F8153266EEA56AB8EEC77A07EE901A07
:10FD5000BCEEC66AFCEEE66A27EE257A8DED016AF6
:10FD6000CDED026AF8EEE77A9DF804009DF80810E0
:10FD700084F81632BCEEC77A67EEA57A88428DED1C
:10FD8000037A38BF0846FCEEE77A9DF80C10CDEDFB
:10FD9000017A884238BF08469DF8041084F817326B
:10FDA0008842C4F8C430C4F8C83084F8D92084F834
:10FDB000DA3084F8DB3084F8DC3084F8DD2084F835
:10FDC000DE3084F8DF3084F8E03084F8E12084F815
:10FDD000E23084F8E33084F8E43084F8E52084F8F5
:10FDE000E63084F8E73084F8E830237938BF0846F5
:10FDF000102500213F2284F8CC0084F81112C4F8A9
:10FE0000D41084F8185284F8CD0084F8CE0084F819
:10FE1000D8201BB1A378002B40F0A381237C1BB119
:10FE2000A37B002B40F09A81237F1BB1A37E002B84
:10FE300040F0918194F8283023B194F82630002BBB
:10FE400040F0858194F8343023B194F83230002B9F
:10FE500040F0798194F8403023B194F83E30002B83
:10FE600040F06D8194F84C3023B194F84A30002B67
:10FE700040F0618194F8583023B194F85630002B4B
:10FE800040F0558194F8643023B194F86230002B2F
:10FE900040F0758194F8703023B194F86E30002BE7
:10FEA00040F0698194F87C3023B194F87A30002BCB
:10FEB00040F05D8194F8883023B194F88630002BAF
:10FEC00040F0518194F8943023B194F89230002B93
:10FED00040F05D8194F8A03023B194F89E30002B5F
:10FEE00040F0518194F8AC3023B194F8AA30002B43
:10FEF00040F0518194F8B83023B194F8B630002B1B
:10FF000040F01181102384F81932254604F1C0080D
:10FF100000262B793BB1AB68AE7018462E71EE709F
:10FF20000BB101F02BFB0C354545F2D194F8D930DB
:10FF30009FED246A94F8DB1007EE903A94F8D230E3
:10FF4000B8EEE77A06EE903A67EE067AF8EEE66AE1
:10FF5000002267EEA67A84F8CE20FCEEE77A84F8D9
:10FF6000CD20CDED017A9DF8043084F8CC2009B184
:10FF700084F8CC3094F8DA20002A40F0288194F8F4
:10FF8000DC200AB184F8CE3094F8E1309FED0D6AA0
:10FF900094F8E31007EE903A94F8D030B8EEE77A90
:10FFA00006EE903A67EE067AF8EEE66A67EEA67A13
:10FFB000FCEEE77ACDED017A9DF8043004E000BF55
:10FFC000A3707D3F0AD7233C31B194F8CC109942FD
:10FFD00038BF194684F8CC1094F8E210002940F09C
:10FFE000EE8094F8E41031B194F8CE00834238BF2B
:10FFF000034684F8CE3094F8DD301FED0E6A94F895
:020000021000EC
:10000000DF0007EE903A94F8D130B8EEE77A06EECA
:10001000903A67EE067AF8EEE66A67EEA67AFCEEAC
:10002000E77ACDED017A9DF8043030B194F8CC0038
:10003000984238BF184684F8CC0094F8DE000028B7
:1000400040F0B58094F8E00030B194F8CE50AB4267
:1000500038BF2B4684F8CE3094F8E5301FED276A80
:1000600094F8E75007EE903A94F8CF30B8EEE77A7C
:1000700006EE903A67EE067AF8EEE66A67EEA67A42
:10008000FCEEE77ACDED017A9DF8043035B194F8B5
:10009000CC509D4238BF1D4684F8CC5094F8E650B1
:1000A000002D7CD194F8E85035B194F8CE60B3427D
:1000B00038BF334684F8CE302AB920B919B915B9FA
:1000C0007F2384F8CE30012541F654600A22394658
:1000D00084F81D52C2F2010014F0E0FC45F61470E1
:1000E0000721C0F202000FF0F5FC41F65460C2F2A5
:1000F000010014F065FC014641F65460C2F20100B3
:100100000FF0E8FC45F61C700921C0F202000FF068
:10011000E1FC4EF24020C2F200000BF045FE284602
:1001200004B0BDE8F081002384F8B630EAE600238D
:1001300084F85630A6E6002384F84A309AE6002375
:1001400084F83E308EE6002384F8323082E60023C5
:1001500084F8263076E60023A3766BE60023A373AB
:1001600062E6A1705AE6002384F88630AAE60023EE
:1001700084F87A309EE6002384F86E3092E60023FD
:1001800084F8623086E6002384F89E30AAE60023D5
:1001900084F892309EE6002384F8AA30AAE694F808
:1001A000CD509D4238BF1D4684F8CD507AE794F873
:1001B000CD00984238BF184684F8CD0042E794F845
:1001C000CD10994238BF194684F8CD1009E784F85C
:1001D000CD30D4E610B5044614F0F2FB01462046BB
:1001E000BDE810400FF076BC10B5044614F0E8FBF3
:1001F000014620460FF06EFC04464EF24020C2F24B
:1002000000000BF0D1FD204410BD00BF2DE9F041EE
:1002100000262F270C468E600E604E60C1F80B60E2
:100220000A2201F8017B804613F09EFF204614F05D
:10023000C7FB08EB480540F23002C2F2010208EBAE
:1002400085051544431C27542946E01814F054FB37
:100250004EF2402745F62870C2F200072121C0F275
:1002600002000FF037FC33460A22414638460BF0B5
:10027000ADFD45F64C700A21C0F202000FF02AFCD9
:10028000284614F09DFB014628460FF023FC45F656
:1002900068200321C0F202000FF01CFC204614F07D
:1002A0008FFB014620460FF015FC45F21860C0F2A6
:1002B000020001210FF00EFC3846BDE8F0410BF0C2
:1002C00073BD00BF10B584B00C460146684614F0FB
:1002D00013FB45F624716846C0F2020114F012FCCB
:1002E00028B10146204614F007FB04B010BD45F6C6
:1002F0005873C0F2020303CB2060616004B010BDEC
:100300002DE9F04194B0044604A804F083FB41F6C3
:10031000F440C2F201004FF4B072002114F020FA50
:1003200041F25C53C2F201031B7833B904A804F014
:100330007FFB002014B0BDE8F08148F21F53C5F2E6
:10034000EB13A3FB04235B09642000FB1340C0B242
:100350006946FFF75BFF45F660701E21C0F20200A0
:100360000FF0B8FB684614F02BFB014668460FF00F
:10037000B1FB45F218600121C0F202000FF0AAFBA8
:100380004EF24020C2F200000BF00EFD49F21401C3
:1003900001236A460CA8C2F2010104F017FC14AB59
:1003A0009DF8344053F8131DCDF81D105A689E680F
:1003B0001D7B0E99CDF82120139B9DF83C20CDF894
:1003C00025600CA88DF829508DF8144006918DF801
:1003D0001C200B9304F02CFB04A804F043FB002822
:1003E000A4D004A804F03AFB41F2080398420DD0CF
:1003F00045F680701A21C0F202000FF06BFB4EF23E
:100400004020C2F200000BF0CFFC8FE704A804F0FC
:1004100071FAF0280DD045F69C701F21C0F2020041
:100420000FF058FB4EF24020C2F200000BF0BCFC73
:100430007CE704A804F05EFA43280DD045F6BC70B2
:100440001C21C0F202000FF045FB4EF24020C2F228
:1004500000000BF0A9FC69E741F2070104A804F0D1
:10046000F3FA04A804F046FAF72806D045F6DC7043
:10047000C0F20200FFF7B8FE58E7032104A804F019
:10048000E3FA04A804F036FA092806D045F6FC7011
:10049000C0F20200FFF7A8FE48E741F2060104A8F7
:1004A00004F0D2FA04A804F025FA062146B204A802
:1004B00004F0CAFA04A804F01DFA002741F6F44536
:1004C00002463C46B846C2F2010516E004F012FAB4
:1004D00004F07F0108EB880308EB43030246A1F117
:1004E000760009282B449CBF5B1803F8762C7F29E3
:1004F00004BF08F101085FFA88F80134A4B2D2B24F
:10050000B4F5805F04A8A7EB0207DFD146F21C0018
:10051000C0F20200FFF75EFE07F07F074EF24020B8
:10052000394600231022C2F200000BF04FFC46F2C5
:100530003000C0F20200FFF74DFE4EF240200023D3
:1005400010223146C2F200000BF040FC45F2186068
:10055000C0F20200FFF748FEB7423FF4E7AE46F2B2
:100560003800C0F20200FFF735FE4EF24020394657
:1005700000231022C2F200000BF028FC46F25800C3
:10058000C0F20200FFF726FE4EF240203146002363
:100590001022C2F200000BF019FC4EF24020C2F211
:1005A00000000BF001FCC1E62DE9F04192B002A879
:1005B00004F030FA40F23000C2F2010040F214526E
:1005C000002114F0CDF841F25C53C2F201031C7813
:1005D000002C00F09E8040F23006C2F2010600249A
:1005E00008E00AA804F024FA02A804F03BFA002864
:1005F00000F08F802F2300250A220DF105012046EF
:1006000001958DF8043013F0AFFD49F21401C2F2E8
:100610000101012301AA0AA804F0D8FA9DF82CE0F0
:100620000C9D9DF834709DF836009DF837109DF8AC
:1006300038209DF839309DF83AC09DF835808DF806
:100640000CE004959DF83BE08DF814709DF83D504A
:100650009DF83C708DF816008DF817109DF83E003F
:100660009DF83F108DF818208DF819309DF8402026
:100670009DF841308DF81F108DF820208DF81AC09C
:100680008DF81BE08DF81E008DF815808DF81C701C
:100690008DF81D508DF821300AA8119B099304F0A4
:1006A000C7F902A804F0DEF9012202A988B30AA85A
:1006B00004F004FB0AA804F0BFF9002891D10AA8AD
:1006C00004F0B8F904EB440504EB85053544014614
:1006D000284614F011F946F260000C21C0F2020025
:1006E0000FF0F8F9284614F06BF9014628460FF090
:1006F000F1F945F218600121C0F202000FF0EAF9A9
:100700004EF24020C2F2000001340BF04DFBE4B287
:1007100067E702A804F08CF9204612B0BDE8F0812A
:100720002DE9F0470E469046054604F097F941F250
:10073000080398420FD045F68070C0F202001A21DB
:100740000FF0C8F94EF24020C2F200000BF02CFB73
:100750000020BDE8F087284604F0CCF8F02805D04A
:1007600045F69C70C0F202001F21E9E7284604F01C
:10077000C1F8432805D045F6BC70C0F202001C2128
:10078000DEE741F20701284604F05EF9284604F04E
:10079000B1F8F72805D045F6DC70C0F202001D2143
:1007A000CEE70321284604F04FF9284604F0A2F8CA
:1007B000092804D045F6FC70C0F20200EFE741F2D0
:1007C0000601284604F040F9284604F093F8062173
:1007D0004FFA80F9284604F037F906F1010A00249F
:1007E0004FEACA1AF6012746284604F083F8B442B5
:1007F000C3B2A7EB030704DBA31B5445B8BF08F83B
:1008000003000134B4F5805FEED146F21C001221E2
:10081000C0F202000FF05EF907F07F074EF24020B1
:10082000002310223946C2F200000BF0CFFA46F244
:1008300030000421C0F202000FF04CF94EF24020CB
:10084000002310224946C2F200000BF0BFFA45F225
:1008500018600121C0F202000FF03CF94EF2402076
:10086000C2F200000BF0A0FA4F4508D140F22C0371
:10087000C2F2010300221A800120BDE8F08746F28F
:1008800038001F21C0F202000FF024F94EF2402080
:10089000394600231022C2F200000BF097FA46F20C
:1008A00058000621C0F202000FF014F94EF2402069
:1008B000494600231022C2F200000BF087FA4EF2E4
:1008C0004020C2F200000BF06FFA0020BDE8F08774
:1008D00030B541F25C52C2F20102B5B01378002B80
:1008E00000F09C80044604A80D4604F093F848F2FA
:1008F0001F53C5F2EB13A3FB04235B09642000FB29
:100900001340C0B26946FFF781FC49F2140101238C
:100910006A4614A8C2F2010104F058F934AB9DF8FC
:10092000544053F8732DCDF81D2059689A681B7BED
:10093000CDF82110CDF8252016999DF85C208DF872
:10094000293014A81B9B8DF8144006918DF81C20AB
:100950000B9304F06DF804A804F084F8044600BB7F
:1009600046F270001021C0F202000FF0B3F86846A2
:1009700014F026F8014668460FF0ACF846F2840001
:10098000C0F2020008210FF0A5F84EF24020C2F29A
:1009900000000BF009FA04A804F04AF8204635B02C
:1009A00030BDDDF82130DDF81D20CDF84130DDF817
:1009B0002530CDF84530CDF83D209DF82930069AF8
:1009C0008DF849300E929DF814308DF8343046F28F
:1009D000F8629DF81C308DF83C30C0F2020205F040
:1009E0001F050B9B0C9229460CA814AA1393FFF722
:1009F00097FE04460CA804F01BF804BB46F2A000C6
:100A00001A21C0F202000FF065F84EF24020C2F247
:100A100000000BF0C9F904A804F00AF846F2BC0083
:100A20001321C0F202000FF055F84EF24020C2F23E
:100A300000000BF0B9F90024204635B030BD0A2281
:100A40000DF1C6010CA814F029F846F290000E2111
:100A5000C0F202000FF03EF8684613F0B1FF014605
:100A600068460FF037F845F688300221C0F20200E0
:100A70000FF030F805EB850341F6F44005EB430534
:100A8000C2F201000544284613F09AFF01462846A9
:100A90000FF020F845F218600121C0F202000FF0BB
:100AA00019F84EF24020C2F200000BF07DF941F23D
:100AB0009053C2F2010314A91868FFF7A1F8044685
:100AC00069E700BF0BF072BB0022C0F8A421C0F898
:100AD0009C21C0F8B421C0F8AC21C0F8C421C0F8F2
:100AE000BC21C0F8D421C0F8CC21C0F8E421C0F862
:100AF000DC21C0F8F421C0F8EC2170472DE9F04F5B
:100B000045F255541646C0F2150404FB06F49A4605
:100B100004F142732DED088B08EE903A4FF04E53DE
:100B20000AEE103A4CF28303CBF6CA6309EE903A10
:100B300043F27A63C3F6AB4309EE103A4DF20A73FF
:100B4000C3F623430BEE103A4AF63B23C4F6B83300
:100B500045F256550AEE903A18EE903AC5F25555C0
:100B600093B085FB022703F231733246A7EBE67799
:100B700046F2181B08EE903A4FEA6A030395814645
:100B8000073F08930C460546C0F2020B0026099168
:100B900090464EE0BAF1000F00F30F816FF0EE01C6
:100BA00001FB02F20732D21000EB0213002F23EAFE
:100BB000E373627B40F3FF801F2FCCBFC2EB421276
:100BC0007A43D21000920AA90EAA09EB060000F09F
:100BD00007FD627CA37CE17C207D002A7AD003F0B3
:100BE000030C4FF0640E40F678031EFB0C11C0F2AC
:100BF000440303FB01F307284FEAE301C3BF0738AF
:100C000043F29143434300230B44C5F86C22C5F8DB
:100C10003032A37B03F0030344365BF82330C5F87E
:100C20005432B6F5CC7F04F1150405F1040500F04B
:100C3000D48020782179627863790A90A0780E9127
:100C40000B92A179E2780F930C90E379207C0D92BE
:100C50001193109100F01EFE237AC3EB0803B3F149
:100C6000110200F18680039A217B94F80AE0103B80
:100C700082FB03C2A2EBE37301B303291ED01F2B37
:100C8000DBBF46F2A812C0F20202FA23D35C03FBD8
:100C90000EFE40F2491303FB0EF301294FEAE33342
:100CA00016DD18447F28A8BF7F20BAF17F0F4FEAD6
:100CB0004010E27B7FF76EAF0F2171E703FB0EF36D
:100CC00040F2491202FB03F301294FEA2333E8DC27
:100CD0005B42E6E7B8EEE88A079028EE0A0A06913A
:100CE00020EE290A0593049210F08AF920EE090AF1
:100CF000F1EE0C7A80EE277A0798059B0699073863
:100D000046F2281E03F01F03C0F2020E5EF82330E5
:100D100007EE900A27EE087AF8EEE77AA7EE278A20
:100D2000BDEEC88A18EE102A1A441346049A002908
:100D30003FF46BAF07EE901AF8EEE77AB7EE000AD1
:100D4000A7EE8B0A059310F0DDF9F6EE007AE0EEDF
:100D50002A7A17EE900A12F019FE41EC100B0FF0F0
:100D60002BFC51EC100B13F015F9059B049A03446E
:100D70004BE7039B94F809C0C2F10101E27A83FBBF
:100D8000013EAEEBE17102B3032A1ED01F29DBBF87
:100D900046F2A81EC0F2020EFA211EF8011040F21F
:100DA000491301FB0CF103FB01F3DB13012A3FF7AD
:100DB00078AF5B4275E7002204E746F2D003C0F249
:100DC00002030899595CEF39EAE601FB0CF140F2A5
:100DD000491303FB01F31B13E8E7DDF8248098F8BF
:100DE0007E5098F8824098F87F3098F8830098F801
:100DF00080600A950E9498F8845098F881400B937F
:100E00000F9098F8853011930EAA0AA909F5FC7085
:100E10000C9610950D9401F029FA98F88630C9F8CF
:100E2000883298F887302BB3C3F10803C9F85032E1
:100E300098F88B3003EB830303EB43139B11C9F842
:100E40008C3298F88F3046F21012C0F2020203F092
:100E50000703D35CC9F8903298F88C3003EB830316
:100E600003EB43139B11C9F8843213B0BDEC088B1C
:100E7000BDE8F08F1023D9E72DE9F04F2DED048B5D
:100E800089B0D0F89052DDF8588007918146D0F8AB
:100E90008C0298F80DE09B46A2F5000305FB03F5D4
:100EA00000FB0BF0A0FB0567EB1700FB0377144674
:100EB0008EFB0523900B40EA8340FE1186EAE67321
:100EC00080EAE072A2EBE072A3EBE6739342B8BF54
:100ED000134609F5FC701E4601F000FAD8F8003000
:100EE000002DB4BF4FF0FF320122B3F5005A06FBCC
:100EF00002001AD0D8F80820002A40F0D980D8F88B
:100F000004304FEACA2A07EE90AA07EE103AF8EE2C
:100F1000E77AB8EEC77AF2EE086A67EE877A87EE6C
:100F2000A67AFDEEC77A17EE90AA4FF05A5309EE53
:100F3000103A45F62943C3F68F53D9F8842298F81E
:100F40000C1008EE903A43F23333C4F2431308EE28
:100F5000103A82FB0B23C4F180744FEA122B4BEA48
:100F6000036BE3170BFB03F298F80E30002704FB2A
:100F700007225B04ABFB046781FB0445C3F57E0BD2
:100F8000E30943EA45635B4517444FEA166138BFFE
:100F90005B4641EA0721D8F814208B4238BF0B4644
:100FA00092449B4600EB0A0305934E4609F50C74E8
:100FB0004F46002514E0504401F040F8C6F8A00167
:100FC000384600F065FB626A02BBC6F8980101353D
:100FD000062D07F1440706F1100604F1040452D06F
:100FE00098F818302B4113F0010344D0E36B2068CC
:100FF000002BE0D1059B184401F020F8C6F8A001B1
:10100000384600F045FB626A002ADED0D117ABFB00
:101010000223CDE90223039A06900BFB01230393DD
:10102000DDE90201020E42EA012207EE902AF8EE03
:10103000677AB0EE480A67EE897AA7EEA80A0FF041
:10104000DFFFFCEEC07A069817EE901AC3174FEA3E
:10105000011E0EFB03F3090F00FB0131AEFB002361
:10106000CDE902230B440393029B1A0F039B42EA30
:101070000312801AA9E73846029300F009FB029B8D
:10108000C6F89831A3E7D8F82C00D9F850120268B6
:10109000D9F88832019109F5127100919468079985
:1010A00009F5CC72A04709B0BDEC048BBDE8F08F08
:1010B00021230C21C8F2040391FBF2F202FB0AFA8D
:1010C00083FB0A1353444FEAEA7ACAEB233A41F608
:1010D000FF7393FBF2F303FB0AFA4FEACA2A24E7F1
:1010E00070B50646044600F5CC7520460021443410
:1010F00000F080FBAC42F8D106F5FC700021BDE8A1
:10110000704001F039B900BF2DE9F04F45F2555458
:101110009246C0F2150404FB0AF4994604F14273A6
:101120002DED088B08EE903A4FF04E530AEE103A30
:101130004CF28303CBF6CA6309EE903A43F27A632A
:10114000C3F6AB4309EE103A4DF20A73C3F62343DC
:101150000BEE103A4AF63B23C4F6B83345F2565527
:101160000AEE903A18EE903AC5F2555593B085FBC9
:101170000A2803F23173A8EBEA7846F2181B08EE4E
:10118000903A4FEA69030295074607900891A8F143
:10119000070809930C460546C0F2020B00262AE018
:1011A000B9F1000F00F312816FF0EE0101FB02F2C2
:1011B0000732D21000EB0213B8F1000F23EAE373F9
:1011C000627B40F30181B8F11F0FCCBFC2EB42122A
:1011D00008FB02F2D2100092384601360EAA0AA984
:1011E00000F062FB062E04F1150405F1040507F179
:1011F000440700F0FB80627CA37CE17C207D002A18
:1012000071D003F0030C4FF0640E40F678031EFB20
:101210000C11C0F2440303FB01F307284FEAE3017A
:10122000C3BF073843F29143434300230B44C5F83F
:101230003032A37BC5F86C2203F003035BF8233044
:10124000C5F8543220782179627863790A90A078C1
:101250000E910B92A179E2780F930C90E379207CA8
:101260000D921193109100F015FB237AC3EB0A0342
:10127000B3F1110200F18680029A217B94F80AE012
:10128000103B82FB03C2A2EBE37301B303291ED020
:101290001F2BDBBF46F2A812C0F20202FA23D35C76
:1012A00003FB0EFE40F2491303FB0EF301294FEA44
:1012B000E33316DD18447F28A8BF7F20B9F17F0FE4
:1012C0004FEA4010E27B7FF76BAF0F216EE703FB25
:1012D0000EF340F2491202FB03F301294FEA2333D4
:1012E000E8DC5B42E6E7B8EEE88A069028EE0A0AF8
:1012F000059120EE290A049303920FF081FE20EE5F
:10130000090AF1EE0C7A80EE277A0698049B05997B
:10131000073846F2281E03F01F03C0F2020E5EF8E3
:10132000233007EE900A27EE087AF8EEE77AA7EE68
:10133000278ABDEEC88A18EE102A1A441346039A6B
:1013400000293FF474AF07EE901AF8EEE77AB7EE93
:10135000000AA7EE8B0A04930FF0D4FEF6EE007A93
:10136000E0EE2A7A17EE900A12F010FB41EC100B17
:101370000FF022F951EC100B12F00CFE049B039AB3
:10138000034454E7029B94F809C0C2F10101E27AD8
:1013900083FB013EAEEBE17102B3032A1ED01F298D
:1013A000DBBF46F2A81EC0F2020EFA211EF80110A1
:1013B00040F2491301FB0CF103FB01F3DB13012A9B
:1013C0003FF778AF5B4275E7002204E746F2D003AF
:1013D000C0F202030999595CEF39E7E601FB0CF111
:1013E00040F2491303FB01F31B13E8E7089A07993E
:1013F00092F88630C1F8883292F887303BB3C3F157
:10140000080308461446C0F8503294F88B3003EBBA
:10141000830303EB43139B11C0F88C3294F88F3095
:1014200046F21012C0F2020203F00703D35CC0F8C8
:10143000903294F88C3003EB830303EB43139B113E
:10144000C0F8843213B0BDEC088BBDE8F08F1023D8
:1014500008461446D7E700BF2DE9F84F43F66C7AEB
:10146000804689460646A1F1040B01F1180500F1FA
:1014700060070446C2F2010AD4F8981101F17241E2
:101480004A1340F2FE731340581C5AF823205AF8AE
:101490002000C1F30D0382FB0323920B42EA834237
:1014A0000916C1F1060102440A41304629461034AA
:1014B0004BF8042F00F050FAA74205F1010506F1A0
:1014C0004406D9D109F11E0108F5FC70BDE8F84FBA
:1014D00000F080BF2DE9F04104460F4600F5CC78BE
:1014E00006460D463946204600F03AFAD5F89C31BA
:1014F000C6F89C314434D5F8A431C6F8A43144452B
:1015000007F1440705F1100506F11006EAD1BDE820
:10151000F08100BFD1F8AC31D1F8A42110B4D1F8DA
:101520009C41C0F89C41C0F8A421C0F8AC31D1F86E
:10153000B431C0F8B431D1F8BC31C0F8BC31D1F805
:10154000C431C0F8C431D1F8CC31C0F8CC31D1F8B5
:10155000D431C0F8D431D1F8DC31C0F8DC31D1F865
:10156000E431C0F8E431D1F8EC31C0F8EC31D1F815
:10157000F431C0F8F4315DF8044B70470023C0F833
:101580009C31C0F8A431C0F8AC31C0F8B431C0F817
:10159000BC31C0F8C431C0F8CC31C0F8D431C0F887
:1015A000DC31C0F8E431C0F8EC31C0F8F4317047F8
:1015B0004FF48843C4F22C7307EE103A87EE000A0A
:1015C0004FF0974307EE903A20EE270A4DF6BC63A2
:1015D000BCEEC00AC2F2000383ED000A704700BFF0
:1015E00030B40C680460146804614D684560556847
:1015F00045618D68856095688561C968C160D268FC
:10160000C261132C4FF0000282624263DBBF46F2DC
:10161000CC12C0F202021C3452F82440036264105F
:1016200003EB8413A3F58553026802994162102BE2
:1016300002EB8204B8BF102302EBC4021B04002B90
:1016400001EBA212D4BF0024012401253E2A80F818
:101650004050C36280F8304016DC02F00303921061
:101660000433083203FA02F2D3174DF6BC61C2F21A
:1016700000010968A1FB024501FB0355230E43EA63
:101680000523836330BC70474FF060720023ECE7A2
:10169000426B022AF0B4034605DD032A66D190F8B6
:1016A0004010002962D193F8301071B9986A996B93
:1016B000DC6A401AA042986259DC511C03299C62E2
:1016C00059635BDD2046F0BC70474FF6FF70996AA6
:1016D000C0F2B36081424CDDC1F1885000169D6BB1
:1016E000DC6A05FB0010A042986240DB511C032914
:1016F0009C625963E6DC03EB820251691329DBBF6C
:1017000046F2CC10C0F2020001F11C0550F8215045
:10171000196A586A6D1001EB8511A1F585511029E0
:10172000B8BF102109048C42ACBF00250125D96245
:1017300083F83050526802EB820102EBC10200EBE9
:10174000A2123E2A4CDD4FF0607600274DF6BC62B7
:10175000C2F2000220461268A2FB064502FB0755B2
:10176000220E42EA05229A63F0BC7047986AF0BCE8
:1017700070470021C0F2B4610A20B0E703EB820297
:1017800051691329DBBF46F2CC10C0F2020001F10F
:101790001C0550F82150196A586A6D1001EB85112B
:1017A000A1F585511029B8BF102109048C42ACBFA6
:1017B00000250125D96283F83050526802EB82017E
:1017C00002EBC10200EBA2103E28BCDC00F00306D5
:1017D00080100436083006FA00F00646C717B5E751
:1017E00002F0030692100436083206FA02F2164698
:1017F000D717ABE790F840308B4241D000290CBF9F
:101800000323002330B49D00421980F84010436345
:101810001369816A132BDBBF46F2CC12C0F20202BD
:1018200003F11C0452F82340036A426A641003EB7C
:101830008413A3F58553102BB8BF10231B048B42D0
:10184000D4BF0021012180F83010C362435903EB5B
:10185000830103EBC10302EBA3123E2A11DD4FF01B
:10186000607200234DF6BC61C2F200010968A1FB61
:10187000024501FB0355230E43EA052330BC836375
:10188000704702F0030392100433083203FA02F2A5
:10189000D317E7E71328DBBF46F2CC13C0F20203ED
:1018A0001C3053F82000704730B40C680460146892
:1018B00004614C684460546844618C688460946836
:1018C0008461C968C16090F84010D568029AC5610A
:1018D00003624262002934D0132CDBBF46F2CC11E4
:1018E000C0F202011C3451F824408568816A6410FA
:1018F00003EB8413A3F58553102BB8BF102305EB1E
:1019000085041B0405EBC4058B4202EBA512D4BF72
:101910000021012102243E2AC36280F83010446372
:1019200011DD4FF0607200234DF6BC61C2F2000180
:101930000968A1FB024501FB0355230E43EA052379
:10194000836330BC704702F0030322410433083242
:1019500003FA02F2D317E7E7436B0B70704700BF3F
:101960000A680B69036102604B6843604B6943611D
:101970008B6883608B698361CB68C360F0B5CB698A
:10198000C3610B6A4F6A8E6ACD6A91F830E04C6B86
:101990008A6B036291F8403047628662C56280F8C4
:1019A00030E04463826380F84030F0BD70B54FF0A2
:1019B0009D432DED048B08EE103A41F23063002177
:1019C00043F66C74C3F680730020C4F2D01108EEA5
:1019D000903AC2F201040025B6EE009A0BE078EED0
:1019E000097A17EE900A11F0D1FF41EC100B0EF0BE
:1019F000E3FD51EC100B6E0012F0CCFA013601350C
:101A0000B5F5806F28EE288A44F82600E7D1002338
:101A100040F2FF355A00D11C501C54F8211054F8E4
:101A200020000133091AAB4243F66C7044F82210CF
:101A3000C2F20100EED141F6FC73BDEC048BC35839
:101A400041F6F872C3F10043835070BD002207EEE7
:101A5000902A4FF0974202EE102A4FF06C5204EE9B
:101A6000902A4FF06E5202EE902A4AF6AB22C3F64D
:101A70002A2241F66C7303EE102AC2F201030022FF
:101A8000F6EE003AB7EE006AB0EE004AF0EE465AC3
:101A9000E7EEE75A03EBC2010132B0EE677AA5EE3A
:101AA000A47AB2F5806FB0EE465AA7EE475AF0EE30
:101AB000636AE7EE826AB0EE677AA5EE247AFDEEFD
:101AC000E66AC1ED016AF0EE466AE7EE476AB0EEFB
:101AD000677AA6EEA27A76EE856AB0EE465AA7EE4F
:101AE000475A35EE257AA6EE847AE7EE037ACDD111
:101AF00030B4002240F2FF355100C81C4C1C53F892
:101B0000200053F824400132001BAA4241F66C74B5
:101B100043F82100C2F20104EED14FF0974306EEE4
:101B2000903AB6EE007AA7EEA67A41F6FC7341F63B
:101B3000F872E358FDEEC77A17EE901ACB1AA3504D
:101B400030BC7047704700BF2DE9F04F46F230249B
:101B500091B003EB4303C0F2020404EBC304154647
:101B6000069007910FCC0AAE0FC694E8030000233D
:101B700086E803004FF0010843F66C760AAF05F1E2
:101B800060098DF824808DF825308DF82630C2F25A
:101B9000010605973BE00AF1FF30069B00EB0010C1
:101BA00003EB0010133020F00F0095E8084003F11C
:101BB000724B4FEA6B3340F2FE721A40531C56F8D8
:101BC000222056F82340CBF30D0382FB0323920B14
:101BD0004FEA2B6B42EA8342CBF1060B144444FAE2
:101BE0000BF4BEF58C6F6C601CDAB4F58C6F19DAEF
:101BF000BCF1000F03D110AB9A440AF81CCCEB687F
:101C0000AA6803EB8213EB601035A9452FD0059B22
:101C100053F8041B059311F0030A01F0040CBAD128
:101C20000798C2E710AB9A441AF81C3C1BB11CF190
:101C3000000318BF0123C1F301123AB110AF07EB43
:101C4000020C1CF81CCCBCF1000F13D101F0C00138
:101C5000C02902D11B9A0F2A20DDAA68E9680193E6
:101C60000094734600F0D6F80AF81C8CC7E711B050
:101C7000BDE8F08F0699D5F808C0013A02EB0212D0
:101C800001EB02111331EA68029321F00F01634660
:101C90000194CDF800E000F051F8E5E71746E96857
:101CA000AA6802971A9F03938DE89000734600F08C
:101CB0000FF9D9E710B54FF4097104460AF0AAFDEF
:101CC000204610BD46F23023F0B401EB4101C0F2D2
:101CD000020303EBC1040FCC86B06D460FC5074667
:101CE0000B4694E80300C7F3800485E8030013F073
:101CF000040F44F0020314BF18462046164640F075
:101D00000403039A049916F0040F18BF184640F014
:101D1000080312F0040F059A18BF184611F0040FBB
:101D200040F0100308BF034612F0040F43F02000F8
:101D300008BF184606B0F0BC704700BF2DE9F04F51
:101D4000099E0A9C9DF82C50C6EB040C0CF1200C4B
:101D50009E464FEAAC1C46F6787785B3C2F201077F
:101D60004FF0400B4FF0000A51F82A4014444FEA5C
:101D7000643840F2FE7508EA0505C4F30D0457F80F
:101D80002530013583FB048957F8255050F82A3057
:101D90004FEA983444EA89442C44664484FB06891B
:101DA0004FEA186444EA09242344BBF1010B40F8CC
:101DB0002A3072440AF1010AD6D1BDE8F08FAA4652
:101DC000C2F201074FF0400B51F82A3013445D1363
:101DD00040F2FE742C40C3F30D0357F82450013435
:101DE00085FB038957F824404FEA983343EA894337
:101DF0001C44664484FB0645230E43EA0523BBF1DD
:101E0000010B40F82A3072440AF1010ADCD1BDE826
:101E1000F08F00BF2DE9F043079C9DF82050C3EBE5
:101E2000040C0CF1200C4FEAAC1C46F6787E4DB346
